:100000000C94C5320C94F6320C94F6320C94F63201
:100010000C94F6320C948DAD0C94F6320C94F632AE
:100020000C941EB10C94F6320C94E08D0C94F632C4
:100030000C94F6320C94F6320D94F94C0D94B059A0
:100040000C94F6320C94D1DD0C94F6320C94F6320A
:100050000C94F6320C94F6320C94F6320D943B0765
:100060000C94F6320D942B550C94F6320C94F63217
:100070000C94F6320C94F6320C94F6320C94F63260
:100080000C94F6320C94F6320C94F6320C94F63250
:100090000D94E7540C94F6320C94F6320C94F6322C
:1000A0000C94F6320C94F6320C94F6320C94F63230
:1000B0000C94F6320C94F6320C94F6320C94F63220
:1000C0000C94F6320C94F6320C94F6320D94EF58F0
:1000D0000C94F6320C94F6320C94F6320C94F63200
:1000E0000C94F632254E2B4E314E3C4E474ECC4EA4
:1000F000524E5B4E644E6F4E7A4E854E954EA04EDC
:10010000CC4EAB4EB64EC14E938C978C9D8CA68C2C
:10011000BF8CDC8C198D508D25A22FA2D2A1A0A15D
:100120006FA124A552A282A32BA485A4A1A4D8A424
:1001300031CB47CB5ACB67CB71CB9FCBC0CBC5CB99
:10014000D3CBD6CBD8CBE2CBF3CB04CC8501970174
:10015000730149017F01390165015D01E701A501D5
:10016000E501BD017B0135013901B101B501A101F5
:100170006F01A3014101AB014B017901F70153016B
:1001800047019101DD01CD01CD01A701CD01A701FD
:10019000E1016101084AD73B3BCE016E84BCBFFD43
:1001A000C12F3D6C74319ABD56833DDA3D00C77F47
:1001B00011BED9E4BB4C3E916BAAAABE00000080E0
:1001C0003F05A84CCDB2D44EB93836A9020C50B96F
:1001D000918688083CA6AAAA2ABE000000803F0794
:1001E000634236B79BD8A71A39685618AEBAAB55D2
:1001F0008C1D3CB7CC5763BD6DEDFD753EF6177297
:1002000031BF000000803F08000000BE9224491268
:100210003EABAAAA2ABECDCCCC4C3E00000080BE8C
:10022000ABAAAAAA3E00000000BF000000803F0069
:1002300000000000084178D3BB4387D1133D190E5D
:100240003CC3BD4282AD2B3E68EC8276BED98FE1C5
:10025000A93E4C80EFFFBE01C4FF7F3F00000000BD
:1002600000000D943C950D9447420D9455050D9456
:100270000F3E0D9468050D945F440D9423060D9474
:100280000F060D947D0E0D949C540D9428060D942C
:10029000D30E0D9424050D94AB0E0D94393B0D94A3
:1002A000533A0D9483540D94C50E0D94423F0D9412
:1002B000F7050D94FD3D0D948E940D9439050D9424
:1002C000603A0D9409440D9438060D9435050D944B
:1002D000543F0D94438F0D947E390D9478050D9401
:1002E000690E0D94A53F0D9420050D94F5630D94B2
:1002F000C5920D94B10E0D9451050D94063E0D94CA
:100300002A050D9403060D9450940D942E050D941A
:1003100009060D945FA90D9458390D94158F0D940D
:10032000FD050D94E10E0D94D5930D9469050D9482
:1003300031050D94B03B0D9474390D9423B50D9493
:10034000AB940D9463050D94770E0D9443050D94B5
:1003500003440D94F43D0D948F0E0D947E440D9442
:1003600047930D945B050D94C8940D945F050D940F
:1003700018400D94B6400D9419060D944D050D943A
:1003800002950D9454900D94E5940D9414060D94DB
:100390009A440D9485440D9461940D9400440D94F9
:1003A000A1440D9470940D945B0B0D9475440D94C1
:1003B00049440D94F1900D94E78E0D94F80E0D9430
:1003C000D1380D9406440D9493440D9447050D9433
:1003D0003F050D94A28F0D941E060D9473050D9488
:1003E00092930D948C440D9402940D946D050D948C
:1003F000B70E0D94F1050D94CC900D941F956E6180
:100400006E00696E66004E414E494E495459494E40
:1004100046CDCCCC3D0AD7233C17B7D13877CC2B6F
:10042000329595E6241FB14F0A000020410000C814
:100430004200401C4620BCBE4CCA1B0E5AAEC59D95
:100440007400407A10F35A00A0724E18090010A5EB
:10045000D4E80000E87648170000E40B54020000DE
:10046000CA9A3B000000E1F5050000809698000064
:100470000040420F000000A086010000001027008D
:10048000000000E803000000006400000000000A13
:1004900000000000000100000000002C76D888DC7D
:1004A000674F0823DFC1DFAE59E1B1B796E5E3E45A
:1004B00053C63AE651997696E8E6C28426EB898CD3
:1004C0009B62ED407C6FFCEFBC9C9F40F2BAA56F35
:1004D000A5F490055A2AF75C936B6CF9676DC11B04
:1004E000FCE0E40D47FEF520E6B500D0ED902E03CC
:1004F00000943577050080841E080000204E0A0015
:100500000000C80C333333330F986E12831141EF60
:100510008D2114893BE65516CFFEE6DB18D1844BBE
:10052000381BF77C1D901DA4BBE424203284725E2E
:10053000228100C9F124ECA1E53D276364696E6F57
:1005400070737578585B0025642062797465732038
:100550007772697474656E20746F20454550524FF0
:100560004D20617420616464726573732030782556
:10057000303478004433202D20526561642F577247
:1005800069746520454550524F4D0A0020436F75F0
:100590006E7420583A20005344207072696E74695A
:1005A0006E67206279746520004E6F7420696E203A
:1005B0006661726D206D6F64652E004163746976AB
:1005C000652045787472756465723A2000496E76CC
:1005D000616C6964206578747275646572005A2074
:1005E0004F666673657400556E6B6E6F776E206331
:1005F0006F6D6D616E643A2022004D3230302049BB
:100600006E76616C696420657874727564657220B9
:10061000007A5F6D61783A20007A5F6D696E3A20EA
:1006200000795F6D61783A2000795F6D696E3A20DC
:1006300000785F6D61783A20006F70656E005452EB
:100640004947474552454400785F6D696E3A20003E
:100650005265706F7274696E6720656E6473746F33
:100660007020737461747573000053494C454E5487
:10067000004E4F524D414C002553204D4F44453ABA
:100680002050657263656E7420646F6E653A202534
:10069000643B207072696E742074696D65207265A8
:1006A0006D61696E696E6720696E206D696E733A5F
:1006B0002025640A00456E642066696C65206C69BB
:1006C000737400426567696E2066696C65206C69A9
:1006D0007374000A50494E44412074656D70657210
:1006E00061747572653A20252E3166205A20736830
:1006F00069667420286D6D293A20252E3366000A1C
:10070000537465703A2025642F360A000A537465C5
:10071000703A2025642F362028736B6970706564E9
:10072000290A50494E44412074656D7065726174A8
:100730007572653A202564205A20736869667420B2
:10074000286D6D293A300A000A5A45524F3A202541
:100750002E33660A0073746172742074656D70655F
:100760007261747572653A20252E31660A0025641F
:100770002020252E326600255320583A20252E357C
:100780006620593A20252E3566205A3A20252E35E6
:10079000660A00536C6565702E2E2E004E6F742015
:1007A000696E206661726D206D6F64652E00256430
:1007B0000045303A25642052504D0A50524E303A8E
:1007C00025642052504D0A002564004175746F0065
:1007D00020452F443D00416476616E6365204B3DAA
:1007E000004D3232302053256900255346696C6133
:1007F0006D656E742073657474696E67733A204416
:10080000697361626C65640A00255346696C616DA9
:10081000656E742073657474696E67733A0A255344
:100820002020204D3230302044252E32660A00250B
:1008300053526574726163743A20533D4C656E6720
:10084000746820286D6D2920463A537065656420D0
:10085000286D6D2F6D29205A3A205A4C69667420F4
:10086000286D6D290A25532020204D323037205322
:10087000252E32662046252E3266205A252E3266D7
:100880000A25535265636F7665723A20533D457869
:10089000747261206C656E67746820286D6D292004
:1008A000463A537065656420286D6D2F6D290A25C1
:1008B000532020204D3230382053252E32662046DA
:1008C000252E32660A25534175746F2D5265747258
:1008D0006163743A20533D3020746F206469736102
:1008E000626C652C203120746F20696E74657270A3
:1008F00072657420657874727564652D6F6E6C799D
:10090000206D6F7665732061732072657472616308
:100910007473206F72207265636F76657269657398
:100920000A25532020204D323039205325640A00F7
:10093000255350494420686561746265642073657D
:100940007474696E67733A0A25532020204D333042
:10095000342050252E32662049252E32662044252B
:100960002E32660A00255350494420736574746919
:100970006E67733A0A25532020204D3330312050C2
:10098000252E32662049252E32662044252E3266D9
:100990000A00255353746570732070657220756E5C
:1009A00069743A0A255320204D39322058252E32B9
:1009B000662059252E3266205A252E32662045257E
:1009C0002E32660A25534D6178696D756D20666516
:1009D00065647261746573202D206E6F726D616C39
:1009E00020286D6D2F73293A0A255320204D32306F
:1009F000332058252E32662059252E3266205A255E
:100A00002E32662045252E32660A25534D617869BF
:100A10006D756D20666565647261746573202D2047
:100A2000737465616C746820286D6D2F73293A0AA0
:100A3000255320204D3230332058252E3266205940
:100A4000252E3266205A252E32662045252E326606
:100A50000A25534D6178696D756D20616363656C1E
:100A600065726174696F6E202D206E6F726D616C9E
:100A700020286D6D2F7332293A0A255320204D32DC
:100A800030312058256C752059256C75205A256CFD
:100A9000752045256C750A25534D6178696D756D16
:100AA00020616363656C65726174696F6E202D20CF
:100AB000737465616C746820286D6D2F7332293AE8
:100AC0000A255320204D3230312058256C7520598D
:100AD000256C75205A256C752045256C750A2553A3
:100AE000416363656C65726174696F6E3A20533D52
:100AF000616363656C65726174696F6E2C20543D2F
:100B00007265747261637420616363656C657261A0
:100B100074696F6E0A255320204D323034205325DE
:100B20002E32662054252E32660A255341647661A2
:100B30006E636564207661726961626C65733A20E8
:100B4000533D4D696E206665656472617465202849
:100B50006D6D2F73292C20543D4D696E2074726188
:100B600076656C20666565647261746520286D6DBC
:100B70002F73292C20423D6D696E696D756D207350
:100B800065676D656E742074696D6520286D7329C5
:100B90002C20583D6D6178696D756D205859206A1B
:100BA00065726B20286D6D2F73292C20205A3D6DA6
:100BB0006178696D756D205A206A65726B20286DA9
:100BC0006D2F73292C2020453D6D6178696D756D01
:100BD0002045206A65726B20286D6D2F73290A25C8
:100BE0005320204D3230352053252E326620542597
:100BF0002E32662042252E32662058252E3266205F
:100C000059252E3266205A252E32662045252E3251
:100C1000660A2553486F6D65206F6666736574209C
:100C2000286D6D293A0A255320204D323036205840
:100C3000252E32662059252E3266205A252E326600
:100C40000A004625642025640A004D4D55203C3D90
:100C50002027462564202564270A00504944204166
:100C600075746F74756E652066696E697368656406
:100C7000212050757420746865206C617374204B5A
:100C8000702C204B6920616E64204B6420636F6E72
:100C90007374616E74732066726F6D2061626F761B
:100CA0006520696E746F20436F6E66696775726147
:100CB00074696F6E2E6800504944204175746F74DA
:100CC000756E65206661696C6564212074696D6567
:100CD0006F75740020403A00543A00423A0050497F
:100CE00044204175746F74756E65206661696C652A
:100CF00064212054656D706572617475726520742D
:100D00006F6F206869676800204B643A2000204BB1
:100D1000693A2000204B703A200020436C617373C5
:100D200069632050494420002054753A2000204B2C
:100D3000753A2000206D61783A2000206D696E3A86
:100D4000200020643A200020626961733A2000206C
:100D5000453A00205A3A0020593A0020453A0020EE
:100D60005A3A0020593A00583A00005A30005A3195
:100D700000593000593100583000583100456E6438
:100D80002073746F70732064696167002E0044657E
:100D90006C6574696F6E206661696C65642C2046B1
:100DA000696C653A200046696C652064656C657401
:100DB00065643A004E6F74205344207072696E74FB
:100DC000696E67005072696E7420736176656400A5
:100DD0005344207072696E7420706175736564008D
:100DE0000A002F000A002F2F20616374696F6E3A8A
:100DF00063616E63656C0043524153485F43414EEB
:100E000043454C0043524153485F5245434F56457A
:100E1000520043524153485F5245434F564552009A
:100E2000222832290054004475706C69636174652E
:100E300020542D636F64652069676E6F7265642E40
:100E40000A004475706C696361746520542D636F8A
:100E500064652069676E6F7265642E0A00496E765C
:100E6000616C6964205420636F64652E00556E6B5D
:100E70006E6F776E204D20636F64653A2025732076
:100E80000A006E6F2076616C696420636F6D6D611E
:100E90006E64002C20002C20002C20006E2F61009E
:100EA0002C20002C20002C20006E2F61002F0050E1
:100EB0003A005761697420666F722050494E444170
:100EC000207461726765742074656D7065726174F9
:100ED0007572653A004C414E472053454C20464FB1
:100EE0005243454400222831290030303030303020
:100EF00030302D303030302D303030302D303030FB
:100F0000302D303030303030303030303030002024
:100F1000555549443A0031002045585452554445EE
:100F2000525F434F554E543A0050727573612069B9
:100F300033204D4B3300204D414348494E455F54CB
:100F40005950453A00312E300020626173656420AB
:100F50006F6E204D61726C696E204649524D57414B
:100F600052455F55524C3A68747470733A2F2F672C
:100F700069746875622E636F6D2F7072757361335B
:100F8000642F50727573612D4669726D7761726559
:100F90002050524F544F434F4C5F56455253494F88
:100FA0004E3A004649524D574152455F4E414D45DC
:100FB0003A50727573612D4669726D776172652062
:100FC000004D31313320530020423A0020453A0091
:100FD000543A0020413A0020503A002042403A0062
:100FE00020403A00202F003A00205400202F0020FB
:100FF000423A00202F006F6B20543A002569206D83
:10100000696E2C2025692073656300496E76616CDA
:101010006964204D20636F64653A202573200A00BF
:10102000556E6B6E6F776E204720636F64653A2054
:101030002573200A004D65736820626564206C6525
:1010400076656C696E67206E6F7420616374697673
:10105000652E000A002020000A4D656173757265D7
:101060006420706F696E74733A000A5A2073656168
:10107000726368206865696768743A20002C004EC6
:10108000756D20582C593A2000206D6963726F6E7F
:1010900073004578636573736976652062656420C3
:1010A0006C6576656C696E6720636F7272656374D8
:1010B000696F6E3A2000426564206C6576656C69E4
:1010C0006E67206661696C65642E2053656E736F70
:1010D000722074726967676572656420746F6F202F
:1010E000686967682E0A00426564206C6576656CE5
:1010F000696E67206661696C65642E2053656E7346
:101100006F7220646973636F6E6E656374656420CB
:101110006F72206361626C652062726F6B656E2E08
:101120000A004732382057300050494E4441207061
:10113000726F62652063616C6962726174696F6E5F
:1011400020737461727400473238205730004D327A
:1011500034005345545F43484F505F005345545F3C
:10116000535445505F005345545F574156455F0007
:10117000544D435F0043524153485F0050726573C2
:1011800073206B6E6F6220746F207072656865618A
:1011900074206E6F7A7A6C6520616E6420636F6E66
:1011A00074696E75652E00506C6561736520707290
:1011B00065737320746865206B6E6F6220746F2096
:1011C000756E6C6F61642066696C616D656E74002C
:1011D00052656D6F7665206F6C642066696C616D19
:1011E000656E7420616E642070726573732074681C
:1011F00065206B6E6F6220746F207374617274204F
:101200006C6F6164696E67206E65772066696C61DA
:101210006D656E742E00616E64207072657373204C
:10122000746865206B6E6F6200496E73657274201E
:1012300066696C616D656E7400436F6C6F72206ED1
:101240006F7420636F72726563740046696C616DC0
:10125000656E74206E6F74206C6F6164656400430A
:1012600068616E67656420636F72726563746C7920
:101270003F004C6F6164696E6720636F6C6F720032
:101280004368616E676520737563636573732100DE
:10129000506C65617365206F70656E2069646C6564
:1012A0007220616E642072656D6F76652066696C70
:1012B000616D656E74206D616E75616C6C792E0068
:1012C0005761732066696C616D656E7420756E6C14
:1012D0006F6164207375636365737366756C3F003B
:1012E000506C6561736520757067726164652E006E
:1012F0004E6577206669726D7761726520766572DA
:1013000073696F6E20617661696C61626C653A0029
:1013100057616974696E6720666F722050494E4448
:10132000412070726F626520636F6F6C696E670039
:1013300043726173682064657465637465642E200C
:10134000526573756D65207072696E743F004372EB
:101350006173682064657465637465642E00457804
:101360007472756465720043686F6F736520657889
:101370007472756465723A0043686F6F73652066B6
:10138000696C616D656E743A004E6F206D6F7665A5
:101390002E005761697420666F7220757365722E16
:1013A0002E2E00536F6D652070726F626C656D201C
:1013B000656E636F756E74657265642C205A2D6C52
:1013C0006576656C696E6720656E666F72636564CD
:1013D000202E2E2E00537461626C6520616D62694F
:1013E000656E742074656D706572617475726520C8
:1013F00032312D323643206973206E656564656431
:101400002061207269676964207374616E64206969
:10141000732072657175697265642E00506C656128
:1014200073652072756E2058595A2063616C696229
:10143000726174696F6E2066697273742E007374C2
:101440006172740A006164635F696E69740A001BEB
:101450005B324A1B5B313B31484F726967696E6191
:101460006C2050727573612069331B5B323B3348CB
:1014700050727573612052657365617263680046CE
:101480006163746F72792052455345540041707204
:10149000202031203230313900436F6D70696C6526
:1014A000643A2000286E6F6E652C20646566617555
:1014B0006C7420636F6E666967290041707220202A
:1014C0003120323031392030313A31373A34390035
:1014D00020332E372E302D5243312D323137350AFD
:1014E000002055706C6F616420696E2070726F67A8
:1014F0007265737300205A3A0020593A0020583A16
:101500000043524153485F44455445435445445871
:10151000590043524153485F444554454354454460
:10152000590043524153485F444554454354454450
:1015300058004D3239005072757361206933204D67
:101540004B33204F4B2E00426C61636B6F757420E0
:101550006F636375727265642E205265636F766582
:1015600072207072696E743F0053656C66746573A7
:10157000742077696C6C2062652072756E20746FC0
:101580002063616C69627261746520616363757266
:101590006174652073656E736F726C65737320720E
:1015A00065686F6D696E672E0054686572652069A5
:1015B00073207374696C6C2061206E65656420749F
:1015C0006F206D616B65205A2063616C6962726186
:1015D00074696F6E2E20506C6561736520666F6C48
:1015E0006C6F7720746865206D616E75616C2C205E
:1015F00063686170746572204669727374207374D5
:101600006570732C2073656374696F6E2043616C21
:101610006962726174696F6E20666C6F772E00501C
:1016200072696E74657220686173206E6F742062D7
:1016300065656E2063616C696272617465642079AE
:1016400065742E20506C6561736520666F6C6C6FDD
:101650007720746865206D616E75616C2C206368FD
:10166000617074657220466972737420737465705A
:10167000732C2073656374696F6E2043616C6962BB
:10168000726174696F6E20666C6F772E004F6C64A8
:101690002073657474696E677320666F756E642E4F
:1016A0002044656661756C74205049442C20457354
:1016B00074657073206574632E2077696C6C20628A
:1016C00065207365742E005761726E696E673A20EB
:1016D000626F7468207072696E74657220747970BC
:1016E0006520616E64206D6F74686572626F6172EF
:1016F000642074797065206368616E6765642E008C
:101700005761726E696E673A207072696E746572A5
:101710002074797065206368616E6765642E005778
:1017200061726E696E673A206D6F74686572626F80
:101730006172642074797065206368616E676564A6
:101740002E0045787465726E616C20535049206696
:101750006C61736820573235583230434C206E6FBD
:101760007420726573706F6E64696E672E004372C9
:101770006173684465746563742044495341424C05
:101780004544004372617368446574656374204521
:101790004E41424C454421002020506C616E6E65E4
:1017A0007242756666657242797465733A200020EC
:1017B00046726565204D656D6F72793A2000207C18
:1017C00020417574686F723A2000204C6173742058
:1017D000557064617465643A200020536F667477B5
:1017E0006172652052657365740020576174636887
:1017F000646F67205265736574002042726F776E64
:10180000206F757420526573657400204578746587
:10181000726E616C20526573657400506F776572EB
:101820005570006572726F722077726974696E67A5
:1018300020746F2066696C6500656E6473746F70E8
:1018400073206869743A2000446F6E652073617676
:10185000696E672066696C652E006F6B0058595A77
:101860002063616C6962726174696F6E20616C6C77
:101870002072696768742E20536B65772077696CD6
:101880006C20626520636F727265637465642061A9
:1018900075746F6D61746963616C6C792E00585951
:1018A0005A2063616C6962726174696F6E20616C49
:1018B0006C2072696768742E20582F5920617865F2
:1018C000732061726520736C696768746C7920732A
:1018D0006B657765642E20476F6F64206A6F6221A5
:1018E0000058595A2063616C6962726174696F6E45
:1018F000206F6B2E20582F592061786573206172FC
:10190000652070657270656E646963756C61722EB6
:1019100020436F6E67726174756C6174696F6E736A
:10192000210058595A2063616C6962726174696F51
:101930006E206661696C65642E2052696768742048
:1019400066726F6E742063616C6962726174696F34
:101950006E20706F696E74206E6F742072656163A3
:101960006861626C652E0058595A2063616C696227
:10197000726174696F6E206661696C65642E2046C1
:10198000726F6E742063616C6962726174696F6EEC
:1019900020706F696E7473206E6F7420726561635E
:1019A0006861626C652E0058595A2063616C6962E7
:1019B000726174696F6E206661696C65642E205077
:1019C0006C6561736520636F6E73756C74207468E9
:1019D00065206D616E75616C2E0058595A206361E7
:1019E0006C6962726174696F6E20636F6D70726F83
:1019F0006D697365642E2052696768742066726F22
:101A00006E742063616C6962726174696F6E2070BC
:101A10006F696E74206E6F742072656163686162B5
:101A20006C652E0058595A2063616C69627261744A
:101A3000696F6E20636F6D70726F6D697365642E70
:101A40002046726F6E742063616C696272617469A2
:101A50006F6E20706F696E7473206E6F7420726584
:101A600061636861626C652E0058595A2063616C2D
:101A70006962726174696F6E206661696C65642E5B
:101A8000204265642063616C6962726174696F6E83
:101A900020706F696E7420776173206E6F7420669A
:101AA0006F756E642E00506C6561736520706C619B
:101AB000636520737465656C207368656574206F59
:101AC0006E20686561746265642E00446973746198
:101AD0006E6365206265747765656E207469702039
:101AE0006F6620746865206E6F7A7A6C6520616E0F
:101AF0006420746865206265642073757266616332
:101B00006520686173206E6F74206265656E207356
:101B10006574207965742E20506C6561736520664C
:101B20006F6C6C6F7720746865206D616E75616C89
:101B30002C2063686170746572204669727374202A
:101B400073746570732C2073656374696F6E2046BF
:101B500069727374206C617965722063616C69626B
:101B6000726174696F6E2E00506C61636520612034
:101B70007368656574206F6620706170657220758A
:101B80006E64657220746865206E6F7A7A6C652069
:101B9000647572696E67207468652063616C696240
:101BA000726174696F6E206F66206669727374204B
:101BB0003420706F696E74732E20496620746865D6
:101BC000206E6F7A7A6C6520636174636865732038
:101BD0007468652070617065722C20706F77657213
:101BE000206F666620746865207072696E74657215
:101BF00020696D6D6564696174656C792E00506C47
:101C0000656173652072656D6F76652073746565B7
:101C10006C2073686565742066726F6D20686561FD
:101C2000746265642E00497320737465656C20735B
:101C300068656574206F6E20686561746265643FD5
:101C400000206F66203400536561726368696E67B7
:101C5000206265642063616C6962726174696F6E91
:101C600020706F696E7400206F662039004D6561C9
:101C7000737572696E67207265666572656E6365FD
:101C800020686569676874206F662063616C6962AB
:101C9000726174696F6E20706F696E7400506C654C
:101CA00061736520636C65616E20746865206E6F7A
:101CB0007A7A6C6520666F722063616C696272610A
:101CC00074696F6E2E20436C69636B207768656E54
:101CD00020646F6E652E004175746F20686F6D65AE
:101CE0000078797A63616C5F6D6561737375726595
:101CF0005F656E7465720A0078797A63616C5F73F0
:101D0000706972616C382063783D25642063793D89
:101D10002564207A303D256420647A3D2564207254
:101D200061646975733D25642061643D25640A0022
:101D300078797A63616C5F7365617263685A206E4B
:101D40006F207369676E616C0A20783D256C642092
:101D5000793D256C64207A3D256C640A00204F4E45
:101D60002D5349474E414C20617420783D25642015
:101D7000793D2564207A3D25642061643D25640A0F
:101D80000078797A63616C5F7365617263685A2069
:101D9000783D256C6420793D256C64207A3D256C66
:101DA000640A000A00253032780078797A63616C21
:101DB0005F7363616E5F706978656C735F333278EF
:101DC00033322063783D25642063793D2564206D9E
:101DD000696E5F7A3D2564206D61785F7A3D256488
:101DE0000A00202532642025640A000A00253032CA
:101DF0007800206D696E3D2564206D61783D256415
:101E0000206469663D25640A006D61785F633D2545
:101E10003264206D61785F6C3D25640A006D6178E5
:101E20005F633D2564206D61785F723D2564206DA0
:101E300061785F6D617463683D25640A0020783DB8
:101E4000256420793D2564207A3D25640A002070B0
:101E500061747465726E20666F756E6420617420A3
:101E600025642025640A000000F000F801FC03FE50
:101E700007FE07FE07FE07FC03F801F000000073F1
:101E8000697A656F6628746F74616C293D25640AF0
:101E90000073697A656F6628626C6F636B5F627549
:101EA00066666572293D25640A0078797A63616CFB
:101EB0005F6D656173737572655F6C656176650AE8
:101EC00000706F696E743D256420783D256420792B
:101ED0003D2564207A3D25640A0058025802584D79
:101EE000584DB004F055F055B00478797A63616CC0
:101EF0005F66696E645F6265645F696E6475637472
:101F0000696F6E5F73656E736F725F706F696E7409
:101F10005F787920783D256C6420793D256C6420BC
:101F20007A3D256C640A00203C20005741524E49FE
:101F30004E473A2046726F6E7420706F696E74203F
:101F40006E6F7420726561636861626C652E2059E2
:101F500020636F6F7264696E6174653A00000000FF
:101F600040410000C04000005C430000C040000051
:101F70005C43000046430000404100004643497472
:101F800065726174696F6E3A200043616C696272B8
:101F90006174696F6E206661696C656421204368B5
:101FA00065636B20746865206178657320616E6479
:101FB0002072756E20616761696E2E002220666155
:101FC000696C65643A204275666665722066756C58
:101FD0006C21002200256920686F757273202569C5
:101FE000206D696E757465730054494D454F5554A5
:101FF0003A004D3131300046756C6C205258204209
:102000007566666572006673656E736F725F737472
:102010006F705F616E645F736176655F7072696E29
:10202000740A006673656E736F725F726573746FA6
:1020300072655F7072696E745F616E645F636F6E0C
:1020400074696E75650A0044495341424C45440A1F
:1020500000454E41424C4544004653656E736F72D5
:102060002025530A00504154393132355F696E6979
:10207000743A256868750A00504154393132355F29
:10208000696E69743A256868750A0050415439319F
:102090003235206E6F7420726573706F6E64696E76
:1020A000672028256429210A00656E717565696EAF
:1020B00067202200446F6E65207072696E74696ECD
:1020C000672066696C65005072696E746572207372
:1020D000746F707065642064756520746F2065721C
:1020E000726F72732E20466978207468652065725D
:1020F000726F7220616E6420757365204D393939B5
:1021000020746F20726573746172742E2028546578
:102110006D70657261747572652069732072657384
:1021200065742E205365742069742061667465722D
:102130002072657374617274696E6729004E6F2036
:102140004C696E65204E756D6265722077697468A2
:1021500020636865636B73756D2C204C617374200C
:102160004C696E653A20004E6F20436865636B735F
:10217000756D2077697468206C696E65206E756D69
:102180006265722C204C617374204C696E653A2034
:1021900000636865636B73756D206D69736D617441
:1021A00063682C204C617374204C696E653A200082
:1021B0004C696E65204E756D626572206973206E84
:1021C0006F74204C617374204C696E65204E756D80
:1021D0006265722B312C204C617374204C696E65E2
:1021E0003A20006673656E736F725F6175746F6C11
:1021F0006F61645F636865636B5F737461727420A1
:102200002D206175746F6C6F616420454E41424CA6
:1022100045440A006673656E736F725F6175746F13
:102220006C6F61645F636865636B5F73746F70206C
:102230002D206175746F6C6F616420444953414275
:102240004C45440A0053544F505045442E20006FD3
:102250006B0A0073746172740A004D4D553220662A
:1022600069726D776172652076657273696F6E2031
:10227000696E76616C69642E20526571756972654C
:10228000642076657273696F6E3A206275696C645A
:10229000206E756D626572202564206F72206869FA
:1022A000676865722E004D4D55203D3E20276F6BAF
:1022B000270A004D4D55203D3E20276F6B270A0011
:1022C0002564004D4D55203D3E20276F6B272C2067
:1022D000726573756D65207072696E740A004D4D7C
:1022E0005520726574727920617474656D70742004
:1022F0006E722E2025640A004D4D55203D3E20274C
:102300006F6B270A00410A004D4D55203C3D2027A8
:1023100041270A004D363030004D363030204155CF
:10232000544F005052555341206673656E736F725F
:102330005F7265636F766572002568687500410A93
:10234000004D4D55203C3D202741270A0050300AC2
:10235000004D25640A004D4D55203C3D20274D255C
:1023600064270A0057300A004D4D55203C3D202778
:102370005730270A0053330A004D4D55203C3D206D
:10238000275333270A0052300A004D4D55203C3D5B
:1023900020275230270A004B25640A004D4D552056
:1023A0003C3D20274B2564270A004525640A004D43
:1023B0004D55203C3D2027452564270A0055300A0D
:1023C000004D4D55203C3D20275530270A00433015
:1023D0000A004D4D55203C3D20274330270A004C34
:1023E00025640A004D4D55203C3D20274C2564278F
:1023F0000A005425640A004D4D55203C3D202754C9
:102400002564270A004D4D55202D20454E41424C54
:10241000454400256868750050300A004D310A00B7
:102420004D4D55203C3D20274D31270050300A00AE
:102430004D4D552076657273696F6E2076616C69BB
:1024400064004D4D55203D3E202725646F6B270AC3
:102450000025750053320A004D4D55203C3D202784
:10246000533227004D4D55203D3E202725646F6B8C
:10247000270A002575004D4D55206E6F742072653A
:1024800073706F6E64696E67202D2044495341421A
:102490004C45440053310A004D4D55203C3D20270A
:1024A000533127004D4D55203D3E202773746172F6
:1024B0007427006572726F723A20756E6B6E6F775B
:1024C0006E206D6F76650A006E6F206D6F76650AFF
:1024D00000542D636F64650A00756E6C6F61640A49
:1024E000006C6F61640A006D6D755F6765745F7283
:1024F0006573706F6E7365202D20626567696E204D
:102500006D6F76653A20006D6D755F6765745F72FB
:102510006573706F6E736528292072657475726EAD
:10252000696E673A2025640A00556E6C6F616469B4
:102530006E672066696E697368656420320A0055AB
:102540006E6C6F616420320A00556E6C6F61646955
:102550006E672066696E697368656420310A00558C
:102560006E6C6F616420310A004D4D5520737461AB
:1025700072747320726573706F6E64696E670A009F
:102580004D4D55206E6F7420726573706F6E646967
:102590006E670A000000803F555585410000803F6E
:1025A0000000C84100000040555505420000C03FF2
:1025B000000048420000204055558542000070C18F
:1025C000ABAAA642000060C10000A0410000C0C04C
:1025D0000000204100002041ABAA3A41000020C188
:1025E0005555D540000048C2555505424D3730314C
:1025F000204530004D373031204531004D373031E6
:10260000204532004D373031204533004D373031D1
:10261000204534004D373031204534004D373031BE
:10262000204533004D373031204532004D373031B1
:10263000204531004D3730312045300046696C610E
:102640006D656E74206E72206F7574206F662072D7
:10265000616E676521004164646974696F6E616CC5
:10266000206C6F616420617474656D7074206E728B
:102670002E2025640A00506C6561736520757064B6
:10268000617465206669726D7761726520696E207C
:10269000796F7572204D4D55322E205761697469DE
:1026A0006E6720666F722072657365742E004D4DE3
:1026B00055204F4B2E20526573756D696E672E2E17
:1026C0002E004D4D55204F4B2E20526573756D6970
:1026D0006E6720706F736974696F6E2E2E2E004DB9
:1026E0004D55204F4B2E20526573756D696E6720D6
:1026F00074656D70657261747572652E2E2E00465C
:1027000069782074686520697373756520616E64EB
:10271000207468656E2070726573732062757474BE
:102720006F6E206F6E204D4D5520756E69742E00B2
:10273000507265737320746865206B6E6F622074CD
:102740006F20726573756D65206E6F7A7A6C652087
:1027500074656D70657261747572652E004D4D55AE
:10276000206E65656473207573657220617474658D
:102770006E74696F6E2E00506C65617365207265B2
:102780006D6F76652066696C616D656E7420616E33
:1027900064207468656E2070726573732074686558
:1027A000206B6E6F622E00456A656374696E6720E8
:1027B00066696C616D656E74004D4D55206C6F617E
:1027C00064206661696C65642020202020002563F8
:1027D0002533642F25642563005A206C69766520B3
:1027E00061646A757374206F7574206F66207261FE
:1027F0006E67652E2053657474696E6720746F2050
:10280000302E20436C69636B20746F20636F6E748D
:10281000696E75652E005A206C6976652061646A60
:10282000757374206F7574206F662072616E6765B2
:102830002E2053657474696E6720746F20300020F9
:10284000423A0020453A00543A00494E543400724E
:1028500065636F7665725F6D616368696E655F73EE
:10286000746174655F61667465725F706F776572BD
:102870005F70616E69632C20696E697469616C2098
:10288000007265636F7665725F6D616368696E651E
:102890005F73746174655F61667465725F706F7792
:1028A00065725F70616E69632C20696E697469611D
:1028B0006C20004739322045005052555341207555
:1028C000766C6F004734205330004D32362053254C
:1028D0006C75004D3130362053004D383200473191
:1028E000204625640047312045322A6465666175BB
:1028F0006C745F72657472616374696F6E204634C4
:102900003830004731205A00204632303030002025
:10291000590047312058004D383300506F736974A7
:10292000696F6E20726561642066726F6D206565E7
:1029300070726F6D3A004D3233202573002E67633D
:102940006F0046656564726174653A0047312045E1
:102950002D64656661756C745F7265747261637411
:10296000696F6E20463438300047312045352046A7
:10297000313230004D3833004D3139302053256429
:10298000004D31303920532564004732382058201B
:1029900059004731205A3235204638303000204621
:1029A000004731205A0020460047312045004D386D
:1029B0003300627573793A207061757365642066BF
:1029C0006F7220696E70757400627573793A207049
:1029D000617573656420666F72207573657200623D
:1029E0007573793A2070726F63657373696E6700EF
:1029F0006F6B0A0055564C4F202D20656E642025C4
:102A0000640A007374707325640A00776F726C64D3
:102A100020636F6F7264696E617465733A20282554
:102A20002E33662C20252E33662C20252E33662946
:102A30000A00706879736963616C20636F6F7264F8
:102A4000696E617465733A2028252E33662C202523
:102A50002E33662C20252E3366290A0043757272A8
:102A6000656E7420706F73205A5F415849533A2540
:102A70002E33660A43757272656E7420706F732010
:102A8000455F415849533A252E33660A0041667422
:102A900065722077616974696E6720666F72207451
:102AA000656D703A0A43757272656E7420706F734B
:102AB00020585F415849533A252E33660A437572B0
:102AC00072656E7420706F7320595F415849533A94
:102AD000252E33660A005265636F766572696E67EC
:102AE000207072696E742020202000746D63323172
:102AF00033305F686F6D655F656E746572286178ED
:102B000065735F6D61736B3D307825303278290ACB
:102B100000746D63323133305F686F6D655F657867
:102B2000697420746D63323133305F73675F686F2F
:102B30006D696E675F617865735F6D61736B3D3062
:102B400078253032780A00726573756C742076616E
:102B50006C75653A2025640A0020693D25326420A1
:102B6000636E743D2532642076616C3D2532640AC3
:102B700000636C7573746572733A0A0020693D25B1
:102B8000326420737465703D2532640A00736F727D
:102B90007465642073616D706C65733A0A003A2045
:102BA0000020202020202020202020202020202045
:102BB0002020202000203A2000202020202020203B
:102BC0002020202020202020202020202000202025
:102BD00020202020202020202020200025730054A9
:102BE0004D4320445249564552204F564552544574
:102BF0004D50002533642E2530317525632564251D
:102C000063005A2533642E25303275005A2D2D2D40
:102C10002E2D2D0025632533642525002D2D2D0017
:102C20002533686864002533532533732525002038
:102C300053440020202000555342002025753E2596
:102C40007500203F3E257500204625750020463F33
:102C50000020463020200025632D2D3A2D2D2020E8
:102C600000256325337568202563256300256325CA
:102C70003032753A25303275256325630050494E50
:102C800044412048656174696E670054656D702E1B
:102C90002063616C2E202020202020202020200076
:102CA00043616C6962726174696F6E20646F6E65F6
:102CB0000043616C6962726174696E67205A0042F8
:102CC000656420646F6E65004265642048656174C8
:102CD000696E670048656174696E6720646F6E6530
:102CE0002E0048656174696E67004D3435004D34BF
:102CF00035205A004737360057697A61726420736D
:102D0000746174653A2025640044697361626C657E
:102D1000206661726D206D6F6465004661726D2082
:102D20006E756D626572004D3834004D3434004765
:102D300032382057004739390044697361626C6545
:102D4000206661726D206D6F64653F0043686F6F30
:102D5000736520636F6C6F723A0043616C696272D5
:102D600061746500506C65617365206C6F616420EF
:102D7000504C412066696C616D656E7420666972A5
:102D800073742E00497320504C412066696C616D4C
:102D9000656E74206C6F616465643F0043616E63AF
:102DA000656C0046696C616D656E740053656C6599
:102DB000637420504C412066696C616D656E743A95
:102DC0000052756E6E696E672057697A6172642071
:102DD00077696C6C2064656C6574652063757272CC
:102DE000656E742063616C6962726174696F6E20D4
:102DF000726573756C747320616E64207374617294
:102E0000742066726F6D2074686520626567696EF4
:102E10006E696E672E20436F6E74696E75653F0034
:102E200050726568656174696E67206E6F7A7A6C3E
:102E3000652E20506C6561736520776169742E0082
:102E4000456A65637400556E6C6F61640055736507
:102E500020756E6C6F616420746F2072656D6F7683
:102E6000652066696C616D656E742031206966202D
:102E700069742070726F747275646573206F7574F5
:102E800073696465206F662074686520726561727D
:102E9000204D4D5520747562652E20557365206553
:102EA0006A656374206966206974206973206869A3
:102EB0006464656E20696E20747562652E004C6FC7
:102EC0006164696E672066696C616D656E7400503F
:102ED0006C6561736520696E7365727420504C4136
:102EE0002066696C616D656E7420746F207468650E
:102EF0002065787472756465722C207468656E2024
:102F00007072657373206B6E6F6220746F206C6FCC
:102F100061642069742E00506C6561736520696E70
:102F20007365727420504C412066696C616D656EEA
:102F30007420746F207468652066697273742074DD
:102F4000756265206F66204D4D552C207468656E46
:102F500020707265737320746865206B6E6F6220D9
:102F6000746F206C6F61642069742E00596F752036
:102F700063616E20616C7761797320726573756D22
:102F800065207468652057697A6172642066726F83
:102F90006D2043616C6962726174696F6E202D3EB1
:102FA0002057697A6172642E00506C6561736520E8
:102FB000636865636B206F75722068616E64626F11
:102FC0006F6B20616E64206669782074686520707C
:102FD000726F626C656D2E205468656E2072657329
:102FE000756D65207468652057697A617264206226
:102FF00079207265626F6F74696E672074686520EE
:103000007072696E7465722E00416C6C2069732059
:10301000646F6E652E204861707079207072696EE1
:1030200074696E672100506C6561736520636C651F
:10303000616E206865617462656420616E642074ED
:1030400068656E20707265737320746865206B6E9E
:103050006F622E00446F20796F752077616E742047
:10306000746F20726570656174206C617374207375
:1030700074657020746F20726561646A7573742062
:1030800064697374616E6365206265747765656EEB
:10309000206E6F7A7A6C6520616E64206865617459
:1030A0006265643F00492077696C6C2073746172BB
:1030B0007420746F207072696E74206C696E652064
:1030C000616E6420796F752077696C6C206772611E
:1030D0006475616C6C79206C6F77657220746865BB
:1030E000206E6F7A7A6C6520627920726F746174D9
:1030F000696E6720746865206B6E6F622C20756E38
:1031000074696C20796F75207265616368206F70D7
:1031100074696D616C206865696768742E20436806
:1031200065636B207468652070696374757265737C
:1031300020696E206F75722068616E64626F6F6BBC
:1031400020696E20636861707465722043616C69E8
:1031500062726174696F6E2E004E6F77204920771E
:10316000696C6C2063616C6962726174652064696A
:103170007374616E6365206265747765656E207433
:103180006970206F6620746865206E6F7A7A6C654E
:1031900020616E6420686561746265642073757275
:1031A000666163652E00497320697420504C41208C
:1031B00066696C616D656E743F0053656C65637420
:1031C000206E6F7A7A6C6520707265686561742014
:1031D00074656D7065726174757265207768696376
:1031E00068206D61746368657320796F7572206DF6
:1031F0006174657269616C2E004E6F77204920778B
:10320000696C6C2070726568656174206E6F7A7A83
:103210006C6520666F7220504C412E004973206609
:10322000696C616D656E74206C6F616465643F00EC
:1032300049732066696C616D656E742031206C6F16
:10324000616465643F004E6F7720492077696C6C3C
:103250002070726568656174206E6F7A7A6C652083
:10326000666F7220504C412E00492077696C6C20AB
:1032700072756E207A2063616C6962726174696F25
:103280006E206E6F772E004E6F772072656D6F76B1
:1032900065207468652074657374207072696E743B
:1032A0002066726F6D20737465656C207368656548
:1032B000742E00506C656173652072656D6F766564
:1032C000207368697070696E672068656C706572DC
:1032D000732066697273742E00492077696C6C20C4
:1032E00072756E2078797A2063616C69627261749C
:1032F000696F6E206E6F772E2049742077696C6C31
:103300002074616B6520617070726F782E2031328D
:10331000206D696E732E0046697273742C204920EB
:1033200077696C6C2072756E207468652073656CAB
:10333000667465737420746F20636865636B206DB9
:103340006F737420636F6D6D6F6E20617373656D45
:10335000626C792070726F626C656D732E004869C3
:103360002C204920616D20796F7572204F7269673A
:10337000696E616C205072757361206933207072C0
:10338000696E7465722E20576F756C6420796F7545
:10339000206C696B65206D6520746F2067756964AA
:1033A0006520796F75207468726F7567682074681E
:1033B000652073657475702070726F636573733FF9
:1033C00000452D636F7272656374005A2D636F72CE
:1033D0007265637400592D636F727265637400586F
:1033E0002D636F72726563740053706F6F6C4A6FF8
:1033F000696E2020205B4E2F415D0053706F6F6C13
:103400004A6F696E2020205B6F66665D0053706FA7
:103410006F6C4A6F696E202020205B6F6E5D0053D9
:103420006F756E642020202020205B6C6F75645DBA
:1034300000536F756E642020202020205B6D757412
:10344000655D00536F756E64202020205B73696C8E
:10345000656E745D00536F756E64202020202020FF
:103460005B6F6E63655D00536F756E642020202076
:1034700020205B6C6F75645D00536F727420202098
:10348000202020205B6E6F6E655D00536F7274208C
:1034900020205B616C7068616265745D00536F72BF
:1034A00074202020202020205B74696D655D00530E
:1034B00044206361726420205B6E6F726D616C5D8D
:1034C0000053442063617264205B666C73684169D9
:1034D000725D0052506920706F727420202020208D
:1034E0005B6F6E5D0052506920706F7274202020F7
:1034F000205B6F66665D0054656D702E2063616CA5
:103500002E2020205B6F6E5D0054656D702E206351
:10351000616C2E20205B6F66665D004C696E2E200C
:10352000636F7272656374696F6E004D65736820B6
:10353000626564206C6576656C696E67004D4D55FB
:10354000204D6F64655B537465616C74685D004DFC
:103550004D55204D6F6465205B4E6F726D616C5DE3
:103560000046616E7320636865636B20205B6F6645
:10357000665D0046616E7320636865636B20202082
:103580005B6F6E5D00462E206175746F6C6F6164B9
:10359000205B6F66665D00462E206175746F6C6FF0
:1035A000616420205B6F6E5D00462E206175746F34
:1035B0006C6F6164205B4E2F415D0046696C2E206C
:1035C00073656E736F72205B4E2F415D00446973AB
:1035D00061626C65207374657070657273004D6F05
:1035E000766520617869730054656D7065726174E9
:1035F0007572650054656D702E2063616C6962722E
:103600006174696F6E0052657365742058595A2051
:1036100063616C6962722E005049442063616C6979
:1036200062726174696F6E00426564206C657665D4
:103630006C20636F7272656374004D65736820421D
:103640006564204C6576656C696E670043616C69E2
:103650006272617465205A0043616C6962726174C0
:10366000652058595A0053656C6674657374202040
:1036700020202020202020004669727374206C6175
:103680007965722063616C2E0057697A61726400FB
:103690004C6F61642066696C616D656E74203500E5
:1036A0004C6F61642066696C616D656E74203400D6
:1036B0004C6F61642066696C616D656E74203300C7
:1036C0004C6F61642066696C616D656E74203200B8
:1036D0004C6F61642066696C616D656E74203100A9
:1036E0004C6F616420616C6C004C6F616420666992
:1036F0006C616D656E742035004C6F616420666985
:103700006C616D656E742034004C6F616420666975
:103710006C616D656E742033004C6F616420666966
:103720006C616D656E742032004C6F616420666957
:103730006C616D656E74203100456A656374206646
:10374000696C616D656E74203500456A656374202F
:1037500066696C616D656E74203400456A656374DA
:103760002066696C616D656E74203300456A65631F
:10377000742066696C616D656E74203200456A65FF
:1037800063742066696C616D656E74203100506CE5
:10379000656173652070756C6C206F757420666947
:1037A0006C616D656E7420696D6D656469617465C9
:1037B0006C7900556E6C6F6164696E672066696C28
:1037C000616D656E740057697A61726420656E641C
:1037D0002073746174653A2025640A0020003E005D
:1037E0003E0020003E003E0054656D7065726174BD
:1037F0007572652063616C6962726174696F6E20B5
:103800006661696C65642E20436F6E74696E7565C0
:103810002077697468207072657373696E672074AD
:103820006865206B6E6F622E0054656D7065726105
:10383000747572652063616C6962726174696F6E20
:1038400020646F6E652E20436F6E74696E756520FF
:1038500077697468207072657373696E6720746825
:1038600065206B6E6F622E004738300054656D70B6
:10387000657261747572652063616C6962726174EE
:10388000696F6E206661696C65640054656D706572
:103890007261747572652063616C696272617469CA
:1038A0006F6E2069732066696E6973686564206154
:1038B0006E64206163746976652E2054656D702E88
:1038C0002063616C6962726174696F6E2063616EFE
:1038D0002062652064697361626C656420696E2092
:1038E0006D656E752053657474696E67732D3E54F3
:1038F000656D702E2063616C2E004E2F41002020DC
:1039000030002020310049523A0046494E44413AA5
:103910000050494E44413A0053656E736F722073F4
:1039200074617465004578747275646572004D6FDA
:103930007665205A004D6F76652059004D6F76658B
:103940002058001B5B324A437261736820646574BF
:10395000656374696F6E2063616E1B5B313B304839
:103960006265207475726E6564206F6E206F6E6C78
:103970007920696E1B5B323B30484E6F726D616C13
:10398000206D6F6465001B5B324A5741524E494EB1
:10399000473A1B5B313B3048437261736820646572
:1039A00074656374696F6E1B5B323B304864697386
:1039B00061626C656420696E1B5B333B30485374F5
:1039C00065616C7468206D6F6465004175746F6C1F
:1039D0006F6164696E672066696C616D656E7420E5
:1039E000617661696C61626C65206F6E6C792077BD
:1039F00068656E2066696C616D656E742073656EB6
:103A0000736F72206973207475726E6564206F6EB7
:103A10002E2E2E004552524F523A2046696C616D4F
:103A2000656E742073656E736F72206973206E6F9C
:103A30007420726573706F6E64696E672C20706C91
:103A40006561736520636865636B20636F6E6E6587
:103A50006374696F6E2E004D6F6465206368616EDC
:103A6000676520696E2070726F6772657373202EB0
:103A70002E2E00526573756D696E67207072696EC7
:103A80007400537570706F7274004661696C2073B6
:103A900074617473204D4D55004661696C207374D8
:103AA0006174730053746174697374696373202063
:103AB0000043616C6962726174696F6E0041757474
:103AC0006F4C6F61642066696C616D656E74004552
:103AD0006A6563742066696C616D656E7400556E0D
:103AE0006C6F61642066696C616D656E74004C6F0B
:103AF000616420746F206E6F7A7A6C65004C6F6120
:103B0000642066696C616D656E74004E6F2053446D
:103B10002063617264005072696E742066726F6D0A
:103B200020534400526573756D65207072696E7420
:103B3000005061757365207072696E740050726513
:103B4000686561740054756E65004C697665206126
:103B5000646A757374205A00496E666F20736372CD
:103B600065656E0046696E697368696E67206D6F82
:103B700076656D656E747300536F756E64202020DA
:103B80002020205B6C6F75645D00536F756E642040
:103B900020202020205B6D7574655D00536F756E6D
:103BA00064202020205B73696C656E745D00536F28
:103BB000756E642020202020205B6F6E63655D00A1
:103BC000536F756E642020202020205B6C6F75641D
:103BD0005D004D4D55204D6F64655B537465616CA0
:103BE00074685D004D4D55204D6F6465205B4E6FD0
:103BF000726D616C5D004372617368206465742E40
:103C000020205B4E2F415D00437261736820646524
:103C1000742E2020205B6F6E5D00437261736820FC
:103C20006465742E20205B6F66665D004D6F646571
:103C3000202020205B537465616C74685D004D6FBB
:103C4000646520202020205B4E6F726D616C5D00EA
:103C500046696C2E2073656E736F7220205B6F6EE9
:103C60005D0046696C2E2073656E736F72205B6F0A
:103C700066665D004368616E67652066696C616DAC
:103C8000656E7400466C6F77005370656564004D17
:103C900061676E65747320636F6D702E5B4E2F418C
:103CA0005D004D61676E65747320636F6D702E5B90
:103CB0004F66665D004D61676E65747320636F6D5E
:103CC000702E205B4F6E5D005A2D70726F62652002
:103CD0006E722E202020205B335D005A2D70726F93
:103CE0006265206E722E202020205B355D005A2DEB
:103CF00070726F6265206E722E202020205B315D15
:103D0000004D6573682020202020202020205B3774
:103D100078375D004D65736820202020202020200A
:103D2000205B3378335D0046616E20737065656497
:103D300000426564004E6F7A7A6C65005365747456
:103D4000696E6773005072696E742061626F72747D
:103D5000656400596573004E6F0053746F70207076
:103D600072696E740046696C6520696E636F6D7070
:103D70006C6574652E20436F6E74696E7565206185
:103D80006E797761793F004261636B004D61696EC6
:103D9000004661726D206E756D626572004D363041
:103DA00030004D3234004D323320257300052E2E65
:103DB0000024F4D43050C38E20C2A24017828B70EE
:103DC00011127A910D816CD90AA861E108C7586671
:103DD00007615143061E4B5D05C145A7041A4111F9
:103DE00004093D9803713931034036DB0265339194
:103DF00002D4305402802E1D02632CEE01752AC5B8
:103E000001B028A001102781018F2564012B244BCC
:103E100001E0223401AC211F018D200D01801FFC27
:103E200000841EED00971DDF00B81CD200E61BC603
:103E300000201BBC00641AB200B219A8000A19A025
:103E4000006A189900D117910040178B00B51684AD
:103E50000031167E00B31579003A157300C7146F50
:103E60000058146A00EE1366008813630025135E81
:103E700000C7125B006C12570015125400C111519B
:103E80000070114F0021114B00D61049008D1047D2
:103E9000004610440002104200C00F4000800F3E58
:103EA00000420F3C00060F3B00CB0E3800930E374C
:103EB000005C0E3500270E3400F30D3200C10D31C9
:103EC00000900D3000600D2E00320D2D00050D2CE0
:103ED00000D90C2B00AE0C2900850C29005C0C27A6
:103EE00000350C27000E0C2600E80B2400C40B2420
:103EF00000A00B23007D0B23005A0B2100390B215E
:103F000000180B2000F80A1F00D90A1E00BB0A1E69
:103F1000009D0A1D00800A1D00630A1C00470A1B41
:103F2000002C0A1B00110A1A00F7091A00DD0919F2
:103F300000C4091900AB091900920917007B091880
:103F400000630917004C09160036091600200916EF
:103F5000000A091500F5081500E0081400CC081443
:103F600000B8081400A4081400900813007D08127B
:103F7000006B08130058081200460812003408119C
:103F800000230811001208110001081100F00710A9
:103F900000E0071000D0071000C0071000B0070FA6
:103FA00000A107100091070E0083070F0074070F90
:103FB0000065070E0057070E0049070E003B070D6E
:103FC000002E070E0020070D0013070D0006070D39
:103FD00000F9060C00ED060D00E0060C00D4060CFE
:103FE00000C8060C00BC060C00B0060C00A4060BB2
:103FF0000099060C008D060B0082060B0077060B5D
:10400000006C060B0061060A0057060B004C060AFE
:104010000042060A0038060A002E060A0024060A94
:10402000001A060A001006090007060A00FD050925
:1040300000F4050900EB050900E2050900D90509AE
:1040400000D0050900C7050900BE050900B505082F
:1040500000AD050800A50509009C050800940508A9
:10406000008C050800840508007C0508007405081C
:10407000006C050700650508005D0507005605088A
:10408000004E0507004705070040050800380507F2
:1040900000310507002A050700230507001C050657
:1040A00000160507000F05070008050600020507B2
:1040B00000FB040600F5040700EE040600E8040611
:1040C00000E2040700DB040600D5040600CF040666
:1040D00000C9040600C3040600BD040600B70406B8
:1040E00000B1040500AC040600A6040600A0040507
:1040F000009B04060095040500900406008A040550
:104100000085040500800406007A04050075040596
:1041100000700405006B04050066040500610405D9
:10412000005C04050057040500520405004D040519
:104130000048040500430405003E0404003A040559
:104140000035040500300404002C04050027040495
:1041500000230405001E0404001A040400160405CC
:1041600000110404000D0404000904050004040403
:104170000000040400FC030400F8030400F403043A
:1041800000F0030400EC030400E8030400E403046B
:1041900000E0030400DC030400D8030400D403049B
:1041A00000D0030400CC030400C8030300C50303CC
:1041B0000024F404D9201BC40C5C0E9804C4095FCD
:1041C0000265077101F405F900FB04B30048048798
:1041D00000C10369005803550003034500BE023ABD
:1041E000008402310053022A002902250004022023
:1041F00000E4011C00C8011900AF01170098011468
:104200000084011300710110006101100051010EC2
:104210000043010D0036010B002B010B0020010BA8
:1042200000150109000C01090003010800FB00084A
:1042300000F3000800EB000700E4000600DE0006C3
:1042400000D8000600D2000600CC000500C700051B
:1042500000C2000500BD000400B9000400B5000460
:1042600000B1000400AD000400A9000400A5000393
:1042700000A20003009F0004009B000300980003BD
:10428000009500020093000300900003008D0002DF
:10429000008B0003008800020086000200840003F7
:1042A00000810002007F0002007D0002007B00020E
:1042B000007900020077000100760002007400021D
:1042C0000072000100710002006F0002006D000129
:1042D000006C0002006A0001006900020067000132
:1042E0000066000100650001006400020062000138
:1042F0000061000100600001005F0002005D00013C
:10430000005C0001005B0001005A0001005900013F
:10431000005800010057000100560001005500013F
:10432000005400010053000000530001005200013E
:104330000051000100500001004F0001004E00003C
:10434000004E0001004D0001004C0001004B000038
:10435000004B0001004A0001004900010048000034
:10436000004800010047000100460000004600012F
:10437000004500000045000100440001004300002A
:104380000043000100420000004200010041000023
:104390000041000100400001003F0000003F00011B
:1043A000003E0000003E0001003D0000003D000115
:1043B000003C0000003C0000003C0001003B00000D
:1043C000003B0001003A0000003A00010039000003
:1043D00000390001003800000038000000380001FA
:1043E00000370000003700010036000000360000F2
:1043F00000360001003500000035000000350001E6
:1044000000340000003400000034000100330000DC
:1044100000330000003300010032000000320000D1
:1044200000320001003100000031000000310001C5
:10443000003000000030000000300001002F0000BC
:10444000002F0000002F0000002F0001002E0000B0
:10445000002E0000002E0001002D0000002D0000A5
:10446000002D0000002D0001002C0000002C000099
:10447000002C0000002C0001002B0000002B00008D
:10448000002B0000002B0001002A0000002A000081
:10449000002A0000002A0001002900000029000075
:1044A0000029000000290000002900010028000068
:1044B000002800000028000000280000002800015B
:1044C0000027000000270000002700000027000050
:1044D0000027000100260000002600000026000042
:1044E0000026000000260001002500000025000035
:1044F0000025000000250000002500000025000127
:10450000002400000024000000240000002400001B
:10451000002400010023000000230000002300000D
:1045200000230000002300000023000000230001FE
:1045300000220000002200000022000000220000F3
:1045400000220000002200010021000000210000E4
:1045500000210000002100000021000000210000D7
:1045600000210001002000000020000000200000C9
:1045700000200000002000000020000000200000BB
:1045800000200001001F0000001F0000001F0000AD
:10459000001F0000001F0000001F0000001F00019E
:1045A000001E0000001E0000001E0000001E000093
:1045B00000000E1315110E00000004120912040071
:1045C00000001C1F11111F00000006191803130C16
:1045D00000040E1F041C000000040A0A0A0A11113C
:1045E0000E001F1511151F0000000103161C080006
:1045F000000000110A04110A040C12120C00000041
:10460000002563252D3138532563002563252E3180
:1046100035533A2573253364002563252E313253F3
:104620003A25732500457872656D65207370616E5B
:10463000206F6620746865205A2076616C756573FA
:104640002100205B6F66665D00426564206C6576C4
:10465000656C696E67206661696C65642E205365C0
:104660006E736F72206469646E7420747269676718
:1046700065722E20446562726973206F6E206E6FC2
:104680007A7A6C653F2057616974696E6720666F3E
:10469000722072657365742E0043757272656E7454
:1046A000005573656420647572696E672070726965
:1046B0006E74005049442063616C2E2066696E69F7
:1046C00073686564005049442063616C2E2020208B
:1046D000202020202020202000506C656173652060
:1046E00077616974004D31313720466972737420E7
:1046F0006C617965722063616C2E005072696E7412
:104700002070617573656400496E76616C69642020
:104710005049442063616C2E20726573756C74730C
:104720002E204E6F742073746F72656420746F2036
:10473000454550524F4D2E004D3530300047312009
:104740005A31352046313530300047393100473154
:104750002058353020593139302045302046373007
:10476000303000473930004D373032004D3730326D
:104770002043004D3730322055004D373032004D48
:104780003730322043004731205A31352046313509
:104790003030004739310047312058353020593109
:1047A0003930204530204637303030004D38330026
:1047B000473930004D3834004D313034205330000B
:1047C0004D3834004D3730322043004731205831C6
:1047D00030205931383020463430303000473120D5
:1047E0005A31302046313330302E303030004D31A8
:1047F0003430205330004D313034205330004731B5
:1048000020452D302E303735303020463231303093
:104810002E3030303030004D3130370047312058A5
:104820003530205935352045332E36323737330071
:1048300047312058323030205935352045302E341C
:104840003933383600473120583230302059373527
:104850002045332E36323737330047312058353034
:10486000205937352045302E34393338360047311A
:1048700020583530205939352045332E36323737D8
:1048800033004731205832303020593935204530F7
:104890002E343933383600473120583230302059E1
:1048A0003131352045332E3632373733004731200A
:1048B00058353020593131352045302E3439333890
:1048C00036004731205835302059313335204533B3
:1048D0002E363237373300473120583230302059A6
:1048E0003133352045302E363631373400473120CC
:1048F0005832303020593135352045322E36323756
:104900003733004731205831303020593135352088
:10491000453200473120583735205931353520454B
:10492000322E3500473120463130383000473120B3
:104930005A302E3135302046373230302E3030303C
:104940000047312058353020593135350047312066
:104950004634303030004D32303420533130303036
:10496000004731205A352046373230302E30303033
:1049700000473120452D312E353030303020463241
:104980003130302E3030303030004D383300473940
:104990003000473231004739322045302E30004751
:1049A0003120583130302E30204531322E352046DE
:1049B000313030302E30004731205836302E302004
:1049C00045392E302046313030302E3000473120EE
:1049D00058352E302045342E302046313030302EA0
:1049E00030004731205A302E3230204631303030BE
:1049F0002E30004731205835352E302045323520B5
:104A000046313430302E3000473120592D322E308F
:104A10002046313030302E3000473120583234308B
:104A20002E30204532352E30202046323230302E86
:104A300030004739322045302E30004731205A307F
:104A40002E332046313030302E300047312058355B
:104A5000352E302045382E302046323030302E3042
:104A60000047312058352E30204533322E30204635
:104A7000313830302E30004731205835352E302037
:104A80004533322E302046313037332E3000473117
:104A9000205A302E342046313030302E300047310D
:104AA00020592D332E302046313030302E30004DFD
:104AB0003833004739322045302E30004732380035
:104AC0004D3130392053323135004D31393020539A
:104AD0003630004D31343020533630004D313034D3
:104AE0002053323135004D3130370046696C616DED
:104AF000656E742073656E736F72005377617070AA
:104B000065640046726F6E742F6C65667420666112
:104B10006E7300417869730041786973206C656E2B
:104B2000677468004C6F6F73652070756C6C657985
:104B300000456E6473746F70206E6F7420686974C2
:104B400000456E6473746F70004D6F746F72004532
:104B50006E6473746F707300576972696E67206555
:104B600072726F7200426564202F2048656174651F
:104B700072004E6F7420636F6E6E656374656400BF
:104B80004865617465722F546865726D6973746FDE
:104B90007200506C6561736520636865636B203AD1
:104BA0000053656C6674657374206572726F722051
:104BB000210046696C616D656E742073656E736F5C
:104BC000723A005072696E742066616E3A004578E0
:104BD0007472756465722066616E3A0043616C6937
:104BE00062726174696E6720686F6D650053656CF1
:104BF0006674657374206661696C65642020004189
:104C00006C6C20636F7272656374202020202020FA
:104C100000436865636B696E672073656E736F72BE
:104C2000732000436865636B696E6720686F746505
:104C30006E64202000436865636B696E672062655F
:104C400064202020202000436865636B696E672024
:104C50005A2061786973202000436865636B696E30
:104C60006720592061786973202000436865636B71
:104C7000696E672058206178697320200043686559
:104C8000636B696E6720656E6473746F7073004543
:104C900072726F72202D20737461746963206D6568
:104CA0006D6F727920686173206265656E206F7622
:104CB00065727772697474656E0043617264207204
:104CC000656D6F766564002D2D2D2D2D2D2D2D2DCF
:104CD0002D2D2D2D2D2D2D2D2D2D2D0000000000E5
:104CE00000110A045052555341334446570020796D
:104CF000303D25640A002078303D25640A004F4B82
:104D00000A004552524F522061643D25640A00203A
:104D100020207A303D25640A00207A303D25640A3F
:104D2000002079303D25640A002078303D25640A52
:104D30000078797A63616C5F66696E645F706F6931
:104D40006E745F63656E746572320A000000210044
:104D5000240027002A002D0030003300010100004C
:104D6000040107010A0100002200250028002B0091
:104D70002E003100340002010000050108010B0182
:104D8000000020002300260029002C002F00320004
:104D900000010000030106010901050505050705DD
:104DA00008080808020202020A0A080804040404A7
:104DB00001010101010101010303030303030303D3
:104DC000040707070C0C0C0C0C0C0C0C0202020262
:104DD00006060606060606060B0B0B0B0B0B0B0B4B
:104DE00007070A0A0A0A0A0A05050504040408084E
:104DF00001021020200808102040102040800201ED
:104E000002010804020101020408102040808040D1
:104E100020100804020180040201804020100804D0
:104E2000020108040201010204081020408001026E
:104E3000040810204080100804088010204004401E
:104E400080102040048000000A0B02090C0D0E089F
:104E50000703040100000000000000000000000043
:104E60000000000000000000000000000000000042
:104E700000001211100000000000000000000000FF
:104E80000000000000000000000000000000000022
:104E900000000000000000000000000043616E6E92
:104EA0006F7420656E746572207375626469723AFE
:104EB000200053442063617264206F6B006F706543
:104EC0006E526F6F74206661696C656400766F6CFA
:104ED000756D652E696E6974206661696C65640024
:104EE000534420696E6974206661696C0057726969
:104EF00074696E6720746F2066696C653A2000469D
:104F0000696C652073656C65637465640020536922
:104F10007A653A200046696C65206F70656E65643D
:104F20003A20001F1F1F1F1F1F1F1F2E002E004E85
:104F30006F772066726573682066696C653A200039
:104F40004E6F7720646F696E672066696C653A20E2
:104F5000002220706F73002220706172656E743AB7
:104F60002200535542524F5554494E452043414C1F
:104F70004C207461726765743A2200747279696EAC
:104F80006720746F2063616C6C207375622D67639A
:104F90006F64652066696C65732077697468207436
:104FA0006F6F206D616E79206C6576656C732E2055
:104FB0004D4158206C6576656C2069733A00536FDB
:104FC0007274696E672066696C657300536F6D65F6
:104FD0002066696C65732077696C6C206E6F742035
:104FE000626520736F727465642E204D61782E2087
:104FF0004E6F2E206F662066696C657320696E2087
:105000003120666F6C64657220666F7220736F72F8
:1050100074696E67206973203130302E00000021E2
:1050200010422063308440A550C660E77008812993
:10503000914AA16BB18CC1ADD1CEE1EFF13112102B
:105040000273325222B5529442F772D662399318E3
:10505000837BB35AA3BDD39CC3FFF3DEE362244337
:105060003420040114E664C774A44485546AA54B33
:10507000B528850995EEE5CFF5ACC58DD5533672CB
:105080002611163006D776F6669556B4465BB77A83
:10509000A719973887DFF7FEE79DD7BCC7C448E557
:1050A000588668A7784008611802282338CCC9EDD3
:1050B000D98EE9AFF9488969990AA92BB9F55AD46B
:1050C0004AB77A966A711A500A333A122AFDDBDC23
:1050D000CBBFFB9EEB799B588B3BBB1AABA66C8777
:1050E0007CE44CC55C222C033C600C411CAEED8F73
:1050F000FDECCDCDDD2AAD0BBD688D499D977EB60B
:105100006ED55EF44E133E322E511E700E9FFFBEC2
:10511000EFDDDFFCCF1BBF3AAF599F788F8891A995
:1051200081CAB1EBA10CD12DC14EF16FE18010A16C
:1051300000C230E3200450254046706760B9839870
:1051400093FBA3DAB33DC31CD37FE35EF3B10290BC
:1051500012F322D2323542145277625672EAB5CB3C
:10516000A5A89589856EF54FE52CD50DC5E234C30C
:1051700024A01481046674476424540544DBA7FA10
:10518000B79987B8975FE77EF71DC73CD7D326F25C
:10519000369106B01657667676154634564CD96D5C
:1051A000C90EF92FE9C899E9898AB9ABA9445865AC
:1051B0004806782768C018E1088238A3287DCB5CB0
:1051C000DB3FEB1EFBF98BD89BBBAB9ABB754A54FC
:1051D0005A376A167AF10AD01AB32A923A2EFD0F7C
:1051E000ED6CDD4DCDAABD8BADE89DC98D267C074C
:1051F0006C645C454CA23C832CE01CC10C1FEF3E50
:10520000FF5DCF7CDF9BAFBABFD98FF89F176E369B
:105210007E554E745E932EB23ED10EF01E7C3C3E07
:105220005E2B3D3F2F5B5D3B2C2A225C00773235A5
:10523000783230636C5F63666D0A0077323578329E
:1052400030636C5F656E7465720A0020746F6F2046
:105250006C6F6E6720657874727573696F6E2070FD
:10526000726576656E7465640020636F6C6420659A
:105270007874727573696F6E2070726576656E747E
:105280006564004D373032004D373031004D3730D6
:1052900032004D37303100464C4558202D20203209
:1052A00034302F35300050502020202D2020323532
:1052B000342F3130300048495053202D20203232D5
:1052C000302F3130300041425320202D2020323504
:1052D000352F3130300050455420202D20203233DE
:1052E000302F383500504C4120202D2020323135D0
:1052F0002F3630004578747275646572006D6D00EC
:105300000059005800580059005A002563252E31D5
:1053100032533A2573252B30362E336600746F20B6
:10532000756E6C6F61642066696C616D656E74008A
:10533000746F206C6F61642066696C616D656E745A
:1053400000507265737320746865206B6E6F620025
:105350003E43616E63656C00507265686561746997
:105360006E6720746F2063757400507265686561A4
:1053700074696E6720746F20656A6563740050728B
:105380006568656174696E6720746F20756E6C6FF7
:1053900061640050726568656174696E6720746F3E
:1053A000206C6F6164005072656865617420746878
:1053B00065206E6F7A7A6C6521004552524F523AE1
:1053C0000046696C616D656E7420657874727564F1
:1053D000696E672026207769746820636F72726532
:1053E000637420636F6C6F723F004175746F6C6FF4
:1053F0006164696E672066696C616D656E742069B1
:1054000073206163746976652C206A7573742070EB
:105410007265737320746865206B6E6F6220616EB5
:105420006420696E736572742066696C616D656E67
:10543000742E2E2E00546F74616C207072696E741D
:105440002074696D6500546F74616C2066696C61CD
:105450006D656E74005072696E742074696D6500BC
:1054600046696C616D656E74207573656400526980
:10547000676874004C6566740059206469737461D0
:105480006E63652066726F6D206D696E0053657680
:1054900065726520736B657700536C69676874206B
:1054A000736B6577004D6561737572656420736B0E
:1054B0006577005B303B305D20706F696E74206FE4
:1054C00066667365740041646A757374696E6720FB
:1054D0005A00526573657400526561722073696485
:1054E00065205B756D5D0046726F6E742073696434
:1054F000655B756D5D0052696768742073696465EA
:105500005B756D5D004C6566742073696465205B36
:10551000756D5D005365742074656D70657261749E
:105520007572653A001B5B324A2553203A1B5B318A
:105530003B394825382E3266206D0A2553203A0A19
:1055400025376C6464203A253268686468203A25FF
:105550003032686864206D001B5B324A25533A1B69
:105560005B313B364825382E32666D200A255320A4
:105570003A1B5B333B38482532646820253032645F
:105580006D2025303264730025362E32666D6D0035
:105590004E2F41001B5B303B304825533A0A2553C0
:1055A0000A25533A0A25533A001B5B303B313548F4
:1055B0004E2F41001B5B303B31354825342E32667F
:1055C00001001B5B303B304825533A0A25530A251E
:1055D000533A202025352E3266010A25533A2020E1
:1055E00025352E32660100526573656E64002553C1
:1055F0003A20256C640A25530A002079645F6D699E
:105600006E3D25752079645F6D61783D2575207943
:10561000645F6176673D25752073685F6176673DDD
:1056200025750A002073745F73756D3D25752079AB
:10563000645F73756D3D25752065725F73756D3D93
:1056400025752065725F6D61783D256868750A0073
:10565000004B494C4C45442E20005072696E7465D5
:10566000722068616C7465642E206B696C6C2829EB
:105670002063616C6C656421004B494C4C3A2025D9
:10568000640A004D31303420496E76616C696420C3
:10569000657874727564657220004D31303520492B
:1056A0006E76616C696420657874727564657220C9
:1056B000004D31303920496E76616C69642065781F
:1056C00074727564657220004D32313820496E76EF
:1056D000616C696420657874727564657220004D30
:1056E00032323120496E76616C696420657874725B
:1056F0007564657220006673656E736F725F6F719B
:105700005F6D656173737572655F73746F702C2064
:10571000256868752073616D706C65730A00667327
:10572000656E736F725F6F715F6D656173737572B4
:10573000655F73746172740A004D363030005052E8
:10574000555341206673656E736F725F7265636F48
:10575000766572006673656E736F725F75706461F3
:105760007465202D204D3630300A006673656E73E7
:105770006F725F6572725F636E74203D20300A0045
:105780004731204533204632303000473120452D07
:105790003320463230300020573A0020453A00543A
:1057A0003A0048656174696E672064697361626C70
:1057B0006564206279207361666574792074696D0F
:1057C00065722E001000C90210012C014001220157
:1057D00070011801B0010E01F00104015002FA003D
:1057E000B002F0003003E600D003DC009004D200E9
:1057F0007005C800A006BE000008B400B009AA00E9
:10580000D00BA000600E960060118C000015820085
:1058100020197800C01D6E00A0226400B0275A0035
:10582000902C500000314600E0343C00103832002B
:10583000903A2800603C1E00A03D1400803E0A0003
:10584000203F000070012C0190012701B0012201CE
:10585000C0011D01F00118011002130130020E01F8
:105860006002090190020401C002FF000003FA0077
:105870004003F5008003F000D003EB002004E600B5
:105880007004E100E004DC004005D700C005D20050
:105890004006CD00D006C8008007C3003008BE0017
:1058A000F008B900C009B400B00AAF00B00BAA00FC
:1058B000D00CA500000EA000500F9B00C010960059
:1058C0005012910000148C00C0158700B0178200A0
:1058D000B0197D00D01B7800001E730040206E00C0
:1058E00090226900F024640040275F0090295A004C
:1058F000E02B5500102E500020304B001032460097
:10590000E033410090353C001037370070383200EA
:10591000A0392D00B03A2800A03B2300603C1E00B7
:10592000103D1900903D1400103E0F00703E0A001B
:10593000C03E0500003F000090137D00B0157800C8
:10594000F0177300601A6E00F01C6900A01F64005D
:1059500050225F0020255A00E0275500902A500071
:10596000202D4B00A02F4600F031410010343C00A8
:10597000F0353700A037320020392D00603A28007A
:10598000703B2300603C1E00203D1900C03D140008
:10599000403E0F00A03E0A00F03E0500403F0000E0
:1059A000703FFBFF903FF6FFB03FF1FFC03FECFFC1
:1059B000D03FE7FFE03FE2FFF03FDDFFF03FD8FFE1
:1059C00020484F54454E4420544845524D414C20A8
:1059D00052554E4157415900204845415442454493
:1059E00020544845524D414C2052554E4157415943
:1059F00000544845524D414C2052554E4157415953
:105A00000042454420544845524D414C2052554E89
:105A1000415741590020544845524D414C20525560
:105A20004E41574159202820505245484541542065
:105A3000484F54454E44290020544845524D414C4E
:105A40002052554E41574159202820505245484533
:105A5000415420484541544245442900505245484C
:105A6000454154204552524F520042454420505225
:105A70004548454154204552524F52004572723AB2
:105A8000204D494E54454D50204245440054656DCB
:105A900070657261747572652068656174656420F3
:105AA000626564207377697463686564206F6666F5
:105AB0002E204D494E54454D5020747269676765DC
:105AC0007265642021004572723A204D494E54455A
:105AD0004D50003A20457874727564657220737772
:105AE000697463686564206F66662E204D494E5464
:105AF000454D5020747269676765726564202100A6
:105B0000504154393132355F5245535F593D256814
:105B100068750A00504154393132355F5245535F40
:105B2000583D256868750A00555341525432207219
:105B3000782046756C6C2121210A005365747469C4
:105B40006E67732053746F7265640053746F72656F
:105B5000642073657474696E67732072657472690A
:105B6000657665640048617264636F6465642044AF
:105B7000656661756C742053657474696E67732013
:105B80004C6F6164656400563200000000C842003A
:105B900000C8420000C84300008C43000048430096
:105BA000004843000040410000F042E8030000E8E4
:105BB000030000C80000008813000000409C44005F
:105BC000409C440000000000000000204E00000047
:105BD00000204100002041CDCCCC3E000020400000
:105BE0000000000000000000000000CDCCCC3E3DD5
:105BF0000A8141FF08433EB099AB438F42FC42E625
:105C00005A343F4C62B045000000000040400000A4
:105C100034420000000000000000000000410000CD
:105C200000E03F0000C8420000C8420000404100C0
:105C300000F042C0030000C0030000C8000000885C
:105C4000130000454550524F4D204572726F72004F
:105C500057616974696E6720666F72206E6F7A7A19
:105C60006C6520616E642062656420636F6F6C698F
:105C70006E670053656C662074657374204F4B002B
:105C800053656C662074657374207374617274203C
:105C90002000457874722066616E207370656564BB
:105CA0003A202564200A005072696E742066616E85
:105CB0002073706565643A202564200A005465737A
:105CC0007420323A0A00457874722066616E20733F
:105CD000706565643A202564200A005072696E740C
:105CE0002066616E2073706565643A202564200A21
:105CF000005465737420313A0A006C63645F736505
:105D00006C66636865636B5F617869732025642CDA
:105D10002025640A004D3834004731205A3135209F
:105D2000463130303000473238205700256320415B
:105D3000584953205347313D25640A00417869731F
:105D4000206C656E67746820646966666572656E4E
:105D500063653A252E33660A004D65617375726579
:105D6000642061786973206C656E6774683A252ECB
:105D700033660A00436F6E74696E756520776974C7
:105D80006820616E6F7468657220626F7764656EFB
:105D90003F0025002020202020200020202020203F
:105DA000200045524153494E4720616C6C2064618C
:105DB000746100466163746F727920524553455493
:105DC0000000007F43008054430000524300000065
:105DD00000000080C09A99193E0000000000008079
:105DE000C09A99193E0000A0400000A040000000A9
:105DF0004025336420737465703D253264206D73D3
:105E0000636E743D2534640A0000007F43008058AF
:105E1000439AD95143FFFFFF46696C616D656E740B
:105E2000206F7574206F662072616E67652025642F
:105E3000200A0067636F64655F4D3730312062650B
:105E400067696E0A00332E372E302D5243310072AF
:105E500063006265746100616C70686100646576FE
:105E60000078797A63616C5F73706972616C32205B
:105E700063783D25642063793D2564207A303D2593
:105E80006420647A3D2564207261646975733D25E0
:105E9000642061643D25640A00746D6332313330DF
:105EA0005F676F746F5F737465702025642025646D
:105EB000202564202564200A002E006F70656E2066
:105EC0006661696C65642C2046696C653A20004DFA
:105ED0003234004D3233202573006175746F2569AB
:105EE0002E670022206661696C65643A20427566FF
:105EF0006665722066756C6C2100456E717565690A
:105F00006E6720746F207468652066726F6E743AD5
:105F10002022004572726F723A002200456E717540
:105F200065696E6720746F207468652066726F6E95
:105F3000743A2022006563686F3A004572723A2015
:105F40005052494E542046414E204552524F520025
:105F50005072696E742066616E207370656564208E
:105F60006973206C6F776572207468656E20657840
:105F7000706563746564004572723A2045585452E6
:105F80002E2046414E204552524F520045787472A1
:105F9000756465722066616E207370656564206942
:105FA00073206C6F776572207468656E20657870F9
:105FB0006563746564002F2F20616374696F6E3AA6
:105FC0007061757365004572723A204D41585445B1
:105FD0004D50003A2045787472756465722073776D
:105FE000697463686564206F66662E204D4158545D
:105FF000454D5020747269676765726564202100A1
:106000004572723A204D415854454D502042454406
:106010000054656D706572617475726520686561A4
:10602000746564206265642073776974636865646D
:10603000206F66662E204D415854454D5020747295
:106040006967676572656420210046696C2E205877
:10605000643A2533642059643A2533640A496E74DE
:106060003A202533642020536875743A2025336420
:106070000046696C616D656E742073656E736F7236
:106080000A69732064697361626C65642E001B5B2E
:10609000303B304825533A202534642052504D0A75
:1060A00025533A20202534642052504D0A00507266
:1060B000696E742046414E004E6F7A7A6C652046B8
:1060C000414E00546F74616C004C617374207072A7
:1060D000696E74004D4D55206C6F61642066616976
:1060E0006C73004D4D55206661696C73004C617393
:1060F00074207072696E74206661696C7572657364
:10610000004D4D5520706F776572206661696C7324
:10611000004D4D55206C6F6164206661696C7300A1
:106120004D4D55206661696C7300546F74616C202D
:106130006661696C757265730043726173680046CD
:10614000696C616D2E2072756E6F75747300506F7F
:10615000776572206661696C7572657300546F743F
:10616000616C206661696C7572657300437261735E
:10617000680046696C616D2E2072756E6F75747360
:1061800000506F776572206661696C757265730087
:106190004C617374207072696E74206661696C75ED
:1061A00072657300546F74616C004C61737420707D
:1061B00072696E7400416D6269656E740042656457
:1061C000004E6F7A7A6C650042656C74207374615E
:1061D00074757300436F6F6C646F776E00566F6CED
:1061E00074616765730054656D7065726174757272
:1061F00065730042656C7420737461747573005329
:10620000656E736F7220696E666F00457874727583
:1062100064657220696E666F0058595A2063616C1C
:106220002E2064657461696C7300756E6B6E6F7798
:106230006E004D4D553220636F6E6E6563746564FC
:1062400000446174653A00686F77746F2E707275E0
:10625000736133642E636F6D00666F72756D2E709F
:106260007275736133642E636F6D00707275736144
:1062700033642E636F6D001B5B303B304825531B2E
:106280005B313B314825532020252D33641B5B3285
:106290003B314825532020252D33641B5B333B3194
:1062A00048001B5B303B304825531B5B313B31487A
:1062B00025532020252D33641B5B323B3148255369
:1062C0002020252D33641B5B333B3148255320258B
:1062D0002D3364001B5B303B304825531B5B313B47
:1062E000314825532020252D33641B5B323B314838
:1062F00025532020252D33641B5B333B3148255328
:1063000020205820252D336420205920252D33644A
:10631000001B5B303B304825531B5B313B3148252C
:10632000532020252D33641B5B323B3148255320FD
:1063300020252D33641B5B333B31482553202058E7
:1063400020252D336420205920252D3364001B5B2C
:10635000323B314825533A2020256425631B5B33AB
:106360003B314850494E44413A20202020256425A5
:1063700063001B5B303B314825533A2020202564C5
:1063800025631B5B313B314825533A2020202020D8
:106390002025642563001B5B313B31485057523A3E
:1063A00020202020202025642E25303164561B5BC0
:1063B000323B31484245443A2020202020202564A9
:1063C0002E2530316456001B5B303B314825531B72
:1063D0005B313B3248582025641B5B323B324859C5
:1063E00020256400464C4558202D20203234302F83
:1063F00035300050502020202D20203235342F31D0
:1064000030300048495053202D20203232302F3177
:1064100030300041425320202D20203235352F319D
:1064200030300050455420202D20203233302F387A
:106430003500504C4120202D20203231352F363070
:1064400000414253202020202D20203235352F318D
:106450003030006E6F7A7A6C65202D202032353016
:106460002F30006661726D2020202D2020323530C3
:106470002F363000466C61736841697220495020A4
:10648000416464723A004D4D553220202020202076
:10649000204E2F410025642E25642E25642D256471
:1064A000002046573A0041707220203120323031AE
:1064B0003900453344763666756C6C0045494E5359
:1064C000795F31306100315F37356D6D5F4D4B3332
:1064D000002D2D2D2D2D2D2D2D2D2D2D2D0020720E
:1064E00065706F20416E67656C530020332E372E28
:1064F000302D5243312D32313735004669726D7778
:106500006172653A0025642E25642E25642E25646B
:10651000002563252E3132533A2573252B30362E34
:106520003166002020202020202020202020202034
:1065300020202020202020003E003E0020003E00A1
:106540003E0020004E6F74207370696E6E696E6736
:10655000005370696E6E696E67004C6566742068E2
:106560006F74656E642066616E3F0046726F6E7474
:10657000207072696E742066616E3F0046616E2005
:106580007465737400009D01890111241FBECFEF53
:10659000D1E2DEBFCDBF00E00CBF16E0A0E0B2E06C
:1065A000E8EAFFE803E00BBF02C007900D92A03BB2
:1065B000B107D9F729E1A0EBB6E001C01D92AB3DD0
:1065C000B207E1F712E3C4ECD2E300E006C0219782
:1065D0000109802FFE010F94E7C6C33CD10780E07C
:1065E0000807A9F70F940B9C0D94C3C70C940000E7
:1065F0002F923F924F925F926F927F928F929F92D3
:10660000AF92BF92CF92DF92EF92FF920F931F93C0
:10661000CF93DF93CDB7DEB7C458D1090FB6F89446
:10662000DEBF0FBECDBF80917F1390918013892B69
:1066300011F40C94EF7582E090E09093290280931E
:10664000280284E493E00F9405668823B1F08091DA
:10665000100D9091110D6AE270E005960F9442C7FB
:10666000009711F0DC011C928091100D9091110D9A
:1066700005960F94CE0C0C94C370C0906E15D090FC
:106680006F1586010C571C4E46E050E065E771E13E
:10669000C8010F9471BA892B09F0EFC089E493E027
:1066A0000F940566882309F49BC088E50F94CEB447
:1066B000182F89E50F94CEB4811112600F94CB8E00
:1066C0008091B10601E0080F0093B106811105C069
:1066D00084E696E10F94271C0EC048EC5FEA60E068
:1066E00070E084E696E10F94E21B882331F010926B
:1066F00064161092B10601E007C0033049F710920A
:1067000064161092B10600E081E00E9442F80E94F7
:1067100038F882E00E9466F010FF15C086E69FE020
:106720000F946EC161E0680F86E69FE00F9480C110
:1067300085E09FE00F947BC1BC016F5F7F4F85E0D8
:106740009FE00F949AC111FF15C088E69FE00F9457
:106750006EC161E0680F88E69FE00F9480C183E01E
:106760009FE00F947BC1BC016F5F7F4F83E09FE090
:106770000F949AC181E00E9442F882E00E9466F084
:106780008EE493E10F944C0B40E061E081E00F94C4
:10679000CF740F94CB8E002321F061E082E19EE064
:1067A0001BC0E091060DF0E0EE0FFF1FE158FA4E1E
:1067B0001182108240E060E080E393E10E94F6D312
:1067C000182F81E00E9442F861E0112319F084E063
:1067D0009EE002C087EF9DE00E9408970C94C37072
:1067E00088E593E00F940566882379F08091F50D94
:1067F000882331F060E070E080E89FE30E9497A575
:1068000081E0809310020C94C37086E693E00F94AD
:106810000566882311F40C94C3701092F50D81E085
:10682000809310028091550D811104C00E9442DCBA
:106830000C94C370813011F00C94C370E6EEFDE04F
:1068400084918F01882339F00F946F550F5F1F4F8C
:10685000F8018491F7CF8AE00F946F55EAE5F8E1EB
:1068600084918F01882311F40C94556F0F946F5508
:106870000F5F1F4FF8018491F5CF44E050E060E7CF
:1068800071E1C8010F9471BA892B09F00EC186011C
:1068900008571C4E49E050E066E671E1C8010F94CC
:1068A00071BA892BD9F4F601EF56FC4E10811534DC
:1068B00031F01855143010F00C94C37001C013E07F
:1068C0004AE050E060E070E0C6018E569C4E0F94A6
:1068D00028B8812F0F9467790C94C37049E050E079
:1068E0006CE571E1C8010F9471BA892B61F5F6016D
:1068F000EF56FC4E1081153431F01855143010F05D
:106900000C94C37001C013E04AE050E060E070E016
:10691000C6018E569C4E0F9428B8E12FF0E0E85E39
:10692000F84F40E051E0008002C0569547950A9428
:10693000E2F7842F880F880F81506823812F0F94EE
:10694000157B0C94C37049E050E062E571E1C80129
:106950000F9471BA892B11F00C94C370F601EF56A5
:10696000FC4E8081853449F008EA902E980EF3E0C1
:10697000F91510F40C94C37002C013E0912EE92CA9
:10698000F12C5701AA0CBB1CF501EC5CFD4F1081EA
:10699000012F0F70712E7294BFE07B22272D27707C
:1069A000722E111F1127111F61816770660F162B40
:1069B000F501EB5CFD4F8081882E86948694869449
:1069C000382D3370832E1A821982C6018E569C4E42
:1069D000DC012C912223E1F14AE050E0BE016F5F1F
:1069E0007F4F0F9428B8062F0F7089819A810097E6
:1069F00079F1FC012081222359F14AE050E0BE01E7
:106A00006F5F7F4F0F9428B86770762E89819A81C7
:106A10000097F1F0DC012C912223D1F04AE050E004
:106A2000BE016F5F7F4F0F9428B8162F1F708981AA
:106A30009A81009769F0FC012081222349F04AE005
:106A400050E0BE016F5F7F4F0F9428B86370862EB1
:106A5000F501EC5CFD4F972D97709295907F612F1B
:106A6000679566276795902B962B9083612F669587
:106A70001181107E882D8370880F880F880F162B48
:106A8000182B1183C701815E9D4FD701AD5DBD4FAE
:106A9000B701685E784FFC0120814C91DB016C915D
:106AA000892D0E94ABBE0C94C37083E793E00F94D2
:106AB0000566882309F4BFC189E793E00F94056652
:106AC000882391F080913F0F882311F40C94C370B8
:106AD0000F94A45960937A1670937B1680937C165A
:106AE00090937D160C94C3708EE793E00F94056627
:106AF000882349F08091920D8F938091910D8F930F
:106B000088EC97E03DC082E893E00F940566882307
:106B100029F140913310509134102CE3249FC0018F
:106B2000259F900D11249F938F9340913110509188
:106B30003210249FC001259F900D11249F938F93A5
:106B400081EB97E09F938F930F949EBB0F900F90D4
:106B50000F900F900F900F900C94C37086E893E005
:106B60000F9405668823C9F080913F0F882391F028
:106B7000809132078F93809131078F938EEA97E04F
:106B80009F938F930F949EBB0F900F900F900F9039
:106B90000C94C3708CE997E0FAC089E893E00F94F5
:106BA0000566882321F0109230070C94C3708DE89D
:106BB00093E00F940566882349F060E085EA9FE042
:106BC0000F9480C161E08EE491E106CE82E993E00A
:106BD0000F940566882321F00E94A2900C94C37044
:106BE00082EA93E00F940566882321F00E9430A189
:106BF0000C94C37089EA93E00F940566882319F119
:106C000080913F0F8823C9F08AEA95E5DC018093E3
:106C1000FC1F9093FD1FA093FE1FB093FF1F88E001
:106C20008093FB1F98E10FB6F894A89590936000AD
:106C30000FBE80936000F894FFCF8FEA93E00F942B
:106C400071560C94C37081EC93E00F940566882311
:106C500039F18091100D9091110D41E061E00396A2
:106C60000F941F128091AE189091AF18A091B01898
:106C7000B091B11880935B1990935C19A0935D1942
:106C8000B0935E1986EA98E10F941E228C010F944E
:106C90006F550A30110531F70F947B810C94C37046
:106CA00084EC93E00F940566882381F00F94D86CF0
:106CB00081E0809343078091100D9091110D41E088
:106CC00060E004960F941F120C94C37088EC93E05C
:106CD0000F940566882309F45EC080913F0F8823D6
:106CE00009F453C0109281156091D5197091D6198D
:106CF0008BE390E00F9419BB6091D5197091D61970
:106D000083E590E00F9419BB19821B821A82CE0191
:106D100001960F94D61B00E010E0FF24F3948091BD
:106D2000A30E9091A40E2091A50E3091A60E821B69
:106D3000930B8F779927892B81F00F94CB54F09286
:106D400081156091D5197091D61990E00F9419BBF7
:106D50000F5F1F4F10928115E2CF64E670E0CE0105
:106D600001960F94AD1B811103C003311105BCF2D4
:106D700081E0809381156091D5197091D6198AE0D0
:106D800090E00F9419BB0C94C37089EA95E00F94BE
:106D9000C6BB0C94C3708BEC93E00F9405668823FC
:106DA00061F00FEC13E0F80181918F01882311F459
:106DB0000C94556F0F946F55F6CF8EED93E00F94B2
:106DC0000566882361F002EE13E0D8018D918D01F4
:106DD000882311F40C94556F0F946F55F6CF81E012
:106DE00094E00F94056681110C94C37086E094E0E2
:106DF0000F940566882341F060E070E088EF9FE023
:106E00000F94A2400C94C37089E094E00F9405663F
:106E1000882321F00F94A4590C94C3708EE094E061
:106E20000F940566882311F40C94C37080E00F94CE
:106E3000FB670C94C3708EE50F94CEB481110C9453
:106E4000C37087E40F94CEB4F82E882311F40C9409
:106E500023470F94C6B40F9459C36C34710509F4D9
:106E600001C27CF56430710509F4F8C054F4623055
:106E7000710509F4DEC00CF0E5C077FF69C00C9421
:106E800017476C31710509F43BC15CF46A30710538
:106E900009F431C16B30710511F00C94174780E093
:106EA0002BC16E31710509F46DC16B34710511F0A0
:106EB0000C94174708E210E0FEE6EF2EF7E0FF2EF5
:106EC000B2C16835710511F40C94C370CCF461350E
:106ED000710511F40C94DE4534F46035710509F444
:106EE00030C70C9417476635710511F40C9487462A
:106EF0006735710511F00C94174781E00C948846B2
:106F00006C35710511F40C9490467CF46A3571056A
:106F100011F40C948C466B35710511F00C941747E5
:106F200081E08093830F0C94C3706236710511F475
:106F30000C94F0466336710511F00C9417471092CB
:106F40003F0F60E084EC9FE00F9480C10C941247E7
:106F50008091BC0F81110C94C3700F9457B3609152
:106F6000E20D7091E30D8091E40D9091E50D0F9489
:106F700097BC6B017C014090621050906310609050
:106F800064107090651080904C0F90904D0FA09001
:106F90004E0FB0904F0FA5019401C301B2010F94A1
:106FA000F9C120E030E048EC52E40F9400B69B01B8
:106FB000AC01C701B6010F9445C41816D4F4A3015F
:106FC0009201C501B4010F94F9C120E030E048EC12
:106FD00052E40F9400B6A70196010F94FAC10F94E2
:106FE0005FC36093E20D7093E30D8093E40D909383
:106FF000E50D80911C11882311F40C94C17088E573
:107000000F94CEB481110C94C17089E50F94CEB465
:1070100081110C94C1708AE50F94CEB481110C9447
:10702000C17085E40F94CEB481110C9498700C94C7
:10703000C1708091BC0F81110C94C3700F9414B473
:1070400081E008C08091BC0F81110C94C3700F9433
:1070500014B480E00F9426AD0C94C37080E50F94B7
:10706000CEB4882339F00F94C6B40F945FC36B017C
:107070007C0103C0C12CD12C760183E50F94CEB4E2
:10708000882361F00F94C6B420E030E04AE754E46E
:107090000F9400B60F945FC36B017C01C114D1043F
:1070A000E104F10421F083E997E00F944C0B0F9475
:1070B000CB8E0F94A459C60ED71EE81EF91E0F944E
:1070C000A4596093880F7093890F80938A0F9093CF
:1070D0008B0F0F94A4596C157D058E059F0510F03C
:1070E0000C94C3700F94FF8780E00F94394680E0C2
:1070F0000E9466F0EECF81E00F940CAB0C94C3704D
:1071000088E50F94CEB48AAF0F94BCB41B012C0158
:1071100089E50F94CEB4682E0F94BCB422966CAF60
:107120007DAF8EAF9FAF22978AE50F94CEB4D82E55
:107130000F94BCB44B015C0187E50F94CEB4782E5C
:1071400083E40F94CEB47F928F93CD2C2296ECAC37
:10715000FDAC0EAD1FAD2297262DB201A1018AAD67
:107160000F94EF710F900F90BAADB1110C94C370E2
:1071700061100C94C37071100C94C370D1100C94F6
:10718000C370DFC50F94CB8E81E00F941B648C011C
:1071900080E090E0A8E4B4E4809356029093570214
:1071A000A0935802B093590243E060E070E080E29F
:1071B00091EC0F944B10809161108F93809160102F
:1071C0008F9380915F108F9380915E108F93809149
:1071D0005D108F9380915C108F9380915B108F93E3
:1071E00080915A108F93809159108F9380915810ED
:1071F0008F93809157108F93809156108F9381E3D6
:107200009DE39F938F9387E797E09F938F930F94CE
:107210009EBBC8010F94FA630FB6F894DEBF0FBE91
:10722000CDBF0C94C370B801012E000C880B990BD4
:107230000F9499BC0E94E9B19F938F937F936F93B2
:107240001F930F93FF92EF920F949EBB0F5F1F4F00
:107250000FB6F894DEBF0FBECDBF0F36110519F77C
:107260000C94C3700F94556B8A3F30F08CE194E11D
:107270000E949AD40C94C3708091070D882341F02A
:107280008091080D882321F08091090D811106C09D
:1072900081E080937E1387E491E16DC585ED93E1F4
:1072A0000E949AD440E060E086E29CE10E94F6D31E
:1072B000882309F493C080E090E0A0EAB0E48093D2
:1072C0005E1090935F10A0936010B09361102091B6
:1072D0005A1030915B1040915C1050915D1060919C
:1072E0005610709157108091581090915910F6E0F7
:1072F0006F2EFDE07F2E7F926F92812C912CA8E45F
:10730000AA2EA2E4BA2EB2E6CB2EB0E1DB2EE12CFF
:10731000F12C00EA10E40F942D2780925E109092D9
:107320005F10A0926010B092611080E090E0A4E342
:10733000B3E480935A1090935B10A0935C10B093C9
:107340005D10609156107091571080915810909177
:1073500059107F926F928501740120E030E044E380
:1073600053E40F942D270F94CB8E8EEF9BE10E9458
:107370009AD4E2E6FFE1259135914591549120930D
:107380005A1030935B1040935C1050935D10EEE503
:10739000FFE165917591859194916093561070937A
:1073A00057108093581090935910E0905E10F09011
:1073B0005F1000916010109161107F926F920F9496
:1073C0002D270F94CB8E41E060E080E00F94CF74C6
:1073D0000F900F900F900F900F900F9020E030E0E3
:1073E0004CE052E460919219709193198091941934
:1073F000909195190F9445C418160CF0A4C0809173
:107400003F0F8111A0C080E090E0A8ECB2E480932F
:107410005E1090935F10A0936010B0936110209164
:107420005A1030915B1040915C1050915D1060914A
:107430005610709157108091581090915910E6E0B5
:10744000FDE0FF93EF93812C912C18E4A12E12E420
:10745000B12E02E6C02E00E1D02EE12CF12C08EC7A
:1074600012E40F942D2780E090E0ACE0B2E48F8F1F
:1074700098A3A9A3BAA30E9416F319821A821B82A9
:107480001C82CE0101960F94E08010920B0D109299
:107490000A0D19821A821B821C821D82CE0101965E
:1074A0000F94271C0F900F902F8D38A149A15AA13E
:1074B00060919219709193198091941990919519F6
:1074C0000F9445C4181694F580E193E10E94A8D367
:1074D00064E080E00E9442F382E00E944D8C82E9E9
:1074E00099E10E94D8910E94DFF181E194E00E942D
:1074F000DFF1CE014F960E94D8910E94DFF183E127
:1075000094E00E94DFF188EE93E00F947C4A0E94A1
:1075100093B140E053E567E070E0CE0101960F942F
:10752000E21B882309F4C0CF10E001C011E06CED2C
:107530007CE481E00E94F7F281E00E9442F81111A0
:1075400002C080E0FAC381E00E9442F881E090E04E
:107550009093290280932802E9E2F1E184918F015E
:10756000882339F00F946F550F5F1F4FF8018491F6
:10757000F7CF8AE00F946F551A821982C090921942
:10758000D0909319E0909419F090951920E030E094
:1075900040EA50E4C701B6010F94E8C20F9459C302
:1075A00025E0269FA001279F500D1124BA01550FF9
:1075B000880B990B0F9499BC3B01382E292E20E0A3
:1075C00030E04CE052E40F9493BC87FF06C0612C7E
:1075D000712CACE03A2EB2E42B2EC101262D372DB2
:1075E000492F522DC701B6010F9445C4181674F4E3
:1075F00020E030E040EA50E4F101662D772D8F2F36
:10760000922D0F94FAC13B01382E292E2F923F92D2
:107610007F926F9285E597E09F938F930F949EBB27
:1076200020E030E040EF51E4F101662D772D8F2FFF
:10763000922D0F94F9C120E030E04CE852E40F9411
:10764000FAC10F9459C370930B0D60930A0D84E037
:1076500090E09093DB0D8093DA0D81E090E09093C1
:10766000FF0E8093FE0E8BE89CE20F944C0B80E0A3
:1076700090E0A0EAB0E480935E1090935F10A09336
:107680006010B093611020915A1030915B104091BE
:107690005C1050915D106091561070915710809160
:1076A000581090915910B6E04B2EBDE05B2E5F92C2
:1076B0004F92812C912C18E4A12E12E4B12E02E6F7
:1076C000C02E00E1D02EE12CF12C00EA10E40F9442
:1076D0002D2780E090E0A0EAB1E4809356109093CB
:1076E0005710A0935810B093591080E090E0A0E795
:1076F000B2E480935A1090935B10A0935C10B09307
:107700005D10E0905E10F0905F100091601010919D
:1077100061105F924F929C01AD0160E070E080EAE1
:1077200091E40F942D278AE999E9A9E1BEE38093BA
:107730005E1090935F10A0936010B0936110209141
:107740005A1030915B1040915C1050915D10609127
:1077500056107091571080915810909159105F9267
:107760004F921AE9E12E19E9F12E09E11EE30F9477
:107770002D270F94CB8E0FB6F894DEBF0FBECDBF72
:107780002091921930919319409194195091951923
:10779000F101662D772D8F2F922D0F9445C4181669
:1077A0003CF488EE93E00F947C4A0E9493B1E8CFBA
:1077B00060E086EA9FE00F9480C180E090E0A0EA5C
:1077C000B0E480935E1090935F10A0936010B0932C
:1077D000611020915A1030915B1040915C105091D3
:1077E0005D106091561070915710809158109091D3
:1077F000591006E0402E0DE0502E5F924F92812CE2
:10780000912CE8E4AE2EE2E4BE2EF2E6CF2EF0E1BB
:10781000DF2EE12CF12C00EA10E40F942D27EEE589
:10782000FFE16591759185919491609356107093E5
:1078300057108093581090935910E2E6FFE125917C
:1078400035914591549120935A1030935B10409399
:107850005C1050935D10E0905E10F0905F1000910E
:107860006010109161105F924F920F942D270F942A
:10787000CB8E43E060E070E080E89FEB0F944B100C
:107880000F900F900F900F90882309F45ACE3091EB
:107890005E1027963FAF279740915F102B964FAF12
:1078A0002B97509160102F965FAF2F9780916110AA
:1078B00063968FAF63978F935F934F933F9388E463
:1078C00097E09F938F930F949EBB0F900F900F9014
:1078D0000F900F900F90AEEABFE0BFAFAEAF442461
:1078E0004A94542C13E2C12ED12CE12CF12C8201AC
:1078F000B6010D2C000C880B990B0F9499BC4B0111
:107900005C01A7014F5F5F4F5BAF4AAFDF92CF9241
:107910005F934F938CE097E09F938F930F949EBB60
:107920000F900F900F900F900F900F90BFEF4B168E
:107930005B0611F40C949875BE016F5F7F4F8EAD9E
:107940009FAD0F94A240A5019401F101662D772D02
:107950008F2F922D0F9493BC1816ACF4E5E0EE1621
:10796000F10479F0B5E0CB0ED11CEFEF4E1A5E0AB0
:107970002EAD3FAD2E5F3F4F3FAF2EAFEAACFBAC1D
:10798000B6CF05E010E0C8018752984F4C01880C33
:10799000991C9BAE8AAE380123E0620E711C25E073
:1079A000209FC001219F900D11241FAE1EAEAC017F
:1079B000435D5F4F68965FAF4EAF6897A6E04A2E73
:1079C000ADE05A2EC301029705970CF0B5C1689639
:1079D0006EAD7FAD68978EAD9FAD680F791F072E96
:1079E000000C880B990B0F9499BC26966CAF7DAF59
:1079F0008EAF9FAF26977F926F92AFEFB6E0BF93A7
:107A0000AF930F949EBB7092FF0E6092FE0E20E02B
:107A100030E040EF51E426966CAD7DAD8EAD9FAD6C
:107A200026970F94F9C120E030E040E251E40F9432
:107A300000B620E030E040EA50E40F94E8C220E0D5
:107A400030E048E452E40F94FAC10F9459C37093A4
:107A50000B0D60930A0D80E090E0A0EAB0E4809303
:107A60005E1090935F10A0936010B093611020910E
:107A70005A1030915B1040915C1050915D106091F4
:107A800056107091571080915810909159105F9234
:107A90004F92812C912CF8E4AF2EF2E4BF2EA2E697
:107AA000CA2EA0E1DA2EE12CF12C00EA10E40F94AA
:107AB0002D27812C912C10EAA12E11E4B12E809259
:107AC000561090925710A0925810B092591020E082
:107AD00030E040E752E420935A1030935B1040931B
:107AE0005C1050935D10E0905E10F0905F1000917C
:107AF0006010109161105F924F92812C912C88E45C
:107B0000A82E82E4B82E60E070E080EA91E40F9441
:107B10002D278AE999E9A9E1BEE380935E1090934D
:107B20005F10A0936010B093611020915A103091B3
:107B30005B1040915C1050915D10609156107091F7
:107B4000571080915810909159105F924F921AE9F6
:107B5000E12E19E9F12E09E11EE30F942D270F9470
:107B6000CB8E0FB6F894DEBF0FBECDBF2091921919
:107B700030919319409194195091951926966CADB6
:107B80007DAD8EAD9FAD26970F9445C418163CF47D
:107B900088EE93E00F947C4A0E9493B1E7CF80E097
:107BA00090E0A0EAB0E480935E1090935F10A09301
:107BB0006010B093611020915A1030915B10409189
:107BC0005C1050915D10609156107091571080912B
:107BD0005810909159105F924F92812C912CB8E4DB
:107BE000AB2EB2E4BB2E12E6C12E10E1D12EE12C59
:107BF000F12C00EA10E40F942D27EEE5FFE16591EA
:107C0000759185919491609356107093571080935D
:107C1000581090935910E2E6FFE125913591459176
:107C2000549120935A1030935B1040935C10509302
:107C30005D10E0905E10F0905F1000916010109168
:107C400061105F924F920F942D270F94CB8E43E0DB
:107C500060E070E080E89FEB0F944B10EEADFFAD5D
:107C60003596FFAFEEAFFFEF6F1A7F0A0F900F90C0
:107C70000F900F90811103C00F9464AA5DC02796E6
:107C80007FAD27972B966FAD2B972F969FAD2F9794
:107C900063968FAD6397272F362F492F582F60910A
:107CA0005E1070915F1080916010909161100F9440
:107CB000F9C1162F072FF82EE92E2091A61030912A
:107CC000A7104091A8105091A910D801F7016B2F6F
:107CD0007A2F8F2F9E2F0F9400B60F9459C37A835B
:107CE0006983EF92FF920F931F93809195198F9361
:107CF000809194198F93809193198F938091921909
:107D00008F93A3ED8A2EA6E09A2E9F928F920F94C6
:107D10009EBBBE016F5F7F4F8AAD9BAD0F94A240AB
:107D20002AAD3BAD2E5F3F4F3BAF2AAF0FB6F89465
:107D3000DEBF0FBECDBF46CE81E00F9464AA0C9487
:107D4000C37081E08093F30D8091070D882341F08B
:107D50008091080D882321F08091090D811113C0B5
:107D600080912A0F90912B0F029749F081E0809328
:107D70007E1382E291E10F9479830C94C370109288
:107D8000F30D0C94C3708EE40F94CEB4882341F0AD
:107D90000F94B0B48AAF873041F053E05AAF05C0BA
:107DA0008BEA9DE00F946EC18AAF82E50F94CEB44A
:107DB000882349F00F94B0B42B968FAF2B978B305C
:107DC00048F08AE004C08AEA9DE00F946EC12B96C9
:107DD0008FAF2B978CEA9DE00F946EC16B968FAF9F
:107DE0006B9780912A0F90912B0F029741F2A091EF
:107DF000DA0DB091DB0D6E96BFAFAEAF6E97E0912E
:107E0000FE0EF091FF0EA096FFAFEEAFA09781E0BF
:107E100090E09093DB0D8093DA0D9AAC892C912C35
:107E200024969FAE8EAE2497BAACBB9C5001112411
:107E30006096BFAEAEAE6097C5010A969093FF0EF6
:107E40008093FE0E81E00E9466F00F94147C0E94E5
:107E50003BEB80E090E0A0EAB0E480935E1090936A
:107E60005F10A0936010B093611020915A10309170
:107E70005B1040915C1050915D10609156107091B4
:107E800057108091581090915910B6E06B2EBDE0BC
:107E90007B2E7F926F9215E5812E982CA82C11E4F1
:107EA000B12E02E6C02E00E1D02EE12CF12C00EA2A
:107EB00010E40F942D2780E090E0A0E8BFE38093CA
:107EC000561090935710A0935810B0935910809368
:107ED0005A1090935B10A0935C10B0935D106AE50C
:107EE00070E186E590E10F94C766E0905E10F09037
:107EF0005F10009160101091611020915A10309124
:107F00005B1040915C1050915D1060915610709123
:107F1000571080915810909159107F926F92812C38
:107F2000912CF8ECAF2EF2E4BF2E0F942D270F9476
:107F3000CB8E0F94BBAA8EAF80E00F941B64A496E7
:107F40009FAF8EAFA4970F900F900F900F90312C92
:107F50002AAD2150A5962FAFA59724968EAD9FAD43
:107F60002497092E000CAA0BBB0BA9968CAF9DAFD2
:107F7000AEAFBFAFA99724968EAD9FAD2497019762
:107F80004C01990FAA08BB08AD968CAE9DAEAEAE63
:107F9000BFAEAD97A32CB12C6496BFAEAEAE6497C6
:107FA00060962EAD3FAD60972A153B0509F42AC2B5
:107FB000832D6AAD0F948BC627968FAF2797292EF6
:107FC00080FF05C0A5963FADA597391B232E4AAD6E
:107FD000473099F4822D63E00F948BC6911112C043
:107FE00027968FAD27970F948BC691110BC00F94D6
:107FF000BBAA81110C94A77505C05EAD51110C94FC
:10800000B67501C01EAE412C512C3201211012C098
:1080100027968FAC279781100DC020E030E040EA12
:1080200050E420935E1030935F10409360105093A3
:10803000611024C0A9966CAD7DAD8EAD9FADA997A2
:108040000F9499BC9B01AC0160E070E080E090E48B
:108050000F94E8C29B01AC0160915E1070915F10BB
:1080600080916010909161100F94FAC160935E103E
:1080700070935F10809360109093611080915E10F8
:1080800090915F10A0916010B09161106A968CAFD2
:108090009DAFAEAFBFAF6A9720915A1030915B1081
:1080A00040915C1050915D10609156107091571086
:1080B0008091581090915910A6E0BDE0BF93AF9306
:1080C000812C912CF0EAAF2EF1E4BF2EA2E6CA2E4D
:1080D000A0E1DA2E6A96ECACFDAC0EAD1FAD6A974E
:1080E0000F942D270F94CB8EAD966CAD7DAD8EADDC
:1080F0009FADAD970F9499BC6B017C01622D70E030
:1081000080E090E00F9497BC20E030E04CE453E432
:108110000F9400B6A70196010F94E8C220E030E06A
:1081200040E85FE30F94FAC16093561070935710C4
:1081300080935810909359102796FFAD27976F2F73
:1081400070E080E090E00F9497BC20E030E04CE4D9
:1081500053E40F9400B6A70196010F94E8C220E003
:1081600030E040E85FE30F94FAC160935A107093D7
:108170005B1080935C1090935D106AE570E186E57A
:1081800090E10F94C766E0905E10F0905F10009150
:1081900060101091611020915A1030915B10409145
:1081A0005C1050915D106091561070915710809145
:1081B000581090915910B6E08B2EBDE09B2E9F92E7
:1081C0008F92812C912CE6E1AE2EE3E4BE2EF2E6F6
:1081D000CF2EF0E1DF2E0F942D270F94CB8E0F9032
:1081E0000F900F900F90BEACBB2059F0332049F098
:1081F00020E030E040E85FE3C301B2010F94F9C131
:1082000004C060E070E080E291EC2B964FAD2B97BC
:108210000F944B10811103C089E496E47EC0209135
:108220005E1030915F1040916010509161106A961D
:108230006CAD7DAD8EAD9FAD6A970F94F9C12DECFD
:108240003CEC4CEC5DE30F9493BC87FF6DC020E0E9
:1082500030E040EA50E420935E1030935F1040938A
:1082600060105093611020915A1030915B10409132
:108270005C1050915D106091561070915710809174
:10828000581090915910A6E0BDE0BF93AF93812C98
:10829000912CB0EAAB2EB1E4BB2E12E6C12E10E158
:1082A000D12EE12CF12C00EA10E40F942D270F942D
:1082B000CB8E0F900F90FEADFF2359F0332049F085
:1082C00020E030E040E85FE3C301B2010F94F9C160
:1082D00004C060E070E080E291EC2B964FAD2B97EC
:1082E0000F944B10882309F497CF20915E103091A2
:1082F0005F10409160105091611060E070E080EA82
:1083000090E40F94F9C12DEC3CEC4CEC5DE30F9440
:1083100093BC87FF09C087EE90E19F938F930F94E2
:108320009EBB0F900F906EC08EAC8820C1F0209144
:108330005E1030915F104091601050916110C30148
:10834000B2010F94F9C19F7720E030E040E85FE38D
:108350000F9445C418161CF486EB90E1DECFC09054
:108360009219D0909319E0909419F09095198091FA
:1083700017078823A9F00F94EC67882389F0C701B9
:10838000B6010E94E9B12091A6103091A71040914A
:10839000A8105091A9100F94E8C29B01AC0103C032
:1083A00020E030E0A901F7E09F2E2796AFAC279799
:1083B0009A9C80011124020D111D000F111F000F46
:1083C000111F04571A4E60915E1070915F108091DA
:1083D0006010909161100F94F9C1D80111966D93BE
:1083E0007D938D939C9314978091FE0E9091FF0E38
:1083F00001979093FF0E8093FE0E339481E00E94CC
:1084000066F0C8CD80E090E0A0EAB0E480935E1012
:1084100090935F10A0936010B093611020915A1058
:1084200030915B1040915C1050915D10609156103E
:10843000709157108091581090915910E6E0FDE02E
:10844000FF93EF93812C912CA0EAAA2EA1E4BA2EDF
:10845000B2E6CB2EB0E1DB2EE12CF12C00EA10E4E9
:108460000F942D270F94CB8E0F900F906096EEAD4A
:10847000FFAD609764968EAC9FAC6497E815F905E4
:1084800009F4AAC085E090E00E94B8E9F6E06F2EFA
:10849000FDE07F2E1701280183EA93E10E94A8D313
:1084A0008EE190E00F94FFA90F9454649090520FC6
:1084B0009AAE1092520F1092510F20E030E040E837
:1084C0005FE360915E1070915F10809160109091F9
:1084D00061100F94F9C17B018C0160935E10709361
:1084E0005F10809360109093611020915A1030912A
:1084F0005B1040915C1050915D106091561070912E
:10850000571080915810909159107F926F92812C42
:10851000912CF0EAAF2EF1E4BF2EA2E6CA2EA0E124
:10852000DA2E0F942D270F94CB8EAA24A394A09219
:10853000520F1092510F84E00E9484C020925E106E
:1085400030925F10409260105092611020915A104A
:1085500030915B1040915C1050915D10609156100D
:108560007091571080915810909159107F926F928E
:10857000812C912CB0EAAB2EB1E4BB2EE12CF12C76
:1085800000EA10E40F942D270F94CB8E0E94EDBFCC
:10859000BAACB092520F1092510F82E00F94B88E85
:1085A0000F900F900F900F90A80197010F9445C462
:1085B00018160CF471CF1092DB0D1092DA0D81E0D9
:1085C0000E9442F841E061E081E00F94CF7481E0C5
:1085D00080937E130C94C370A4968EAD9FADA49728
:1085E0000F94FA630E94E8EA6091040D7091050D02
:1085F000072E000C880B990B0F9499BC9058209172
:10860000A6103091A7104091A8105091A9100F9476
:10861000E8C20E94F9EA80EC9FE00F946EC12B96AD
:108620008FAF2B979E012F5F3F4F28963FAF2EAF06
:108630002897712C80908C0290908D02A0908E02D1
:10864000B0908F0262968CAE9DAEAEAEBFAE62971A
:1086500024962EAD3FAD24972150310924963FAF8B
:108660002EAF24974901092C000CAA08BB082296BA
:108670008CAE9DAEAEAEBFAE229762968CAC9DAC7A
:10868000AEACBFAC629789829A82AB82BC822896DC
:10869000AEADBFAD28978D912896BFAFAEAF2897EE
:1086A0000F94CEB4882329F00F94BCB46B017C01E5
:1086B00020C02B96BFAD2B97B13009F092C1E1E0FD
:1086C000E71528F0772049F08EEB9FE00BC0F2E031
:1086D0007F1631F08CEB9FE005C08FEB9FE002C06E
:1086E0008DEB9FE00F946EC1C82E880FDD08EE0859
:1086F000FF08C114D104E104F10409F472C1D701E7
:10870000C601F7FE07C088279927DC018C199D094F
:10871000AE09BF0985369105A105B1050CF42FC03E
:10872000E3E1FFE584918F01882339F00F946F55C1
:108730000F5F1F4FF8018491F7CFE2E9F0E18491D8
:108740008F01882339F00F946F550F5F1F4FF80189
:108750008491F7CFC701B6010F94596BE9E8F0E1B6
:1087600084918F01882339F00F946F550F5F1F4F4D
:10877000F8018491F7CF8AE00F946F5532C1C70199
:10878000B6010F9499BC2FE632E143E85AE30F9407
:1087900000B66B017C01F2E07F1609F496C0E3E0BD
:1087A0008E2E781409F4D9C099249394791409F47D
:1087B0004BC0912CAAACA91409F413C1812C27E059
:1087C000299D50011124882D90E024964EAD5FAD77
:1087D000249784179507B4F58501080F191F000F1A
:1087E000111F000F111F04571A4EBA01681B790B95
:1087F000072E000C880B990B0F9499BCA7019601CA
:108800000F9400B61B012C0122966CAD7DAD8EAD90
:108810009FAD22970F9499BC9B01AC01C201B1019D
:108820000F94E8C2D80111962D913D914D915C9124
:1088300014970F94FAC1F801618372838383948340
:108840008394C1CF9394B6CF61E9A62E65E1B62E8D
:10885000612CFAADF61509F4C4C0450100E010E042
:108860000F5F1F4F2AAD021758F5B801012E000CFB
:10887000880B990B0F9499BCA70196010F9400B631
:108880001B012C0122966CAD7DAD8EAD9FAD229764
:108890000F9499BC9B01AC01C201B1010F94E8C2D5
:1088A0009B01AC01D4016D917D918D919C910F94B0
:1088B000FAC1F40161937193819391934F01D0CFE9
:1088C0006394FCE1AF0EB11CC4CF5CE8852E55E18A
:1088D000952E612CAAACA61409F483C024960EAD83
:1088E0001FAD249754010F3F2FEF120789F1B801F4
:1088F000012E000C880B990B0F9499BCA7019601CF
:108900000F9400B61B012C0122966CAD7DAD8EAD8F
:108910009FAD22970F9499BC9B01AC01C201B1019C
:108920000F94E8C29B01AC01D50111966D917D9128
:108930008D919C9114970F94FAC1F5016183728314
:1089400083839483FCE1AF0EB11C01501109CBCF9E
:10895000639424E0820E911CBDCF4CE8842E45E147
:10896000942E612C3AAD3615E1F18401A12CB12C85
:108970004FEFA41AB40A045E1F4F5AADA51660F556
:10898000B5010B2C000C880B990B0F9499BCA70117
:1089900096010F9400B61B012C0122966CAD7DADA3
:1089A0008EAD9FAD22970F9499BC9B01AC01C20183
:1089B000B1010F94E8C29B01AC01D80111966D91F1
:1089C0007D918D919C9114970F94FAC1F801618368
:1089D000728383839483CCCF6394F4E08F0E911CD5
:1089E000C1CF739434E0832E781047CE2AAD233064
:1089F00019F40F942C7C9CC03AAD373009F098C024
:108A00006B964FAD6B97442309F492C021E7C22EB9
:108A100025E1D22E00E07601712C55245394500E9E
:108A200044244A94400E47E0672D802F0F94E3B40E
:108A300066246394670C81116DC047E0662D802F1A
:108A40000F94E3B4882381F020E030E0A901D7013E
:108A5000D8966D917D918D919C91DB970F94FAC181
:108A60004B015C0111E004C0812C912C540110E0F9
:108A700047E06FEF670D802F0F94E3B4882361F018
:108A8000F7012081318142815381C501B4010F94E6
:108A9000FAC14B015C011F5F47E0672D852D0F94E4
:108AA000E3B4882371F0D70190962D913D914D91BB
:108AB0005C919397C501B4010F94FAC14B015C011D
:108AC0001F5F47E0672D842D0F94E3B4882369F07E
:108AD000F701208D318D428D538DC501B4010F9466
:108AE000FAC14B015C011F5F02C0112399F0612F95
:108AF00070E080E090E00F9499BC9B01AC01C5014F
:108B0000B4010F94E8C2D7015C966D937D938D9369
:108B10009C935F97762CBCE1EB0EF11CE7E06E12A4
:108B200082CF0F5FF4E0CF0ED11C073009F073CF76
:108B300081E080938C150E9494EBE091060D24E077
:108B4000E29FF0011124EB5FF04F20E030E04FE2B4
:108B500053E460817181828193810F9445C418161A
:108B600084F480911707882361F00F94EC678823C1
:108B700041F080910A0D90910B0DC29714F00C9466
:108B8000197181E090E0909329028093280286E396
:108B900095E10F944C0B6E964EAD5FAD6E97509372
:108BA000DB0D4093DA0DA0968EAD9FADA09790930C
:108BB000FF0E8093FE0E1092F30D34C180918C1540
:108BC000882309F495C0EFE7F0E184918F018823B1
:108BD00039F00F946F550F5F1F4FF8018491F7CF55
:108BE00067E070E080E090E00F94596BEDE7F0E112
:108BF00084918F01882339F00F946F550F5F1F4FB9
:108C0000F8018491F7CF67E070E080E090E00F9486
:108C1000596BEAE6F0E184918F01882339F00F94D3
:108C20006F550F5F1F4FF8018491F7CF65E070E03B
:108C300080E090E00F94596BE8E5F0E184918F01BA
:108C4000882339F00F946F550F5F1F4FF8018491FF
:108C5000F7CF8AE00F946F5500E010E085E5682EAD
:108C600080E1782E93E5A92E90E1B92EE12CF12C2C
:108C70004801F8EA8F0E911CF3018491B5E5CB2EE3
:108C8000B0E1DB2E882341F00F946F55FFEFCF1A30
:108C9000DF0AF6018491F6CFF701E80DF91DE457DC
:108CA000FA4E618172818381948145E00F94F4557D
:108CB000F4E0EF0EF11C2CE1E216F104E9F6F50107
:108CC0008491A3E5EA2EA0E1FA2E882341F00F94C7
:108CD0006F55FFEFEF1AFF0AF7018491F6CF0C51A1
:108CE00011090C33FFEF1F0709F0C0CF0C94C370BC
:108CF000E5E3F0E184918F01882311F40C94556F22
:108D00000F946F550F5F1F4FF8018491F5CF86EEDA
:108D10000F94F6670C94C3701092830F0C94C37079
:108D200085E40F94CEB4811102C00F94CB8E7AE00B
:108D3000672E73E0772EE6E5AE2EE0E1BE2EF2EF71
:108D40008F2EF0E19F2ED12CD3018D913D010F94F8
:108D5000CEB48823C9F1B3E0DB120CC00F94C6B4C3
:108D6000F501608371838283938382E690E10E94A0
:108D70006AEA2AC00F94C6B49B01AC01D4016D917C
:108D80007D918D919C910F94FAC1F501608371835F
:108D900082839383E0905E10F0905F1000916010EA
:108DA0001091611020915A1030915B1040915C102D
:108DB00050915D106091561070915710809158102D
:108DC000909159100F94B677D394F4E0AF0EB11C84
:108DD00024E0820E911C34E0D312B6CF0C94C37001
:108DE00081E080933F0F0F94A45960937A1670939B
:108DF0007B1680937C1690937D1660913F0F84ECD8
:108E00009FE00F9480C161E377E081EC9FE00F94D5
:108E1000A2401092DC0D60E08FEF9FE00F9480C1C4
:108E20000C94C37082E00E9466F00C94C370809131
:108E30006E1590916F158C579C4E9F938F9380E287
:108E400090E10C94C0358DE40F94CEB4882311F4D6
:108E50000C94116EE091100DF091110D31968191ED
:108E60008032E9F38930D9F380538A3060F0809101
:108E70006E1590916F158C579C4E9F938F938BE03E
:108E800090E10C94C0350F94C6B40F9459C3AB0154
:108E9000BC01CA015093400D40933F0D4937510525
:108EA00011F40C9406560CF0DEC04F32510509F453
:108EB00092C70CF061C04931510509F461C33CF51A
:108EC0004431510509F4C3C294F44131510509F408
:108ED000B4C234F44230510508F4FCC10C94FA6D6C
:108EE0004231510511F40C94FB520C94FA6D463149
:108EF000510509F4F0C20CF4EAC24731510509F4F6
:108F0000F0C24831510509F404C30C94FA6D4E3196
:108F1000510509F46BC48CF44B31510509F44BC372
:108F20000CF43BC34C31510509F434C44D315105A7
:108F300011F40C940C6E0C94FA6D4A32510509F43C
:108F40001CC654F44F31510509F4BCC540325105DB
:108F500009F41DC50C94FA6D4C32510509F42CC767
:108F60004D32510511F00C94FA6D8AE50F94CEB490
:108F70000E9409760C940C6E4936510511F40C943C
:108F8000C54FA4F54435510511F40C94FB52DCF4A3
:108F90004135510511F40C94DD5234F44934510536
:108FA00009F461C70C94FA6D4235510511F40C9423
:108FB000F7524335510511F00C94FA6D81E080931E
:108FC000440D0C940C6E4635510511F40C945D5310
:108FD00014F40C9442534C35510511F40C947C5309
:108FE0004836510509F49CC70C94FA6D4037510579
:108FF00009F4B5C7A4F44B36510511F40C94D752BB
:1090000014F40C94A7524D36510511F40C94E4500D
:109010004E36510511F40C9400540C94FA6D4337FC
:10902000510511F40C94505484F44137510511F456
:109030000C9413544237510511F00C94FA6DE7E685
:10904000FDE084918F010C9429554737510511F4A7
:109050000C940B564837510511F00C94FA6D109290
:1090600027020C940C6E8E3541E0940711F40C9499
:10907000406D0CF081C0803D910511F40C9479593C
:10908000DCF58B3C910511F40C94D9570CF58E3B13
:10909000910511F40C947E5134F48C38910509F447
:1090A00063C70C94FA6D883C910511F40C94285711
:1090B000893C910511F00C94FA6D4AE0C42E43E00E
:1090C000D42E5AE9E52E50E1F52E10E00C94945779
:1090D0008D3C910511F40C94775814F40C9432588B
:1090E0008E3C910511F40C9426598F3C910511F496
:1090F0000C9442590C94FA6D803F910511F40C9434
:109100000C6ECCF48C3D910511F40C94F6593CF4A2
:10911000813D910511F40C94A1590C94FA6D8D3D8B
:10912000910511F40C94215A823E910511F40C948E
:10913000425A0C94FA6D8E32A1E09A0711F40C9405
:109140002E5C6CF48C32E1E09E0711F40C94A45A6E
:109150008D32914011F40C94DA5A0C94FA6D8F32DE
:1091600021E0920711F40C94435C8033914011F498
:109170000C94965B0C94FA6D8A3542E0940711F4D6
:109180000C94CD680CF049C0853FA1E09A0711F41A
:109190000C947660ECF48039E1E09E0711F40C94B5
:1091A0002E603CF48F35914011F40C940C6E0C94AD
:1091B000FA6D833931E0930711F40C943260843FE7
:1091C000914011F00C94FA6D0F9462580C940C6E4F
:1091D0008D3F51E0950711F40C9436636CF4863F93
:1091E000B1E09B0711F40C947A60873F914011F431
:1091F0000C947E600C94FA6D8835F2E09F0711F4B0
:109200000C9411648935924011F00C94FA6D0F940E
:10921000461B0F943C950C940C6E8D3533E09307F0
:1092200011F40C94A169DCF48E3B52E0950711F423
:109230000C94E96D3CF48D3B924011F40C94DD6D7F
:109240000C94FA6D8335E3E09E0711F40C9452639D
:109250008C35934011F40C94D0680C94FA6D8C38D2
:1092600023E0920711F40C940C6E94F4843843E0DC
:10927000940711F40C94BD6B8B38934011F00C944F
:10928000FA6D1AE0A12E13E0B12E00E00C94206DCF
:10929000803AA3E09A0709F4E6C3873E934011F0B1
:1092A0000C94FA6D1092BC0F10921E0F80918C0FCF
:1092B00090918D0FA0918E0FB0918F0F8093120D12
:1092C0009093130DA093140DB093150D0F949E4A17
:1092D0000C940C6EE091100DF091110D8F010E5F4A
:1092E0001F4F80E50F94CEB4882371F00F94C6B45D
:1092F0000F945FC36B017C01AA24A394672B682B96
:10930000692B31F4A12C04C0A12CC12CD12C7601E5
:1093100083E50F94CEB4882391F00F94C6B420E077
:1093200030E04AE754E40F9400B60F945FC36B013A
:109330007C01BB24B394672B682B692B09F4B12CF7
:109340006AE270E0C8010F9442C7009711F0FC0177
:109350001082F801CF0121912032E1F3A11007C062
:10936000B11005C0222319F00F94CE0C04C082E97D
:1093700093E10F944C0B81E08093E10D1092E00D8E
:109380000F94CB8E0F94A4596093880F7093890F1C
:1093900080938A0F90938B0FC114D104E104F104E0
:1093A00019F10F94A459C60ED71EE81EF91E84E0C9
:1093B00090E090932902809328020F94A4596C1591
:1093C0007D058E059F0510F00C945B710E943AF1AB
:1093D00081110C945B710F94FF8781E00F943946E3
:1093E00080E00E9466F0E9CF84E090E0909329024B
:1093F000809328020E943AF1811109C00F94FF87DF
:1094000081E00F94394680E00E9466F0F3CF82E05D
:1094100090E09093290280932802809180168823FF
:1094200031F083E79AE30F944C0B0C940C6E86E3B7
:1094300095E10F944C0B0C940C6E89E893E10F941A
:109440004C0B17981698159814980C940C6EE3EC26
:10945000F6E084918F01882339F00F946F550F5FE8
:109460001F4FF8018491F7CF8AE00F946F55109247
:1094700061191092601984ED96E10F948D1F8BE1B4
:10948000E4EDF6E1DE01119601900D928A95E1F787
:1094900040E050E0BE016F5F7F4F84E194E00F94A5
:1094A000C085CE0101960F941966E5EBF6E0849134
:1094B0008F01882339F00F946F550F5F1F4FF8010C
:1094C0008491F7CF8AE00F946F550C940C6E0F9433
:1094D000F2160C940C6E10928016109281160C9459
:1094E0000C6E8091100D9091110D6AE270E004965F
:1094F0000F9442C7009711F0DC011C928091100D6F
:109500009091110D41E061E004960F941F120C94AC
:109510000C6E8091821681111EC060E086E69FE08D
:109520000F9480C160E088E69FE00F9480C160E006
:1095300085E69FE00F9480C160E084E69FE00F9491
:1095400080C160E082ED9EE00F9480C160E08FEC0E
:109550009EE00F9480C180918116882329F081E0DC
:1095600080938016109282160F94A4596093EA0D8E
:109570007093EB0D8093EC0D9093ED0D0C940C6EAD
:1095800080918016882311F40C940C6E1092801632
:1095900081E0809382160C940C6E80918116882352
:1095A00011F40C940C6E83E50F94CEB481110C94DD
:1095B00067710C940C6E80918016882309F4B8C0F2
:1095C0000CE916E1F80181918F01882319F00F94BD
:1095D0006F55F8CFE4EEFDE084918F01882339F0D8
:1095E0000F946F550F5F1F4FF8018491F7CFE7E994
:1095F000F5E084918F01882339F00F946F550F5F48
:109600001F4FF8018491F7CF60915B1970915C193D
:1096100080915D1990915E194AE00F948355E2EEB6
:10962000FDE084918F01882339F00F946F550F5F0F
:109630001F4FF8018491F7CF60915319709154191D
:1096400080915519909156194AE00F9483558AE0FC
:109650000F946F550F94A45950E6C52E5AEED52E8F
:10966000E12CF12CA70196010F94BEC149015A01CA
:109670006091EA0D7091EB0D8091EC0D9091ED0DE4
:10968000A70196010F94BEC18401021B130BC801F0
:109690006CE370E00F94A4C6CB019927EAE0F0E0F8
:1096A000BF010F94B8C6282FCB01BF010F94B8C6D5
:1096B000805D8093C219205D2093C3191092C41954
:1096C00062ECE62E69E1F62E6701D6018D916D01FF
:1096D000882319F00F946F55F8CF8AE30F946F55D4
:1096E000C8016CE370E00F94A4C66AE070E00F94C8
:1096F000B8C6605D6093C219805D8093C3191092F3
:10970000C419F70181917F01882319F00F946F55D7
:10971000F8CFE0EEFDE084918F01882311F40C94E2
:109720000C6E0F946F550F5F1F4FF8018491F5CFAA
:1097300080918216882371F0E0EDFDE084918F0125
:10974000882309F4BFCE0F946F550F5F1F4FF801A8
:109750008491F6CF8091F50D882371F0E4ECFDE063
:1097600084918F01882309F4ADCE0F946F550F5F5C
:109770001F4FF8018491F6CFE4EBFDE084918F0157
:10978000882309F49FCE0F946F550F5F1F4FF80188
:109790008491F6CF8091100D9091110D6AE270E0E6
:1097A00004960F9442C78C01892BA9F080916E1505
:1097B00090916F156EE470E08C579C4E0F9442C7E9
:1097C00060E270E00F9442C701969093110D809370
:1097D000100DD8011C928091100D9091110D41E057
:1097E00060E004960F941F120C940C6E8091811609
:1097F000882311F40C940C6E0F947B818091100DD2
:109800009091110D6AE270E004960F9442C78C01AA
:10981000892BA9F080916E1590916F156EE470E020
:109820008C579C4E0F9442C760E270E00F9442C781
:1098300001969093110D8093100DF8011082C09045
:10984000100DD090110D86010C5F1F4F8091811675
:10985000882311F40C940C6E86EA98E10F94B322DD
:10986000109280161F8E1AA284ED96E19093F01646
:109870008093EF160115110591F0D60114968C9185
:109880008F3239F4BE01615E7F4FC8010F94277794
:1098900006C081EF96E19093F0168093EF166091E9
:1098A000EF167091F01619821C8222E0A801CE01F9
:1098B00001960F947A248823A1F0CE0101960F948B
:1098C0002E85882371F061E0CE0101960F94342239
:1098D000009739F025EEFC0120831C820F94B81C00
:1098E000F82ECE0101960F941966FF2021F1E6EAC9
:1098F000FDE084917F01882341F00F946F55FFEFC5
:10990000EF1AFF0AF7018491F6CFD8018D918D01EE
:10991000882319F00F946F55F8CF8AE00F946F5594
:1099200010925B1910925C1910925D1910925E19D9
:109930000F94E01426C0EEE8FDE084917F018823B7
:1099400041F00F946F55BFEFEB1AFB0AF7018491BA
:10995000F6CFD8018D918D01882319F00F946F55A2
:10996000F8CFECE8FDE084918F01882339F00F9463
:109970006F550F5F1F4FF8018491F7CF8AE00F9466
:109980006F55CE014F960F9419660C940C6E809112
:10999000801681110F94CB8E0091100D1091110D36
:1099A0000C5F1F4F6AE270E0C8010F9442C77C0150
:1099B00061E270E0C8010F9442C7009719F08C0172
:1099C0000F5F1F4FE114F10411F0D7011C9280E5E5
:1099D0000F94CEB4F82E8091100D9091110D0817B0
:1099E000190708F4F12C80918116882311F40C9446
:1099F0000C6E41E04F2561E0C8010F941F1283E512
:109A00000F94CEB48823B9F08091100D9091110D70
:109A10008017910780F40F94BCB4AB01BC01409354
:109A20005B1950935C1960935D1970935E1986EA17
:109A300098E10F94F71E80918116882329F081E028
:109A40008093801610928216F1100C940C6E0F9475
:109A5000A4596093EA0D7093EB0D8093EC0D9093F5
:109A6000ED0D0C940C6E8091100D9091110D6AE229
:109A700070E005960F9442C78C01892BA9F0809164
:109A80006E1590916F156EE470E08C579C4E0F949C
:109A900042C760E270E00F9442C701969093110DA7
:109AA0008093100DF80110828091100D9091110D8E
:109AB00021E020937F1641E060E005960F941F128D
:109AC0000C940C6E0F94A4590091EA0D1091EB0DBB
:109AD0002091EC0D3091ED0D6B017C01C01AD10A83
:109AE000E20AF30AC701B60128EE33E040E050E095
:109AF0000F94BEC1CA01B9012CE330E040E050E050
:109B00000F94BEC17F936F93C701B60120E63AEE72
:109B100040E050E00F94BEC13F932F938CEF9FE045
:109B20009F938F938E010F5F1F4F1F930F930F947F
:109B3000F7BBE5E3FFE584910FB6F894DEBF0FBEF7
:109B4000CDBF7F01882341F00F946F553FEFE31A9B
:109B5000F30AF7018491F6CF7801D7018D917D0149
:109B6000882319F00F946F55F8CF8AE00F946F5542
:109B7000C8010F94CE0C0C940C6E83E50F94CEB4F8
:109B8000882311F40C940C6E0F94C6B40F9459C32F
:109B90004B015C017B0180E50F94CEB4882339F042
:109BA000BFEF8B16910409F010F40C9478710DE05E
:109BB00010E0E0E9F2E0819191918017910711F4B2
:109BC0000C940C6E22E0E83CF207A9F70630110570
:109BD00029F49092CB198092CA1904C017FF02C0D1
:109BE0000C940C6ED02E61E0802F0F94FF06682D30
:109BF000802F0F94D10661E0802F0F94FF06E114AF
:109C0000F10431F460E0802F0F94D1060C940C6EB7
:109C10003FEFE316F10431F461E0802F0F94D10699
:109C20000C940C6EF801FF27EA5BF14BE4918E2F48
:109C300090E0FC013197E231F10508F0ADC08827D2
:109C4000EE58FF4F8F4F0D94E7C684B5806884BDF2
:109C500087BC0C940C6E84B5806284BD88BC0C9467
:109C60000C6E8091800080688093800090928900C3
:109C7000809288000C940C6E8091800080628093AA
:109C8000800090928B0080928A000C940C6E8091E0
:109C9000800088608093800090928D0080928C007C
:109CA0000C940C6E8091B00080688093B00080921C
:109CB000B3000C940C6E8091B00080628093B00071
:109CC0008092B4000C940C6E809190008068809318
:109CD000900090929900809298000C940C6E809164
:109CE000900080628093900090929B0080929A00F6
:109CF0000C940C6E809190008860809390009092FC
:109D00009D0080929C000C940C6E8091A000806855
:109D10008093A0008091A0008F7B8093A000909200
:109D2000A9008092A8000C940C6E8091A000806223
:109D30008093A0009092AB008092AA000C940C6ECD
:109D40008091A00088608093A0009092AD008092E6
:109D5000AC000C940C6E80912001806880932001EF
:109D600090922901809228010C940C6E8091200120
:109D700080628093200190922B0180922A010C94A2
:109D80000C6E8091200188608093200190922D01BB
:109D900080922C010C940C6E40E8E416F10434F42B
:109DA00060E08D2D0F94D1060C940C6E61E08D2D2A
:109DB0000F94D1060C940C6E8FEF0F94F66760E051
:109DC00070E088EF9FE00F949AC10E94ECED0E9432
:109DD000CEED0C940C6E84E090E090932902809379
:109DE00028020E9438F80E94848D0F94FF8781E03A
:109DF0000F94394660E080E00E9442F38DE79DE0D9
:109E00000E9469F261E080E00E9442F31E9903C063
:109E100087E79DE002C08AE79DE00E9469F262E068
:109E200080E00E9442F31D9903C081E79DE002C0DB
:109E300084E79DE00E9469F263E080E00E9442F3C3
:109E40001C9903C08BE69DE002C08EE69DE00E9457
:109E500069F20E943AF1882341F20E9438F80F9487
:109E60003C940C940C6E80E50F94CEB4882331F0B2
:109E70000F94C6B40F945FC360933D0282E50F94C4
:109E8000CEB4882341F00F94C6B40F945FC370938F
:109E900043026093420281E50F94CEB4882331F0EF
:109EA0000F94C6B40F945FC360933C0283E50F9494
:109EB000CEB4882341F00F94C6B40F945FC370935F
:109EC000410260934002809143028F93809142024D
:109ED0008F9380913D021F928F9381E796E09F932D
:109EE0008F9308E716E01F930F930F949EBB80910A
:109EF00041028F93809140028F9380913C021F9288
:109F00008F938AE696E09F938F931F930F930F94FE
:109F10009EBB0FB6F894DEBF0FBECDBF0C940C6E87
:109F2000BE016F5F7F4F88E690E00F94DDB2811134
:109F30000C940C6E83E50F94CEB4882311F40C942A
:109F40000C6E19810F94C6B411110C940C6E0F9401
:109F500059C37093801560937F150C940C6E63E069
:109F600089E696E00F94DA4583E50F94CEB4882312
:109F700011F40C940C6E0F94C6B40F9459C37093E3
:109F80000B0D60930A0D0C940C6EBE016F5F7F4F3A
:109F900089E690E00F94DDB281110C940C6EE6EF2F
:109FA000FFE084918F01882339F00F946F550F5F84
:109FB0001F4FF8018491F7CFE98124E0E29FF0017F
:109FC0001124EB5FF04F608171818281938141E0C8
:109FD0000F94F455E3EFFFE084918F01882339F06B
:109FE0000F946F550F5F1F4FF8018491F7CFE981F0
:109FF000F0E0EE0FFF1FE158FA4E60817181072EED
:10A00000000C880B990B0F9499BC41E00F94F45508
:10A01000EFEEFFE084918F01882339F00F946F55A4
:10A020000F5F1F4FF8018491F7CF60911007709177
:10A030001107809112079091130741E00F94F45596
:10A04000ECEEFFE084918F01882339F00F946F5577
:10A050000F5F1F4FF8018491F7CF60910A0D709147
:10A060000B0D072E000C880B990B0F9499BC41E047
:10A070000F94F455E9EEFFE084918F01882339F0C5
:10A080000F946F550F5F1F4FF8018491F7CF60E079
:10A0900070E0CB010F94596BE7EEFFE084918F01E4
:10A0A000882339F00F946F550F5F1F4FF80184918B
:10A0B000F7CF6091050F7091060F8091070F909177
:10A0C000080F41E00F94F455E4EEFFE084918F0116
:10A0D000882339F00F946F550F5F1F4FF80184915B
:10A0E000F7CF60917F1570918015072E000C880BBB
:10A0F000990B0F9499BC41E00F94F455E0EEFFE00A
:10A1000084918F01882339F00F946F550F5F1F4F93
:10A11000F8018491F7CFE981F0E0E654F04F6081D7
:10A1200070E080E090E00F94596BEBEDFFE08491DC
:10A130008F01882339F00F946F550F5F1F4FF8017F
:10A140008491F7CF6091B90F70E080E090E00F94B8
:10A15000596BE7EDFFE084918F01882339F00F946C
:10A160006F550F5F1F4FF8018491F7CF60919219DF
:10A1700070919319809194199091951941E00F94E1
:10A18000F455E3EDFFE084918F01882339F00F94BB
:10A190006F550F5F1F4FF8018491F7CF60918E19B3
:10A1A00070918F19809190199091911941E00F94BD
:10A1B000F4558AE00F946F5581E090E09093290266
:10A1C000809328020C94EF75BE016F5F7F4F8DE680
:10A1D00090E00F94DDB281110C940C6E82EE9CE243
:10A1E0000F944C0B81E090E090937E0D80937D0D59
:10A1F00080913F0F882329F060E081E090E00E9489
:10A20000C7CF83E50F94CEB4882379F019810F94DA
:10A21000C6B4111106C00F9459C370938015609392
:10A220007F1581E08093060212C082E50F94CEB4C0
:10A23000882369F019810F94C6B4111106C00F94D8
:10A2400059C37093801560937F15109206020F9486
:10A25000A4594B015C01F9800F2D10E0F801EE0FBD
:10A26000FF1FE158FA4E60817181072E000C880BA8
:10A27000990B0F9499BCF801EE0FFF1FEE0FFF1F13
:10A28000EB5FF04F11E020813181428153810F94C7
:10A2900045C418160CF010E01093900F81E090E088
:10A2A00090932902809328021092F40D4F2DC5013E
:10A2B000B4010F942A4984ED9CE20F944C0B82E088
:10A2C00090E0909329028093280290937E0D8093D2
:10A2D0007D0D80913F0F882329F060E082E090E0BF
:10A2E0000E94C7CF0F94A4596093880F7093890F71
:10A2F00080938A0F90938B0F0C940C6E88EC9CE2E9
:10A300000F944C0B83E090E090937E0D80937D0D35
:10A3100080913F0F882329F060E081E090E00E9467
:10A32000C7CF83E50F94CEB4882361F00F94C6B4F1
:10A330000F9459C370930B0D60930A0D81E08093C5
:10A3400006020FC082E50F94CEB4882351F00F941B
:10A35000C6B40F9459C370930B0D60930A0D1092FD
:10A3600006020F94A4594B015C011092F40D609108
:10A370000A0D70910B0D072E000C880B990B0F9492
:10A3800099BC11E0209110073091110740911207FC
:10A39000509113070F9445C418160CF010E0109359
:10A3A000900F81E090E0909329028093280200EDC5
:10A3B0001FE08CECE82E8FE0F82E98ECC92E9FE081
:10A3C000D92E8091900F60910A0D70910B0D88230A
:10A3D000B9F08091F40D811113C0072E000C880B89
:10A3E000990B0F9499BC209110073091110740915F
:10A3F0001207509113070F9445C41816BCF08BC078
:10A40000072E000C880B990B0F9499BC2091100714
:10A410003091110740911207509113070F9493BC8C
:10A4200087FF79C080910602811175C00F94A459ED
:10A43000DC01CB0188199909AA09BB09893E93401F
:10A44000A105B10508F45EC080913F0F811156C08F
:10A45000E091060D24E0E29FF0011124EB5FF04F44
:10A460004080518062807380F8018491B0EDAB2E02
:10A47000BFE0BB2E882341F00F946F55FFEFAF1A5A
:10A48000BF0AF5018491F6CF42E0C301B2010F94F7
:10A49000F455F7018491ACECAA2EAFE0BA2E8823D4
:10A4A00041F00F946F55FFEFAF1ABF0AF501849189
:10A4B000F6CF6091060D70E080E090E00F94596B4C
:10A4C000F6018491F8ECAF2EFFE0BF2E882341F017
:10A4D0000F946F55FFEFAF1ABF0AF5018491F6CFC5
:10A4E00060911007709111078091120790911307E6
:10A4F00041E00F94F4558AE00F946F550F94A459DE
:10A500004B015C010F94FF8780E00F94394680E097
:10A510000E9466F056CF8FEB9CE20F944C0B82E0CA
:10A5200090E0909329028093280284E090E0909339
:10A530007E0D80937D0D0F94A4596093880F7093C6
:10A54000890F80938A0F90938B0F0C940C6E83E588
:10A550000F94CEB4882319F10F94C6B420E030E0F4
:10A56000A9010F9493BC87FD0FC00F94C6B420E0DF
:10A5700030E04FE753E40F9445C4181644F00F94AD
:10A58000C6B40F9459C305C060E070E002C06FEF1D
:10A5900070E07093CB196093CA190C940C6E8FEF16
:10A5A00090E09093CB198093CA190C940C6E109282
:10A5B000CB191092CA190C940C6E0F94184F0F946B
:10A5C000CB8E149A0F94DE8E1092CB191092CA196A
:10A5D00068EE73E080E090E00F946C5985E194E0C0
:10A5E0000F944C0B80E00E9466F00C940C6E10925D
:10A5F000440D0C940C6E83E50F94CEB4882399F02F
:10A600000F94C6B420E030E04AE754E40F9400B65B
:10A610000F945FC3609380027093810280938202E3
:10A62000909383021DC088E50F94CEB481110C94E1
:10A630007F7189E50F94CEB481110C947F718AE506
:10A640000F94CEB481110C947F7185E40F94CEB435
:10A6500081110C947F710F94CB8E149A0F94DE8E1F
:10A660008FEF9FEF909343028093420290934102B9
:10A670008093400280933D0280933C021092450DEE
:10A680000C940C6E83E50F94CEB4882311F40C94D3
:10A690000C6E0F94C6B420E030E04AE754E40F9407
:10A6A00000B60F945FC36093840F7093850F8093FF
:10A6B000860F9093870F0C940C6E83E50F94CEB4A5
:10A6C000882311F40C940C6E0F94C6B420E030E093
:10A6D0004AE754E40F9400B60F945FC360937C0282
:10A6E00070937D0280937E0290937F0289E696E1CB
:10A6F0000F94271C0C940C6E2AE033E03BAF2AAF7A
:10A700000AE910E1E3E1CE2EEEE0DE2EF12CAAAD57
:10A71000BBAD8D91BBAFAAAF0F94CEB4882309F423
:10A7200063C0B3E0FB1259C00F94C6B42B013C01C7
:10A7300020E030E040EA51E40F9493BC87FF45C02D
:10A74000A3019201F80164817581868197810F943C
:10A75000E8C24B015C019B01AC016091EE1070916D
:10A76000EF108091F0109091F1100F9400B660936B
:10A77000EE107093EF108093F0109093F1102090F2
:10A78000500230905102A5019401D1011C966D91A7
:10A790007D918D919C911F970F9400B6F101648774
:10A7A000758786879787D6016D917D918D919C9154
:10A7B0000F9497BCA50194010F9400B60F945FC34A
:10A7C000F6016083718382839383D80114964D923E
:10A7D0005D926D927C92179707C00F94C6B4F801F2
:10A7E0006483758386839783F3940C5F1F4FF4E033
:10A7F000CF0ED11C74E0872EF81089CF0C940C6E0C
:10A800008EE40F94CEB4882311F40C940C6E0F9444
:10A81000BCB46093120D7093130D8093140D90933C
:10A82000150D0C940C6E83E50F94CEB4882379F04B
:10A830008091100D9091110D4AE050E060E070E0C1
:10A8400001960F9428B8609333020C940C6EE5E3E4
:10A85000FFE584918F01882339F00F946F550F5FC6
:10A860001F4FF8018491F7CFC0903302D12CE12C17
:10A87000F12CE1ECFFE084918F01882339F00F94F3
:10A880006F550F5F1F4FF8018491F7CF4AE0C70162
:10A89000B6010F9483558AE00F946F550C940C6E9B
:10A8A00086E50F94CEB4882379F0E5E4FEE5849143
:10A8B0008F01882311F40C94624A0F946F550F5F37
:10A8C0001F4FF8018491F5CF85E50F94CEB4382E53
:10A8D0008823D9F1E090100DF090110DFFEFEF1AE1
:10A8E000FF0AF092110DE092100D27016701460159
:10A8F000D6018D916D0190ED980F9A30C0F38E3294
:10A9000011F00C940C6E5D013501F50181915F0130
:10A9100090ED980F9A30C0F38E3211F00C940C6EBB
:10A92000CF018C01DC012C90019620ED220D2A3004
:10A93000C0F3822D0F94220B81110C949E71BDE205
:10A940002B120C940C6E0C949E71E3EAFFE0849140
:10A950008F01882339F00F946F550F5F1F4FF80157
:10A960008491F7CFE5E4FEE584918F01882339F0E7
:10A970000F946F550F5F1F4FF8018491F7CFE9E4F3
:10A98000FFE084918F01882339F00F946F550F5F9A
:10A990001F4FF8018491F7CFE5E4FFE084918F0128
:10A9A000882339F00F946F550F5F1F4FF801849182
:10A9B000F7CFE6E3FFE084918F01882339F00F940D
:10A9C0006F550F5F1F4FF8018491F7CFE9E2FFE069
:10A9D00084918F01882339F00F946F550F5F1F4FBB
:10A9E000F8018491F7CFE8E1FFE084918F0188239B
:10A9F00039F00F946F550F5F1F4FF8018491F7CF17
:10AA0000E6E1FFE084918F01882339F00F946F55C0
:10AA10000F5F1F4FF8018491F7CFEFE0FFE08491C3
:10AA20008F01882339F00F946F550F5F1F4FF80186
:10AA30008491F7CFEAEEFEE084918F01882311F430
:10AA40000C94624A0F946F550F5F1F4FF801849169
:10AA5000F5CF882339F00F946F550F5F1F4FF80122
:10AA60008491F7CF609156107091571080915810D3
:10AA70009091591042E00F94F455E3E6FDE0849183
:10AA80008F01882339F00F946F550F5F1F4FF80126
:10AA90008491F7CF60915A1070915B1080915C1097
:10AAA00090915D1042E00F94F455EFE5FDE0849144
:10AAB0008F01882339F00F946F550F5F1F4FF801F6
:10AAC0008491F7CF60915E1070915F10809160105B
:10AAD0009091611042E00F94F455EBE5FDE0849114
:10AAE0008F01882339F00F946F550F5F1F4FF801C6
:10AAF0008491F7CF6091621070916310809164101F
:10AB00009091651042E00F94F455ECE8F5E08491E3
:10AB10008F01882339F00F946F550F5F1F4FF80195
:10AB20008491F7CF80E00F94AA8E0F9499BC209166
:10AB30009E1030919F104091A0105091A1100F9441
:10AB4000E8C242E00F94F455E7E5FDE084918F01FF
:10AB5000882339F00F946F550F5F1F4FF8018491D0
:10AB6000F7CF81E00F94AA8E0F9499BC2091A21088
:10AB70003091A3104091A4105091A5100F94E8C2F9
:10AB800042E00F94F455E3E5FDE084918F018823C2
:10AB900039F00F946F550F5F1F4FF8018491F7CF75
:10ABA00082E00F94AA8E0F9499BC2091A610309148
:10ABB000A7104091A8105091A9100F94E8C242E04C
:10ABC0000F94F455EFE4FDE084918F01882339F070
:10ABD0000F946F550F5F1F4FF8018491F7CF83E0FB
:10ABE0000F94AA8E0F9499BC2091AA103091AB10AB
:10ABF0004091AC105091AD100F94E8C242E00F9418
:10AC0000F4558AE00F946F550C940C6E81E080939C
:10AC100027020C940C6EE0E5F6E084918F01882306
:10AC200039F00F946F550F5F1F4FF8018491F7CFE4
:10AC30008AE00F946F55E8E4F6E084918F01882351
:10AC400039F00F946F550F5F1F4FF8018491F7CFC4
:10AC50001E9B0DC0EEE3F6E084918F018823A1F0E6
:10AC60000F946F550F5F1F4FF8018491F7CFE9E301
:10AC7000F6E084918F01882339F00F946F550F5FB0
:10AC80001F4FF8018491F7CF8AE00F946F55E1E3ED
:10AC9000F6E084918F01882339F00F946F550F5F90
:10ACA0001F4FF8018491F7CF8091060182FF0DC0FC
:10ACB000EEE3F6E084918F018823A1F00F946F55A5
:10ACC0000F5F1F4FF8018491F7CFE9E3F6E084911D
:10ACD0008F01882339F00F946F550F5F1F4FF801D4
:10ACE0008491F7CF8AE00F946F55E9E2F6E0849102
:10ACF0008F01882339F00F946F550F5F1F4FF801B4
:10AD00008491F7CF1D9B0DC0EEE3F6E084918F0197
:10AD10008823A1F00F946F550F5F1F4FF8018491A6
:10AD2000F7CFE9E3F6E084918F01882339F00F949F
:10AD30006F550F5F1F4FF8018491F7CF8AE00F9492
:10AD40006F55E1E2F6E084918F01882339F00F948A
:10AD50006F550F5F1F4FF8018491F7CF8091060167
:10AD600087FF0DC0EEE3F6E084918F018823A1F008
:10AD70000F946F550F5F1F4FF8018491F7CFE9E3F0
:10AD8000F6E084918F01882339F00F946F550F5F9F
:10AD90001F4FF8018491F7CF8AE00F946F55E9E1D6
:10ADA000F6E084918F01882339F00F946F550F5F7F
:10ADB0001F4FF8018491F7CF1C9B0DC0EEE3F6E026
:10ADC00084918F018823A1F00F946F550F5F1F4F5F
:10ADD000F8018491F7CFE9E3F6E084918F018823AD
:10ADE00039F00F946F550F5F1F4FF8018491F7CF23
:10ADF0008AE00F946F55E1E1F6E084918F0188239A
:10AE000039F00F946F550F5F1F4FF8018491F7CF02
:10AE100001990FC0EEE3F6E084918F01882311F4CD
:10AE20000C94624A0F946F550F5F1F4FF801849185
:10AE3000F5CFE9E3F6E084918F01882311F40C94B7
:10AE4000624A0F946F550F5F1F4FF8018491F5CF41
:10AE50001091060D84E50F94CEB4882301F10F9470
:10AE6000C6B40F945FC3162F6623C9F0E5E3FFE570
:10AE700084918F01882339F00F946F550F5F1F4F16
:10AE8000F8018491F7CF0AEF15E0D8018D918D017B
:10AE9000882311F40C940C6E0F946F55F6CF84E454
:10AEA0000F94CEB4882311F40C940C6E0F94C6B496
:10AEB00020E030E0A9010F9493BC811103C01092EF
:10AEC00031112EC00F94C6B4B4E01B9FF0011124C1
:10AED000EE5CFE4E6083718382839383C090321157
:10AEE000D0903311E0903411F090351120E030E033
:10AEF000A901C701B6010F9493BC811106C0C12CF2
:10AF0000D12C60EEE62E6FE3F62EC0923211D09275
:10AF10003311E0923411F092351181E080933111B8
:10AF20000F94A8440C940C6EF60181916F010F945C
:10AF3000CEB4882399F10F94C6B40F945FC3123036
:10AF4000ACF4653CF9E07F0781059105A0F4562F2C
:10AF5000472F382F292F613CA3E07A0781059105FF
:10AF600090F050EC43E030E020E00DC0562F472F2A
:10AF7000382F292F08C050EC43E030E020E064EC8B
:10AF800079E080E090E0F70164A375A386A397A31E
:10AF9000E455FF4F50834183328323831F5FF4E0E6
:10AFA000EF0EF11C143009F0BFCF0E940CEA0C9494
:10AFB0000C6E2AE0A22E23E0B22E3AE9C32E30E135
:10AFC000D32E912CD5018D915D010F94CEB48823A1
:10AFD00009F43EC00F94C6B47B018C01B1E0B915F1
:10AFE00014F120E030E048E453E40F9445C418160F
:10AFF0003CF4512C612C88E4782E93E4892E04C013
:10B000005E2C6F2C702E812E20E030E048EC52E454
:10B01000B701C8010F9445C418164CF4E12CF12C6B
:10B0200008EC12E404C0562E6F2C782E812E852D4C
:10B03000962DA72DB82DF601848B958BA68BB78BFB
:10B04000C701D801E456FF4F80839183A283B38365
:10B050009394F4E0CF0ED11CB4E08B2E9810B2CFB5
:10B060000C940C6E83E50F94CEB48823E9F00F9412
:10B07000C6B46093CE107093CF108093D01090938D
:10B08000D11084E50F94CEB4882311F40C940C6E87
:10B090000F94C6B46093D2107093D3108093D410E1
:10B0A0009093D5100C940C6E80E50F94CEB4882349
:10B0B00051F00F94C6B46093CE107093CF1080936C
:10B0C000D0109093D11082E50F94CEB4882351F024
:10B0D0000F94C6B46093D2107093D3108093D410A1
:10B0E0009093D51084E50F94CEB40C940C6E83E548
:10B0F0000F94CEB4882351F00F94C6B46093D61049
:10B100007093D7108093D8109093D91084E50F9442
:10B11000CEB4882351F00F94C6B46093DA107093C4
:10B12000DB108093DC109093DD1082E40F94CEB49A
:10B13000882361F00F94C6B40F945FC36093DE1050
:10B140007093DF108093E0109093E11088E50F94E6
:10B15000CEB4882391F00F94C6B46093E610709338
:10B16000E7108093E8109093E9106093E2107093D9
:10B17000E3108093E4109093E51089E50F94CEB42A
:10B18000882351F00F94C6B46093E6107093E710D3
:10B190008093E8109093E9108AE50F94CEB4882349
:10B1A00051F00F94C6B46093EA107093EB10809343
:10B1B000EC109093ED1085E40F94CEB4882351F0F9
:10B1C0000F94C6B46093EE107093EF108093F0105C
:10B1D0009093F11020E030E040E251E46091E21001
:10B1E0007091E3108091E4109091E5100F9445C4A4
:10B1F000181664F480E090E0A0E2B1E48093E210DD
:10B200009093E310A093E410B093E51020E030E0B9
:10B2100040E251E46091E6107091E7108091E810EF
:10B220009091E9100F9445C4181614F00C940C6E0C
:10B2300080E090E0A0E2B1E48093E6109093E71004
:10B24000A093E810B093E9100C940C6EAAE0EA2EDB
:10B25000A3E0FA2E02EF10E1D7018D917D010F944A
:10B26000CEB4882339F00F94C6B4F801608371839B
:10B27000828393830C5F1F4FF0E10E3F1F0761F73E
:10B280000C940C6E83E50F94CEB4882351F00F9488
:10B29000C6B460931D1170931E1180931F1190937B
:10B2A000201186E40F94CEB4882381F00F94C6B4A5
:10B2B00020E030E040E752E40F94E8C260932111AF
:10B2C0007093221180932311909324118AE50F9497
:10B2D000CEB4882311F40C940C6E0F94C6B4609312
:10B2E00025117093261180932711909328110C94A7
:10B2F0000C6E83E50F94CEB4882351F00F94C6B43E
:10B300006093291170932A1180932B1190932C1123
:10B3100086E40F94CEB4882311F40C940C6E0F9431
:10B32000C6B420E030E040E752E40F94E8C26093F6
:10B330002D1170932E1180932F11909330110C9436
:10B340000C6E83E50F94CEB4882311F40C940C6E2C
:10B350000F94C6B40F9459C36115710551F0613053
:10B36000710569F481E080931C111092500F0C94C8
:10B370000C6E10921C111092500F0C940C6EE5E3A1
:10B38000FFE584918F01882339F00F946F550F5F8B
:10B390001F4FF8018491F7CFE7EEF5E084918F011C
:10B3A000882339F00F946F550F5F1F4FF801849178
:10B3B000F7CF00916E1510916F150C571C4ED801E8
:10B3C0008D918D01882319F00F946F55F8CFE5EE1C
:10B3D000FEE084918F01882311F40C94624A0F944B
:10B3E0006F550F5F1F4FF8018491F5CF82E40F94E2
:10B3F000CEB4882341F080914B0290914C029093FF
:10B4000005028093040283E50F94CEB4882341F0B3
:10B410000F94C6B40F9459C370934C0260934B02BF
:10B4200082E50F94CEB4882311F40C940C6E8091B5
:10B4300004029091050290934C0280934B020C946D
:10B440000C6E83E50F94CEB4882309F469CD0F9474
:10B45000C6B40F9459C36B017C0184E50F94CEB43C
:10B46000882359F0BE016F5F7F4F8DED90E00F9400
:10B47000DDB281110C940C6E53CDD0925B02C09260
:10B480005A024ECD80E50F94CEB4882311F40C946B
:10B490000C6E0F94C6B40F9459C3F62E862F972FB7
:10B4A0006C0183E50F94CEB4882331F00F94C6B4B9
:10B4B0000F9459C38B0102C00FEF1FEFC801019613
:10B4C000039710F00C940C6EE0E9F2E081919191F9
:10B4D000C816D90611F40C940C6E22E0E83CF20771
:10B4E000A9F7D7FE02C00C940C6E0F94CB8EEF2CF4
:10B4F00060E08F2D0F94FF060F3F3FEF130731F0F1
:10B500000130110571F401E010E00DC08F2D0F9492
:10B51000A90631E020E0892B09F030E0032F122F3B
:10B5200002C000E010E08E2D0F94A906801791074D
:10B5300011F40C940C6E0F94FF8780E00F94394641
:10B5400080E00E9466F0EFCF83E50F94CEB48823AD
:10B5500031F00F94C6B40F9459C38B0102C00EE6AC
:10B5600010E080E50F94CEB4882329F00F94C6B480
:10B570000F9459C302C068EE73E0072E000C880BCD
:10B58000990B1016110694F42091090730910A07BF
:10B590002230310528F42091020124602093020119
:10B5A0000F946C590F94A9800C940C6E0F946C59E5
:10B5B0000C940C6E80E50F94CEB4882351F00F9458
:10B5C000C6B4609302117093031180930411909399
:10B5D000051189E40F94CEB4882381F00F94C6B48A
:10B5E0002CEA35EC47E25EE30F9400B66093061157
:10B5F00070930711809308119093091184E40F94BC
:10B60000CEB4882381F00F94C6B42CEA35EC47E21F
:10B610005EE30F94E8C260930A1170930B1180935C
:10B620000C1190930D1183E40F94CEB4882351F044
:10B630000F94C6B4609300027093010280930202DB
:10B64000909303020F94D98DEAE5F8E184918F017C
:10B65000882339F00F946F550F5F1F4FF8018491C5
:10B66000F7CF02E214E0D8018D918D01882319F003
:10B670000F946F55F8CF6091021170910311809172
:10B6800004119091051142E00F94F45506E214E084
:10B69000F80181918F01882319F00F946F55F8CF2D
:10B6A0002CEA35EC47E25EE36091061170910711D8
:10B6B00080910811909109110F94E8C242E00F9413
:10B6C000F4550AE214E0D8018D918D01882319F018
:10B6D0000F946F55F8CF2CEA35EC47E25EE36091AA
:10B6E0000A1170910B1180910C1190910D110F9412
:10B6F00000B642E00F94F4550EE214E0F801819197
:10B700008F01882319F00F946F55F8CF60910002D4
:10B7100070910102809102029091030242E00F9425
:10B72000F4558AE00F946F550C940C6E80E50F94DD
:10B73000CEB4882351F00F94C6B460930E11709369
:10B740000F11809310119093111189E40F94CEB4CE
:10B75000882381F00F94C6B42CEA35EC47E25EE30F
:10B760000F9400B66093121170931311809314110B
:10B770009093151184E40F94CEB4882381F00F9434
:10B78000C6B42CEA35EC47E25EE30F94E8C260935E
:10B7900016117093171180931811909319110F942B
:10B7A000D98DEAE5F8E184918F01882339F00F946F
:10B7B0006F550F5F1F4FF8018491F7CF02E214E03D
:10B7C000D8018D918D01882319F00F946F55F8CF12
:10B7D00060910E1170910F118091101190911111C3
:10B7E00042E00F94F45506E214E0F80181918F01D4
:10B7F000882319F00F946F55F8CF2CEA35EC47E207
:10B800005EE3609112117091131180911411909167
:10B8100015110F94E8C242E00F94F4550AE214E0C7
:10B82000D8018D918D01882319F00F946F55F8CFB1
:10B830002CEA35EC47E25EE3609116117091171126
:10B8400080911811909119110F9400B642E00F9455
:10B85000F4558AE00F946F550C940C6E83E50F94A9
:10B86000CEB4882319F00F94C6B403C060E070E032
:10B87000CB0160935C0270935D0280935E029093B3
:10B880005F020C940C6E85E40F94CEB4882359F0BB
:10B890000F94C6B40F9459C324967FAF6EAF24970C
:10B8A00077FF05C013C024961FAE1EAE2497639683
:10B8B0001FAE639767961FAE679726E16B962FAF13
:10B8C0006B9733E46D963FAF6D970EC063961FAED6
:10B8D000639767961FAE67974CE86B964FAF6B9771
:10B8E00052E46D965FAF6D9783E50F94CEB48823D5
:10B8F00071F00F94C6B463966FAF639767967FAF8E
:10B9000067976B968FAF6B976D969FAF6D9783E43C
:10B910000F94CEB4882349F00F94C6B40F9459C342
:10B92000E3967FAF6EAFE39706C085E090E0E396C5
:10B930009FAF8EAFE397E3968EAC9FACE397909268
:10B940007A0D8092790D1092FD0E10927C0D10925E
:10B950007B0D0F94A45962966CAF7DAF8EAF9FAFF5
:10B9600062972496AEACBFAC2497B7FC05C02AE022
:10B97000E4962FAFE49704C03DE2E4963FAFE4972E
:10B980000F94A459C458DF4F688379838A839B83BB
:10B99000CC57D04024968EAC9FAC24971814190431
:10B9A000B4F402E314E0D8018D918D01882319F0DD
:10B9B0000F946F55F8CF8AE00F946F5581E0809314
:10B9C000FD0E10927C0D10927B0D0C940C6E0CE50C
:10B9D00014E0F80181918F01882319F00F946F55BD
:10B9E000F8CF8AE00F946F550F94184F24968EACC1
:10B9F0009FAC24978FE7892809F456C08093B90F2C
:10BA00008EEF0F94FA5962968CAC9DACAEACBFAC85
:10BA10006297A2968CAE9DAEAEAEBFAEA297EC96EC
:10BA20008CAE9DAEAEAEBFAEEC972B961FAE2B97F5
:10BA3000A3961FAEA39720E4A5962FAFA5973CE150
:10BA4000A6963FAFA69746E4AA964FAFAA97AE96A2
:10BA50001FAEAE97AF961FAEAF97E0961FAEE097C2
:10BA6000E1961FAEE197EFE78E2E912CA12CB12C21
:10BA70002A968CAE9DAEAEAEBFAE2A97FFE74F2E94
:10BA8000512C612C712CE8961CAE1DAE1EAE1FAE63
:10BA9000E89721E0CC57DF4F2883C458D0401AAE36
:10BAA0001EAE212C312C06C08093BA0FACCF80E0A3
:10BAB0000E9466F0A8958091BB0F882309F482C18B
:10BAC0000F949D5324968EAC9FAC2497892859F4EB
:10BAD0009090050F9AAEA090060FAEAE2090070F83
:10BAE0003090080F0AC0B0901007BAAE80901107CE
:10BAF0008EAE20901207309013072AAD3EADA10103
:10BB0000AE966FADAE97AF967FADAF97E0968FAD27
:10BB1000E097E1969FADE1970F9445C4181674F035
:10BB20009AACAE969FAEAE97AEACAF96AFAEAF97B7
:10BB3000E0962FAEE097E1963FAEE197A3962FAD4A
:10BB4000A397A5963FADA597A6964FADA697AA96A3
:10BB50005FADAA976AAD7EADC1010F9445C41816BA
:10BB600074F0BAACA396BFAEA3978EACA5968FAE79
:10BB7000A597A6962FAEA697AA963FAEAA970F9422
:10BB8000A459DC01CB01C458DF4F88809980AA807A
:10BB9000BB80CC57D04088199909AA09BB09853CBC
:10BBA0009940A105B10560F00F94E2870F94A45964
:10BBB000C458DF4F688379838A839B83CC57D040F6
:10BBC000CC57DF4F8880C458D040882009F477C014
:10BBD0002AAD3EADA10163966FAD639767967FADC9
:10BBE00067976B968FAD6B976D969FAD6D970F9422
:10BBF00093BC87FFE7C00F94A459DC01CB01629688
:10BC00008CAC9DACAEACBFAC629788199909AA09FF
:10BC1000BB0989389341A105B10508F4D3C0D3010C
:10BC2000C2012A968CAC9DACAEACBFAC2A978819E9
:10BC30009909AA09BB092496AEACBFAC2497B59567
:10BC4000A79597958795AB2831F08093B90F880F0A
:10BC50000F94FA5902C08093BA0F0F94A459A29678
:10BC60006CAF7DAF8EAF9FAFA2974B015C01629628
:10BC70002CAD3DAD4EAD5FAD6297821A930AA40A1A
:10BC8000B50AE8968CAE9DAEAEAEBFAEE8976396B1
:10BC90008FAC6397AE968FAEAE9767969FAC679763
:10BCA000AF969FAEAF976B96AFAC6B97E096AFAE8B
:10BCB000E0976D96BFAC6D97E196BFAEE1972AAD68
:10BCC0003EADA10163966FAD639767967FAD6797B1
:10BCD0006B968FAD6B976D969FAD6D970F9445C426
:10BCE000181614F00C948B740F94A459DC01CB013A
:10BCF000A2968CAC9DACAEACBFACA297881999094A
:10BD0000AA09BB0989389341A105B10510F40C9427
:10BD10008B740F94A45962966CAF7DAF8EAF9FAFBA
:10BD20006297DC01CB0188199909AA09BB09209106
:10BD30007B0D30917C0D1216130614F40C94B67220
:10BD40002A968CAD9DADAEADBFAD2A97840D951DE5
:10BD5000A61DB71D24968EAC9FAC2497B595A795CC
:10BD600097958795892811F40C9487748093B90F5F
:10BD7000880F0F94FA5980917B0D90917C0D01965C
:10BD800090937C0D80937B0D63969FAC6397A396F5
:10BD90009FAEA3976796AFAC6797A596AFAEA597F2
:10BDA0006B96BFAC6B97A696BFAEA6976D968FAC01
:10BDB0006D97AA968FAEAA9721E0CC57DF4F2883C4
:10BDC000C458D04020E030E040EA51E463966FADC3
:10BDD000639767967FAD67976B968FAD6B976D9600
:10BDE0009FAD6D970F94FAC12AAD3EADA1010F949E
:10BDF00093BC87FF0EC0EEEDFCE084918F01882399
:10BE000009F4D9CD0F946F550F5F1F4FF80184913E
:10BE1000F6CF0F94A459DC01CB01EC968CAC9DAC11
:10BE2000AEACBFACEC9788199909AA09BB09813D52
:10BE30009740A105B10508F4C4C024968EAC9FAC10
:10BE40002497892881F0E090B90FF12CEBEDFCE00C
:10BE500084918F018823B9F00F946F550F5F1F4FA6
:10BE6000F8018491F7CFE090BA0FF12CE8EDFCE0F7
:10BE700084918F01882339F00F946F550F5F1F4F06
:10BE8000F8018491F7CF42E06AAD7EADC1010F9415
:10BE9000F455E4EDFCE084918F01882339F00F9490
:10BEA0006F550F5F1F4FF8018491F7CFB701FF0C5B
:10BEB000880B990B0F94596B8AE00F946F552B9652
:10BEC0008FAC2B97882009F45AC0E4969FACE49776
:10BED000891418F4282D2F5F69C02B968FAC2B97EF
:10BEE000E4969FACE497891064C0282D2F5F2B96B1
:10BEF0002FAF2B97C058DF4F2881C058D040CF5765
:10BF0000DF4F3881C158D040CE57DF4F4881C258EB
:10BF1000D040CD57DF4F5881C358D0406AAD7EAD79
:10BF2000C1010F94F9C16B017C0120E030E0A9014F
:10BF30000F9445C418165CF420E030E040EA50E469
:10BF4000C701B6010F9493BC87FF33C00AC020E03D
:10BF500030E040EA50ECC701B6010F9445C4181612
:10BF600044F524966FAD2497661F6627661F80E010
:10BF70000F94884F81E08093FD0E0C940C6E8AAC78
:10BF8000C058DF4F8882C058D0409EACCF57DF4F9B
:10BF90009882C158D040CE57DF4F2882C258D04037
:10BFA000CD57DF4F3882C358D04021E02B962FAFBA
:10BFB0002B970F94A459EC966CAF7DAF8EAF9FAFCB
:10BFC000EC970F94A4596B017C010F94A459A2968D
:10BFD0000CAD1DAD2EAD3FADA29762968CAC9DAC65
:10BFE000AEACBFAC6297080D191D2A1D3B1DC01ACF
:10BFF000D10AE20AF30ADC01CB018C0D9D1DAE1DB6
:10C00000BF1D81389F44A241B10570F0E7EBFCE011
:10C0100084918F01882309F4CECC0F946F550F5F64
:10C020001F4FF8018491F6CF80917B0D90917C0D8C
:10C03000E3968EAC9FACE397881699060CF037CD4B
:10C04000EBE5FCE084918F01882309F4B4CC0F94D4
:10C050006F550F5F1F4FF8018491F6CF0F94CB8E71
:10C060000C940C6E80913710882311F40C940C6E94
:10C0700085E40F94CEB4882331F00F94C6B40F94A6
:10C080005FC3162F01C01FEF86E40F94CEB4882340
:10C0900031F00F94C6B40F945FC3062F01C00FEFA9
:10C0A0001F920F931F921F938AE49CE09F938F939C
:10C0B0000F949EBB1F920F931F921F9382E49CE0EC
:10C0C0009F938F930E949DEA0FB6F894DEBF0FBE38
:10C0D000CDBF1AE00E9447A1181614F40C940C6E00
:10C0E000115011F00C9492740C940C6E0F94EA564B
:10C0F0000C940C6E0F94B4560C940C6E8091FD1041
:10C100008F938091FC108F938091FB108F9380917F
:10C11000FA108F938091F9108F938091F8108F937C
:10C120008091F7108F938091F6108F938091F51086
:10C130008F938091F4108F938091F3108F9380915F
:10C14000F2108F9305E31FE51F930F931F930F9337
:10C150008091F1108F938091F0108F938091EF1068
:10C160008F938091EE108F938091ED108F9380913B
:10C17000EC108F938091EB108F938091EA108F9346
:10C180008091E9108F938091E8108F938091E71050
:10C190008F938091E6108F938091E5108F9380911B
:10C1A000E4108F938091E3108F938091E2108F932E
:10C1B0008091E1108F938091E0108F938091DF1038
:10C1C0008F938091DE108F938091DD108F938091FB
:10C1D000DC108F938091DB108F938091DA108F9316
:10C1E0008091D9108F938091D8108F938091D71020
:10C1F0008F938091D6108F931F930F931F930F935C
:10C200008091D5108F938091D4108F938091D3100B
:10C210008F938091D2108F938091D1108F938091C2
:10C22000D0108F938091CF108F938091CE108F93E9
:10C230001F930F931F930F93809155118F938091AC
:10C2400054118F93809153118F93809152118F933A
:10C25000809151118F93809150118F9380914F1144
:10C260008F9380914E118F9380914D118F93809178
:10C270004C118F9380914B118F9380914A118F9322
:10C28000809149118F93809148118F93809147112C
:10C290008F93809146118F931F930F931F930F934A
:10C2A0008091CD108F938091CC108F938091CB1083
:10C2B0008F938091CA108F938091C9108F93809132
:10C2C000C8108F938091C7108F938091C6108F9361
:10C2D0008091C5108F938091C4108F938091C3106B
:10C2E0008F938091C2108F938091C1108F93809112
:10C2F000C0108F938091BF108F938091BE108F9349
:10C300001F930F931F930F93809145118F938091EB
:10C3100044118F93809143118F93809142118F9399
:10C32000809141118F93809140118F9380913F11A3
:10C330008F9380913E118F9380913D118F938091C7
:10C340003C118F9380913B118F9380913A118F9381
:10C35000809139118F93809138118F93809137118B
:10C360008F93809136118F931F930F931F930F9389
:10C370008091BD108F938091BC108F938091BB10E2
:10C380008F938091BA108F938091B9108F93809181
:10C39000B8108F938091B7108F938091B6108F93C0
:10C3A0008091B5108F938091B4108F938091B310CA
:10C3B0008F938091B2108F938091B1108F93809161
:10C3C000B0108F938091AF108F938091AE108F93A8
:10C3D0001F930F931F930F938091AD108F938091B4
:10C3E000AC108F938091AB108F938091AA108F9394
:10C3F0008091A9108F938091A8108F938091A7109E
:10C400008F938091A6108F938091A5108F93809128
:10C41000A4108F938091A3108F938091A2108F937B
:10C420008091A1108F938091A0108F9380919F1085
:10C430008F9380919E108F931F930F931F930F9351
:10C4400082E999E09F938F930F949EBB0FB6F89467
:10C45000DEBF0FBECDBF2CEA35EC47E25EE3609154
:10C460000A1170910B1180910C1190910D110F9484
:10C4700000B69F938F937F936F932CEA35EC47E23E
:10C480005EE36091061170910711809108119091FF
:10C4900009110F94E8C29F938F937F936F938091BC
:10C4A00005118F93809104118F93809103118F93C5
:10C4B000809102118F931F930F931F930F9385E623
:10C4C00099E09F938F930F949EBB2CEA35EC47E243
:10C4D0005EE360911611709117118091181190917F
:10C4E00019110F9400B69F938F937F936F932CEA4B
:10C4F00035EC47E25EE36091121170911311809167
:10C500001411909115110F94E8C29F938F937F930C
:10C510006F93809111118F93809110118F9380915F
:10C520000F118F9380910E118F931F930F931F9371
:10C530000F9380E399E09F938F930F949EBB0FB668
:10C54000F894DEBF0FBECDBF80911C111F928F9358
:10C550001F930F931F930F9320E030E040E752E4C6
:10C5600060912D1170912E1180912F1190913011A9
:10C570000F9400B69F938F937F936F9380912C11AC
:10C580008F9380912B118F9380912A118F9380919B
:10C5900029118F931F930F931F930F93809128114D
:10C5A0008F93809127118F93809126118F93809183
:10C5B00025118F9320E030E040E752E46091211193
:10C5C0007091221180912311909124110F9400B643
:10C5D0009F938F937F936F93809120118F9380917E
:10C5E0001F118F9380911E118F9380911D118F9336
:10C5F0001F930F931F930F938FE298E09F938F9356
:10C600000F949EBB0FB6F894DEBF0FBECDBF8091D6
:10C6100031118823E9F0809135118F938091341185
:10C620008F93809133118F93809132118F931F9349
:10C630000F931F930F9389E098E09F938F930F942C
:10C640009EBB0FB6F894DEBF0FBECDBF0C940C6E30
:10C650001F930F938AEE97E09F938F930F949EBB47
:10C660000F900F900F900F900C940C6EE5E3FFE588
:10C6700084918F01882339F00F946F550F5F1F4FFE
:10C68000F8018491F7CFE5EDFEE084918F018823D6
:10C6900011F40C940C6E0F946F550F5F1F4FF8013F
:10C6A0008491F5CF8AE50F94CEB4882309F489C02C
:10C6B0000F94C6B46B017C0120E030E040E751EC00
:10C6C0000F9445C487FD38C020E030E040EA50ECCC
:10C6D000C701B6010F9493BC181674F1F7FAF094E1
:10C6E000F7F8F094C092FE10D092FF10E092001183
:10C6F000F0920111E5E3FFE584918F01882339F081
:10C700000F946F550F5F1F4FF8018491F7CFEEED37
:10C71000F5E084918F01882339F00F946F550F5FF6
:10C720001F4FF8018491F7CF8AE00F946F558AE08C
:10C730000F946F550C940C6EE5E3FFE584918F0127
:10C74000882339F00F946F550F5F1F4FF8018491C4
:10C75000F7CFEEEDF5E084918F01882339F00F9447
:10C760006F550F5F1F4FF8018491F7CFE9E1F6E0B5
:10C7700084918F01882339F00F946F550F5F1F4FFD
:10C78000F8018491F7CF61EF7FEF8FEF9FEF0F9468
:10C79000596BE1E1F6E084918F01882339F00F9421
:10C7A0006F550F5F1F4FF8018491F7CF6BEF7FEF4D
:10C7B0008FEF9FEF0F94596B8AE00F946F550C9495
:10C7C0000C6EE5E3FFE584918F01882339F00F9427
:10C7D0006F550F5F1F4FF8018491F7CFEEEDF5E035
:10C7E00084918F01882339F00F946F550F5F1F4F8D
:10C7F000F8018491F7CF8AE00F946F558091FE1075
:10C800009091FF10A0910011B0910111BC01CD01D8
:10C81000905842E00F94F4558AE00F946F550C94B1
:10C820000C6E0F94CB8E85E40F94CEB4882329F040
:10C830000F94C6B46B017C0105C0C12CD12CE12C36
:10C8400000ECF02E8CE40F94CEB481110F94C6B49A
:10C850008AE50F94CEB4882329F00F94C6B42B0137
:10C860003C011CC020E030E048EC51E460915E10D7
:10C8700070915F1080916010909161100F9493BC43
:10C8800087FF07C0412C512C18ED612E11E4712E49
:10C8900005C0412C512C612CB0E47B2E88E50F940F
:10C8A000CEB4882339F00F94C6B46AAF7BAF8CAF97
:10C8B0009DAF0AC0812C912CA3E5AA2EA3E4BA2E29
:10C8C0008AAE9BAEACAEBDAE89E50F94CEB48823E4
:10C8D00049F00F94C6B422966CAF7DAF8EAF9FAF78
:10C8E000229706C022961CAE1DAE1EAE1FAE22972A
:10C8F00080913710882311F40C9498748FE694E09B
:10C900000F940566882311F40C949874332433949F
:10C910000F94CB8E80913F0F882329F060E086E151
:10C9200090E00E94C7CF90904B0267969FAE6797AA
:10C9300020904C02E091060DF0E0EE0FFF1FE15851
:10C94000FA4EA080B1802496BFAEAEAE2497B5015A
:10C95000BB0C880B990B0F9499BC2A966CAF7DAFDA
:10C960008EAF9FAF2A972091CA193091CB196C9640
:10C970003FAF2EAF6C978091561090915710A091B9
:10C980005810B09159102E968CAF9DAFAEAFBFAF7F
:10C990002E9789839A83AB83BC8380905A109090A2
:10C9A0005B10A0905C10B0905D1062968CAE9DAE56
:10C9B000AEAEBFAE62978D829E82AF82B886209166
:10C9C0005E1030915F10409160105091611066963A
:10C9D0002CAF3DAF4EAF5FAF669729873A874B8745
:10C9E0005C872091621030916310409164105091E7
:10C9F00065102D873E874F87588BC701B6010F946E
:10CA0000FAC16093621070936310809364109093E6
:10CA1000651046E05DE05F934F93812C912C98EE7A
:10CA2000A92E92E4B92E22E6C22E20E1D22E6696DD
:10CA3000ECACFDAC0EAD1FAD669762962CAD3DAD76
:10CA40004EAD5FAD62972E966CAD7DAD8EAD9FAD58
:10CA50002E970F942D270F94CB8E20915E1030913E
:10CA60005F104091601050916110C301B2010F94AA
:10CA7000FAC17B018C0160935E1070935F1080930C
:10CA800060109093611020915A1030915B1040918A
:10CA90005C1050915D10609156107091571080910C
:10CAA000581090915910A6E0BDE0BF93AF93812C30
:10CAB000912CE0E7AE2EE1E4BE2E0F942D270F94CB
:10CAC000CB8E8AAC9BACACACBDAC80925610909235
:10CAD0005710A0925810B092591022962CAD3DAD2F
:10CAE0004EAD5FAD229720935A1030935B10409368
:10CAF0005C1050935D10E0905E10F0905F1000911C
:10CB000060101091611046E05DE05F934F93812CBF
:10CB1000912CF8E4AF2EF2E4BF2E22962CAD3DAD61
:10CB20004EAD5FAD22976AAD7BAD8CAD9DAD0F94E0
:10CB30002D270F94CB8E0F900F900F900F900F908A
:10CB40000F9080913710811124C084E090E0909381
:10CB50002902809328020F94A4592B013C0187EAF3
:10CB600091E10E94A8D3CC24C394D12CE12CF12CC8
:10CB7000D1100C94DC740E943AF1882311F40C94C7
:10CB8000DC749FB7F894809102018B7F809302013F
:10CB90009FBF1092B00680913710882319F00E9431
:10CBA0000EA102C00E94AFC60F94CB8E80913710A9
:10CBB00081115DC084E090E0909329028093280267
:10CBC00041E060E080EC92E10E94F6D38093B006F1
:10CBD000811148C00E9438F862E080E00E9442F370
:10CBE00089ED96E40E9469F220E030E048EC52E4DE
:10CBF0006091561070915710809158109091591073
:10CC00000F94F9C160935610709357108093581089
:10CC100090935910E0905E10F0905F1000916010BA
:10CC20001091611020915A1030915B1040915C106E
:10CC300050915D10E6E0FDE0FF93EF93812C912C85
:10CC4000B8E4AB2EB2E4BB2EE2E6CE2EE0E1DE2E5F
:10CC50000F942D270F94CB8E80E992E10E949AD4F5
:10CC60000F900F9080913710882309F47EC0311007
:10CC700072C08091F50D882329F060E080913F0219
:10CC80000E9455A084E090E09093290280932802AE
:10CC900080ED91E10E94A8D3FF24F39400E010E01E
:10CCA0000E943AF1811139C00F94FF8781E00F94FF
:10CCB0003946043F31E0130711F400E010E08091A1
:10CCC000010184608093010101151105A1F4809197
:10CCD000090790910A07009721F00197B9F4FF2006
:10CCE000A9F09FB7F89480910201846080930201BB
:10CCF0009FBFF12C0BC00431110541F49FB7F8948C
:10CD0000809102018B7F809302019FBF0F5F1F4FB5
:10CD100084E090E00F947C4AC3CF9FB7F894809151
:10CD200002018B7F809302019FBF8091F50D8823C4
:10CD300091F00E9438F862E080E00E9442F389EDB1
:10CD400096E40E9469F287E10E94849E40E060E0E0
:10CD500080E00E94AE9A2A964CAD5DAD6EAD7FAD7F
:10CD60002A97832D0F94F7A859C00E9438F861E0E4
:10CD700080E00E9442F389E292E10E9469F2809190
:10CD80000802811107C062E00E9442F386E192E14D
:10CD90000E9469F284E090E0909329028093280237
:10CDA0000E94178F0E943AF181111AC00F94FF87D9
:10CDB00081E00F9439460E945E8F882399F3809119
:10CDC000090790910A07029728F480910201846074
:10CDD0008093020182E390E00F947C4A0F94A98033
:10CDE0000E94BC8D82E090E09093290280932802FB
:10CDF0000F947EA98091090790910A07029728F461
:10CE00008091020184608093020182E390E00F949C
:10CE10007C4A0F94A98080E00E9442F83110F9C04A
:10CE20001092B006F4E0CF2ED12CA2E0AA2EB12CA5
:10CE30008091B006813009F4ECC01092B006D09217
:10CE40002902C09228020E9438F860E080E00E9427
:10CE500042F38FE592E10E9469F261E081E00E9475
:10CE600042F383E59DE30E9469F262E081E00E9463
:10CE700042F38BE492E10E9469F263E081E00E9458
:10CE800042F389E392E10E9469F261E080E00E944E
:10CE900042F384E794E00E94DFF1E090CC190E2C7D
:10CEA000000CFF080E94848D01E010E08091B00624
:10CEB000811168C00F94FF8781E00F9439468091FB
:10CEC000CC19082E000C990B9701281B390B37FF42
:10CED00003C0319521953109253031050CF444C04A
:10CEE0008E159F0514F401501109E816F90634F463
:10CEF0000F5F1F4F0430110564F009C004301105A5
:10CF000034F40115110529F401E010E002C003E03A
:10CF100010E061E080E00E9442F380E496E00E942D
:10CF2000DFF162E080E00E9442F380E496E00E943C
:10CF3000DFF163E080E00E9442F380E496E00E942B
:10CF4000DFF1602F80E00E9442F384E794E00E94CA
:10CF5000DFF1E090CC190E2C000CFF0864E670E0C5
:10CF600080E090E00F946C590E943AF1882309F414
:10CF70009DCF0093B00664EF71E080E090E00F94E5
:10CF80006C5994CF0E9438F80F943C94B0922902C7
:10CF9000A09228028091B0068230F9F0833071F5BA
:10CFA0000F94CB8E0E94C4A70E9438F860E080E006
:10CFB0000E9442F382E792E10E9469F262E080E01F
:10CFC0000E9442F389ED96E40E9469F287E99DE1AF
:10CFD0000F94BCAC0F94CB8E2BCF8091371088234D
:10CFE00051F02A964CAD5DAD6EAD7FAD2A9780E0D5
:10CFF0000F94F7A81DCF0F947EA91ACF0E9438F87E
:10D0000062E080E00E9442F380E892E10E9469F2CF
:10D010000FCF81E00E9442F86C964EAD5FAD6C97E9
:10D020005093CB194093CA1931103FC020E030E033
:10D0300040EA50E460916210709163108091641036
:10D04000909165100F94FAC1609362107093631011
:10D050008093641090936510E0905E10F0905F10E4
:10D06000009160101091611020915A1030915B1066
:10D0700040915C1050915D10609156107091571066
:10D080008091581090915910E6E0FDE0FF93EF93E6
:10D09000812C912CA12CB0E4BB2EE2E6CE2EE0E157
:10D0A000DE2E0F942D270F900F90E0905E10F090E1
:10D0B0005F1000916010109161102D813E814F81B1
:10D0C000588569817A818B819C81B6E06B2EBDE0A9
:10D0D0007B2E7F926F92812C912CE8E4AE2EE2E4BD
:10D0E000BE2EF2E6CF2EF0E1DF2E0F942D270F9407
:10D0F000CB8EE984FA840B851C852D813E814F817E
:10D10000588569817A818B819C817F926F92812C75
:10D11000912CA0E7AA2EA1E4BA2E0F942D270F94EC
:10D12000CB8ECE010D960E946AEA80E1FE01319617
:10D13000A6E5B0E101900D928A95E1F780E1E6E580
:10D14000F0E1A0E4BFE001900D928A95E1F76796C7
:10D150005FAD679750934B0220924C022F925F93E2
:10D1600081EE97E09F938F938E01015E1F4F1F9377
:10D170000F930F94F7BB60E0C8010E94089786E305
:10D1800095E10F944C0B1092DB0D1092DA0D0FB657
:10D19000F894DEBF0FBECDBF3FC50E94FCDB3CC58F
:10D1A00083E50F94CEB4882309F436C50F94C6B432
:10D1B0000F9459C36B017C012B0189ED96E40F9408
:10D1C0004C0BE2EBFEE084918F01882339F00F9441
:10D1D0006F550F5F1F4FF8018491F7CF0D2C000C96
:10D1E000EE08FF08C701B6010F94596B8AE00F944F
:10D1F0006F550F94A4594B015C011092F40D60918E
:10D200000A0D70910B0D072E000C880B990B0F94D3
:10D2100099BC20E030E0A9010F9493BC811111C0AA
:10D2200060917F1570918015072E000C880B990B6B
:10D230000F9499BC11E020E030E0A9010F9493BC59
:10D24000811110E0052C000C66087708ADEA2A2E43
:10D25000AEE03A2E111115C08091F40D81116CC011
:10D26000C301B2010F9499BC209192193091931986
:10D2700040919419509195190F9445C418168CF04B
:10D280005BC0C301B2010F9499BC209192193091F7
:10D29000931940919419509195190F9493BC87FF5D
:10D2A0004BC00F94A459DC01CB0188199909AA0934
:10D2B000BB09893E9340A105B10508F434C0EFEAEB
:10D2C000FEE084915F01882341F00F946F55FFEFDA
:10D2D000AF1ABF0AF5018491F6CF6091921970914F
:10D2E0009319809194199091951941E00F94F455F8
:10D2F000F1018491FDEAAF2EFEE0BF2E882341F0BC
:10D300000F946F55FFEFAF1ABF0AF5018491F6CF66
:10D31000C701B6010F94596B8AE00F946F550F94B3
:10D32000A4594B015C010F94FF8780E00F943946AC
:10D3300080E00E9466F08ECF8AE598E10F944C0B56
:10D340006BC48FE30F94CEB4882309F4BCC00F9450
:10D35000EC671A821982882381F006E714E0D8016D
:10D360008D918D01882319F00F946F55F8CF8AE0C5
:10D370000F946F550AE814E00AC001EA14E0F801BE
:10D3800081918F01882399F30F946F55F8CFD801BD
:10D390008D918D01882319F00F946F55F8CF8AE095
:10D3A0000F946F5588248A94982C540173E2472E69
:10D3B000512C612C712CE0EB2E2EEFE03E2E1AAE9C
:10D3C00069817A81072E000C880B990B0F9499BC08
:10D3D0002091A6103091A7104091A8105091A9104B
:10D3E0000F94E8C26B017C012AAD21110DC0E9EA5E
:10D3F000FEE084918F01882359F00F946F550F5FE1
:10D400001F4FF8018491F7CFC501B4010F94596BF8
:10D41000E6EAFEE084918F01882339F00F946F557E
:10D420000F5F1F4FF8018491F7CFC301B2010F9432
:10D43000596BE3EAFEE084918F01882339F00F9461
:10D440006F550F5F1F4FF8018491F7CF69817A8183
:10D45000072E000C880B990B0F94596BE0EAFEE045
:10D4600084918F01882339F00F946F550F5F1F4F00
:10D47000F8018491F7CF20E030E04AE754E4C70197
:10D48000B6010F9400B642E00F94F4558AE00F9471
:10D490006F55FAADFF5FFAAFF63009F4BDC3BE01B8
:10D4A0006F5F7F4FC1010F948840B2E02B0E311C9B
:10D4B000E5E04E0E511C611C711CFFEF8F1A9F0A94
:10D4C000AF0ABF0A7DCF81E20F94CEB4882309F45E
:10D4D0004AC061E086EA9FE00F949EC188E090E038
:10D4E0009A838983BE016F5F7F4F80EB9FE00F942B
:10D4F000A24088E190E09A838983BE016F5F7F4FED
:10D5000082EB9FE00F94A24080E390E09A838983AE
:10D51000BE016F5F7F4F84EB9FE00F94A24080E5D8
:10D5200090E09A838983BE016F5F7F4F86EB9FE017
:10D530000F94A24088E790E09A838983BE016F5FD1
:10D540007F4F88EB9FE00F94A24005EB14E0D801D9
:10D550008D918D01882319F00F946F55F8CF8AE0D3
:10D560000F946F5559C38AE50F94CEB4882319F1EF
:10D5700061E086EA9FE00F949EC11A82198200EB57
:10D580001FE0BE016F5F7F4FC8010F94A2400E5F86
:10D590001F4F0A3BBFE01B07A1F706EC14E0F801A0
:10D5A00081918F01882319F00F946F55F8CF8AE08D
:10D5B0000F946F5531C383E50F94CEB4882309F4DB
:10D5C000CEC00F94C6B40F9459C37A83698389E49B
:10D5D0000F94CEB4882309F41FC30F94C6B40F94DC
:10D5E0005FC3653008F018C3862F90E08852984FCB
:10D5F000BE016F5F7F4F880F991F0F94A24000ED0F
:10D6000014E0D8018D918D01882319F00F946F5586
:10D61000F8CF8AE00F946F550AE814E0F801819181
:10D620008F01882319F00F946F55F8CF8AE00F947B
:10D630006F552EEA222E2FE0322E44244A94542C89
:10D64000320143E2842E912CA12CB12C1AAE1A8205
:10D650001982FAADFF2331F0BE016F5F7F4FC10128
:10D660000F94884069817A81072E000C880B990BF2
:10D670000F9499BC2091A6103091A7104091A8104A
:10D680005091A9100F94E8C26B017C012AAD2111C1
:10D690000DC0ECE9FEE084918F01882359F00F94CE
:10D6A0006F550F5F1F4FF8018491F7CFC301B2018F
:10D6B0000F94596BE9E9FEE084918F01882339F0DA
:10D6C0000F946F550F5F1F4FF8018491F7CFC5017D
:10D6D000B4010F94596BE6E9FEE084918F01882331
:10D6E00039F00F946F550F5F1F4FF8018491F7CFFA
:10D6F00069817A81072E000C880B990B0F94596B66
:10D70000E3E9FEE084918F01882339F00F946F558F
:10D710000F5F1F4FF8018491F7CF20E030E04AE718
:10D7200054E4C701B6010F9400B642E00F94F455DB
:10D730008AE00F946F55FAADFF5FFAAF25E0820ED5
:10D74000911CA11CB11C3FEF431A530A630A730AD0
:10D7500042E0240E311CF63009F079CF5DC2E2E8D8
:10D76000FEE084918F01882309F456C20F946F550F
:10D770000F5F1F4FF8018491F6CF0F94CB8E8BE48F
:10D780000F94CEB4882399F00F9487B46B017C0179
:10D7900020E030E0A9010F9445C487FD08C0C09285
:10D7A000670FD092680FE092690FF0926A0F82E5DE
:10D7B0000F94CEB4882361F00F9487B46B017C0181
:10D7C00020E030E0A9010F9493BC87FF89C006C018
:10D7D000C12CD12C90E8E92E9FEBF92E84E40F9414
:10D7E000CEB4882329F00F9487B44B015C0106C0A6
:10D7F000812C912C80E8A82E8FEBB82E87E50F9412
:10D80000CEB4882329F00F9487B42B013C0106C0C5
:10D81000412C512C00E8602E0FEB702E88E40F9401
:10D82000CEB4882339F00F9487B46AAF7BAF8CAF46
:10D830009DAF08C020E030E040E85FEB2AAF3BAF8F
:10D840004CAF5DAF20E030E0A901C501B4010F94F9
:10D8500045C487FD45C020E030E0A901C301B20105
:10D860000F9445C487FD3CC020E030E0A9016AADBB
:10D870007BAD8CAD9DAD0F9445C487FD31C020E0DC
:10D8800030E0A901C501B4010F9493BC882391F144
:10D8900020E030E040E05FE3C501B4010F9400B642
:10D8A0006B017C012AAD3BAD4CAD5DADC301B20156
:10D8B0000F9400B64B015C01A7019601C701B601A8
:10D8C0000F9400B62BED3FE049E450E40F9400B60E
:10D8D0009B01AC01C501B4010F94E8C26B017C014E
:10D8E00020E030E0A901C701B6010F9445C487FFCD
:10D8F00004C00BC0C12CD12C7601C092630FD09212
:10D90000640FE092650FF092660FE5E3FFE5849106
:10D910008F01882339F00F946F550F5F1F4FF80167
:10D920008491F7CFE6EDF7E084918F01882339F0F9
:10D930000F946F550F5F1F4FF8018491F7CF6091DF
:10D94000670F7091680F8091690F90916A0F42E0A4
:10D950000F94F4558AE00F946F55E0EDF7E0849151
:10D960008F01882339F00F946F550F5F1F4FF80117
:10D970008491F7CFC090630FD090640FE090650F53
:10D98000F090660F20E030E0A901C701B6010F94C6
:10D9900093BC882349F042E0C701B6010F94F455C7
:10D9A0008AE00F946F5538C1EBECF7E084918F015A
:10D9B000882311F40C94624A0F946F550F5F1F4F28
:10D9C000F8018491F5CF0F94BCB40F9499BC6B010E
:10D9D0007C0120E030E0A9010F9493BC87FD40C09A
:10D9E00020E030EA40E854E4C701B6010F9445C492
:10D9F000181674F120E030E047E054E4C701B601A6
:10DA00000F9445C487FD2FC020E030E04CE752E47E
:10DA1000C701B6010F9400B620E030EA40E854E4B4
:10DA20000F94E8C20F945FC3162F802F0F94EEA9B6
:10DA3000612F802F0F94DDA90F5F043009F4ECC033
:10DA4000D5018D915D010F94CEB48823A9F3BBCF8E
:10DA5000C12CB0EADB2EB0E8EB2EB4E4FB2ED4CF21
:10DA6000C12CD12C760120E030E04CE752E4C70114
:10DA7000B6010F9400B620E034EB40E954E4D0CF77
:10DA800085E40F94CEB4882309F4C6C00F94C6B4BD
:10DA90000F945FC34B015C018B016830710569F025
:10DAA0006031710551F06032710539F060347105F3
:10DAB00021F06038710509F0AFC00F94CB8E80E083
:10DAC00091E07C0100901B0702C0F694E7940A9451
:10DAD000E2F7C4010E9488BE80931B0720912202B6
:10DAE00040912602682F83E00E94ABBE8090961082
:10DAF00090909710A0909810B0909910E016F106B1
:10DB000070F5C801B7010F94A4C66B01E12CF12C8C
:10DB1000C701B6010F9497BC9B01AC016091AA109C
:10DB20007091AB108091AC109091AD100F9400B635
:10DB30006093AA107093AB108093AC109093AD10CB
:10DB4000A5019401C701B6010F94AFC1609396106F
:10DB50007093971080939810909399105DC0C701AF
:10DB6000B8010F94A4C66B01E12CF12CC701B601DA
:10DB70000F9497BC9B01AC016091AA107091AB10FF
:10DB80008091AC109091AD100F94E8C26093AA10F0
:10DB90007093AB108093AC109093AD10C501B4019D
:10DBA000A70196010F94CBC620939610309397103F
:10DBB00040939810509399102FC08091371088236C
:10DBC00029F085E40F94CEB481119FC70F94756B33
:10DBD00023C083E40F94CEB490913710882329F0AA
:10DBE0009923D1F00E940EA117C09111FBCF0E9482
:10DBF000AFC612C080916E1590916F158C579C4ED8
:10DC00009F938F938DE69EE09F938F930F949EBB7F
:10DC10000F900F900F900F901092400D10923F0DAB
:10DC2000B2C284E50F94CEB4882309F442C1209196
:10DC3000100D3091110DF90131968F01021B130B5C
:10DC40007F0181918032C9F38930B9F3082E000C2D
:10DC5000990B0F94FFC6F7018083E091100DF091AE
:10DC6000110DE00FF11F808190ED980F953008F4B1
:10DC700061C08F3309F447C0883781F08336A9F13A
:10DC8000EDE5FEE084918F01882309F40EC10F9425
:10DC90006F550F5F1F4FF8018491F6CF80913710B9
:10DCA000882309F470C240E050E063EA7DE288E72F
:10DCB00093E10E94CCC780933E0290913F0289136A
:10DCC00007C08091460D882319F082E49EE064C06D
:10DCD0000F94CB8E80913E028F5F0E94849E43E022
:10DCE00061E081E00E94AE9A4EC280913710882395
:10DCF00009F449C20F94CB8E0E94489F80913E0246
:10DD000080933F0261C08091371040E050E088234B
:10DD100051F063EA7DE288E793E10E94CCC78093EB
:10DD20003E0211E01BC06EE573E187E693E10E94BD
:10DD3000CCC752C70F94C6B40F945FC3862F6093AD
:10DD40003E0290913710992341F09091ED0699236E
:10DD500021F09091490291113DC710E00F94CB8EB4
:10DD600080913E0221E030E0082E01C0220F0A948B
:10DD7000EAF79091450D292B2093450D909137108E
:10DD8000992329F190913F0289130DC09091460D7E
:10DD9000992349F087E29EE09F938F930F949EBB57
:10DDA0000F900F90F0C18F5F0E94849E43E061E06E
:10DDB00081E00E94AE9A0E94489F80913E0280932B
:10DDC0003F02112309F4DFC10E94E898DCC18823D7
:10DDD00009F432C0E5E3FFE584918F01882339F02F
:10DDE0000F946F550F5F1F4FF8018491F7CFE5E255
:10DDF000FEE084918F01882339F00F946F550F5FF7
:10DE00001F4FF8018491F7CF60913E0270E080E0EF
:10DE100090E00F94596B8AE00F946F55EDECF5E0AC
:10DE200084918F01882309F440C00F946F550F5FD0
:10DE30001F4FF8018491F6CF86E40F94CEB4882367
:10DE400099F00F94C6B46B017C0120E030E0A90189
:10DE50000F9445C4181644F4C0925602D09257024B
:10DE6000E0925802F0925902E5E3FFE584918F01B8
:10DE7000882339F00F946F550F5F1F4FF80184917D
:10DE8000F7CFEBEBF5E084918F01882339F00F9405
:10DE90006F550F5F1F4FF8018491F7CF6091060D0A
:10DEA00070E080E090E00F94596B8AE00F946F551A
:10DEB0006AC184E40F94CEB4882309F403C10F949B
:10DEC000C6B40F9459C36330710509F05CC184E78F
:10DED00095E09F938F930F949EBB81E40F94CEB4F3
:10DEE0000F900F908823B9F08091100D9091110D33
:10DEF000DC0111962C91283741F440E150E060E0BC
:10DF000070E002960F9428B804C00F94C6B40F9422
:10DF100059C37B0102C0E12CF12C83E40F94CEB4F1
:10DF2000882339F00F94C6B40F9459C3262F872F36
:10DF300002C020E080E1BFE1FB22A22EB82EE1E08A
:10DF4000AE16E0E1BE0618F0A12CA0E1BA2EC50184
:10DF50008E0D9F1D8130904128F080E090E15C01A2
:10DF6000AE18BF0888E50F94CEB4882309F470C0BA
:10DF70002091100D3091110D2F5F3F4FAE014F5F7B
:10DF80005F4F6A01FA0100E010E0D9018C912F5F28
:10DF90003F4F882389F10031110561F18032A9F3E7
:10DFA0008A3051F190ED980F9A3018F48295807F65
:10DFB00007C09FE9980F9630A8F48295807F80571C
:10DFC0009D012E5F3F4F11969C9140ED490F4A30C5
:10DFD00010F4842B0BC04FE9490F463018F49755C5
:10DFE000892B04C011950195110906C081930F5F1B
:10DFF0001F4FCBCF00E110E058010115110541F191
:10E00000812C912CD6016D916D01C4018E0D9F1D47
:10E010000F949EC1BFEF8B1A9B0A0815190591F743
:10E02000FF92EF921F930F9387E495E09F938F9356
:10E030000F949EBB6091D5197091D6198AE090E03B
:10E040000F9419BB0F900F900F900F900F900F909F
:10E050006701E12CF12CA114B10409F494C08D2DB9
:10E060000F944EB48C2D0F944EB46091D5197091CD
:10E07000D61980E290E00F9419BB10E1EFEFCE1AB1
:10E08000DE0AEE0AFE0AC60101970F946EC1082F40
:10E090006091D5197091D61980E290E00F9419BB68
:10E0A000802F0F944EB4F1E0AF1AB10811F0115067
:10E0B00029F76091D5197091D6198AE090E00F94F4
:10E0C00019BBC9CFE5E3FFE584918F01882339F0BF
:10E0D0000F946F550F5F1F4FF8018491F7CFE7EE54
:10E0E000F5E084918F01882339F00F946F550F5F0D
:10E0F0001F4FF8018491F7CF00916E1510916F15A5
:10E100000C571C4ED8018D918D01882319F00F9466
:10E110006F55F8CFE0E2FEE084918F01882309F487
:10E12000C4CE0F946F550F5F1F4FF8018491F6CF47
:10E13000C0904C0FD0904D0FE0904E0FF0904F0FCD
:10E1400020916210309163104091641050916510DD
:10E15000C701B6010F94F9C14B015C012DEC3CECF9
:10E160004CEC5DEB0F9493BC87FD3AC02DEC3CEC7E
:10E170004CEC5DE3C501B4010F9445C418160CF4D2
:10E1800038C00F9481B081E090E090932902809391
:10E1900028020F94A4596093880F7093890F80937D
:10E1A0008A0F90938B0FE0916E15F0916F15EF57DA
:10E1B000FC4E8081813019F0863009F010C5EAE507
:10E1C000F8E184918F01882339F00F946F550F5F28
:10E1D0001F4FF8018491F7CF8AE00F946F55FFC469
:10E1E000E091060DF0E0E05BF04F8081811194C476
:10E1F00009C0E091060DF0E0E05BF04F80818823DC
:10E2000009F4BFCFC0926210D0926310E092641004
:10E21000F092651082E690E10E946AEAE091060DB4
:10E22000F0E0E05BF04F908181E089270F940CAB28
:10E23000D6C420E030E040E85FE360916210709166
:10E24000631080916410909165100F94FAC16093EF
:10E250006210709363108093641090936510E09047
:10E260005E10F0905F10009160101091611020918D
:10E270005A1030915B1040915C1050915D1060918C
:10E280005610709157108091581090915910E6E0F7
:10E29000FDE0FF93EF93812C912CE8ECAE2EE3E4AC
:10E2A000BE2EF2E6CF2EF0E1DF2E0F942D270F9039
:10E2B0000F900C94C14582E090E0909329028093E6
:10E2C00028021092E10D1092E00D0C940D4A0F946B
:10E2D000BCB4AB01BC0140935B1950935C196093D3
:10E2E0005D1970935E1986EA98E10F94F71E94CC3D
:10E2F0000F94C6B40F9459C38B010C94D94D0F944D
:10E30000CB8E88E50F94CEB4882319F0179A10921B
:10E31000070D89E50F94CEB4882319F0169A109250
:10E32000080D8AE50F94CEB485E40F94CEB488230B
:10E3300011F40C943053149A0C9430531A821982AD
:10E340004AE050E0BE016F5F7F4FC7010F9428B8CD
:10E3500078A36F8F89819A818816990609F05CCC21
:10E360004AE050E0BE016F5F7F4FC6010F9428B8AE
:10E370007AA369A389819A816816790609F04CCC41
:10E380004AE050E0BE016F5F7F4FC5010F9428B88F
:10E390007CA36BA389819A810817190709F03CCCEB
:10E3A0008FE790E09EA38DA35801EFEFAE1ABE0A4F
:10E3B000D8018C918D3211F575016701BFEFCB1A31
:10E3C000DB0AF70180810F94220B382E811102C0E5
:10E3D0007601F3CFEA18FB08DE2CC70199278330BA
:10E3E000910569F543E050E06DE57EE5C5010F94C8
:10E3F00071BA892B09F042C01EA21DA2332009F474
:10E400000BCCCE0101960F94307F882309F404CC05
:10E41000FE017F96DE011196AE01495D5F4F2191AD
:10E4200031918D919D918217930708F44CC0281764
:10E43000390708F4F1CB4E175F0789F7EDCB85302C
:10E44000910571F445E050E067E57EE5C5010F9464
:10E4500071BA892B99F481E090E09EA38DA3CECF71
:10E46000049761F444E050E062E57EE5C5010F9455
:10E4700071BA892B19F482E090E0EFCF8EEF8E0D08
:10E48000823008F0C9CBD80111968C9111978F7DFD
:10E49000823509F0C1CB12968C918F7D833409F0BF
:10E4A000BBCBB2E0DB1203C083E090E0D6CFF80133
:10E4B000838190ED980F9A3008F0AECB082E000CB7
:10E4C000990B8E97CACF80EF92E10E94A8D34AE6BB
:10E4D0005DE062E080E00E942DF8D2011D912D01E7
:10E4E000812F0F94220B811108C06EEC76E0812FF2
:10E4F000110F990B0F9419BBF0CF40EE52E163E07E
:10E5000080E00E942DF88091090790910A070297F8
:10E5100028F48091020184608093020182E390E0FC
:10E520000F947C4A0F94A98084EF91E00F947C4A69
:10E530008091090790910A07029728F480910201BF
:10E5400084608093020182E390E00F947C4A0F94F0
:10E55000A98080E090E00F94FFA981E00E9442F83A
:10E560000E9438F880E00E9466F056CBE896CCAC6A
:10E57000DDACEEACFFACE897C80ED91EEA1EFB1E60
:10E58000E8962CAD3DAD4EAD5FADE897281B390B3D
:10E590004A0B5B0B2A966CAD7DAD8EAD9FAD2A9775
:10E5A0000F94AFC1A70196010F94CBC6DA01C90140
:10E5B000840D951DA61DB71D84319105A105B105DA
:10E5C000E4F02C013D018C3E9105A105B1052CF034
:10E5D0006BEE462E512C612C712C40E844165104F0
:10E5E00061047104DCF05EEF852E912CA12CB12C1E
:10E5F00084189508A608B7080AC034E1432E512CA8
:10E60000612C712C44E1842E912CA12CB12C2A96E2
:10E610008CAE9DAEAEAEBFAE2A9706C02A964CAE6B
:10E620005DAE6EAE7FAE2A97E7E4FDE084918F0188
:10E63000882339F00F946F550F5F1F4FF8018491B5
:10E64000F7CFC301B2010F94596BE2E4FDE084916E
:10E650008F01882339F00F946F550F5F1F4FF8011A
:10E660008491F7CF2A966CAD7DAD8EAD9FAD2A9784
:10E670000F94596BEBE3FDE084918F01882339F00F
:10E680000F946F550F5F1F4FF8018491F7CF42E051
:10E69000A3966FADA397A5967FADA597A6968FADD0
:10E6A000A697AA969FADAA970F94F455E4E3FDE0D0
:10E6B00084918F01882339F00F946F550F5F1F4F9E
:10E6C000F8018491F7CF42E0AE966FADAE97AF966A
:10E6D0007FADAF97E0968FADE097E1969FADE19764
:10E6E0000F94F4558AE00F946F5580917B0D9091B3
:10E6F0007C0D039714F40C94A05E2A966CAD7DAD4E
:10E700008EAD9FAD2A970F9499BC20E030E040E891
:10E7100050E40F9400B64B015C01A3962FADA39774
:10E72000A5963FADA597A6964FADA697AA965FADC5
:10E73000AA97AE966FADAE97AF967FADAF97E096C6
:10E740008FADE097E1969FADE1970F94F9C120ED71
:10E750003FE049E450E40F9400B620E030E040E0B0
:10E760005FE30F9400B69B01AC01C501B4010F94A7
:10E77000E8C24B015C01C701B6010F9499BC20E0CF
:10E7800030E04AE754E40F94E8C26B017C01EEE20A
:10E79000FDE084918F01882339F00F946F550F5F4E
:10E7A0001F4FF8018491F7CF42E0C501B4010F94E7
:10E7B000F455E8E2FDE084918F01882339F00F944D
:10E7C0006F550F5F1F4FF8018491F7CF42E0C701EB
:10E7D000B6010F94F4558AE00F946F552AE939E990
:10E7E00049E15FE3C501B4010F9400B64B015C0140
:10E7F0006093F90E7093FA0E8093FB0E9093FC0ECB
:10E800009B01AC010F94FAC1A70196010F94E8C2D5
:10E810006093F50E7093F60E8093F70E9093F80EBA
:10E82000A5019401C701B6010F9400B620E030E0C5
:10E8300040E05EE30F9400B66093F10E7093F20E29
:10E840008093F30E9093F40EEAE1FDE084918F0142
:10E85000882339F00F946F550F5F1F4FF801849193
:10E86000F7CF8AE00F946F55E4E1FDE084918F01CA
:10E87000882339F00F946F550F5F1F4FF801849173
:10E88000F7CF6091F90E7091FA0E8091FB0E909186
:10E89000FC0E42E00F94F4558AE00F946F55EEE0C1
:10E8A000FDE084918F01882339F00F946F550F5F3D
:10E8B0001F4FF8018491F7CF6091F50E7091F60E1D
:10E8C0008091F70E9091F80E42E00F94F4558AE093
:10E8D0000F946F55E8E0FDE084918F01882339F0B3
:10E8E0000F946F550F5F1F4FF8018491F7CF609120
:10E8F000F10E7091F20E8091F30E9091F40E42E0C1
:10E900000F94F4558AE00F946F550C94A05E809399
:10E91000BA0F0C94BB5ECC57DF4F1882C458D0405E
:10E920000C94E25E84E690E00F947C4A0C946A605A
:10E93000312C0C948864E12CF12C809101018460CD
:10E9400080930101E114F10409F04EC080910907A0
:10E9500090910A070097F1F10197D1F1AFEFEA1A10
:10E96000FA0AB1E0DB1609F452C0DB1608F04AC01F
:10E9700084E090E00F947C4A0F94A45993018201A3
:10E980000054184D264F3F4F061717072807390721
:10E9900010F00C94B8658CE791E10E94A8D31F8E0B
:10E9A00018A219A21AA2CE014F960F94E0800F94DC
:10E9B000CB8E149ADD24D3940F94FF8781E00F94BB
:10E9C0003946F4EFEF16F1E0FF0609F0B6CFB3CF0A
:10E9D000CC2021F29FB7F89480910201846080934B
:10E9E00002019FBFC12CBACF94E1E916F10409F0EE
:10E9F000B5CF9FB7F894809102018B7F809302017D
:10EA00009FBFACCFE2E0DE16E1F00C94B86584E085
:10EA100090E00F947C4A0E943AF1882369F2E091D9
:10EA2000060DF0E0EE0FFF1FE158FA4E24968EAC73
:10EA30009FAC2497918280820F94374002E0D02EC1
:10EA4000BBCF0091060D10E0F801EE0FFF1FE1585B
:10EA5000FA4E60817181072E000C880B990B0F9480
:10EA600099BC000F111F000F111FF801EB5FF04F51
:10EA700020813181428153810F94F9C14B015C01A6
:10EA800020E030E0A9010F9445C418165CF420E0A2
:10EA900030E040E85FE3C501B4010F9493BC87FF09
:10EAA00016C00AC020E030E040E85FEBC501B401C9
:10EAB0000F9445C418165CF487EA91E10E94A8D32C
:10EAC0000F94A4592B013C01D12C0C94BB6564E03C
:10EAD00081E00E9442F3E091060D24E0E29FF00104
:10EAE0001124EB5FF04F80819181A281B3818F8FE0
:10EAF00098A3A9A3BAA3CE014F960E94D8910E94D1
:10EB0000DFF1F4E1EF2EF12C57CF0F94C6B40F9440
:10EB10005FC360933E025AC82DEC3CEC4CEC5DE3C5
:10EB2000C501B4010F9445C418160CF46BCB29CB66
:10EB3000A5019401F101662D772D8F2F922D0F9451
:10EB400093BC181614F40C94B23C0C94C33C3320C0
:10EB5000E9F18BEA289E212D112426952796AFAD49
:10EB600027978A2F90E0820F911D0EC0332011F459
:10EB70000C940340822D90E02796EFAD2797B3E0E9
:10EB8000EB9F800D911D1124880F991F8D53904F7D
:10EB90000F947BC1BC01990F880B990B0F9499BC02
:10EBA0002AE037ED43E25CE30F9400B620918D1527
:10EBB00030918E1540918F15509190150F94FAC198
:10EBC0002B013C01F1E0FEAF0C94064021E02EAF9A
:10EBD0000C9403400F9457B480933E02BEC8CC57A8
:10EBE000DF4F0FB6F894DEBF0FBECDBFDF91CF91E0
:10EBF0001F910F91FF90EF90DF90CF90BF90AF905B
:10EC00009F908F907F906F905F904F903F902F904C
:10EC100008952F923F924F925F926F927F928F92C0
:10EC20009F92AF92BF92CF92DF92EF92FF920F939B
:10EC30001F93CF93DF93CDB7DEB7C95CD1090FB671
:10EC4000F894DEBF0FBECDBF782E81E00F94B56C77
:10EC5000711025C010920B0D10920A0D19821A82A4
:10EC60001B821C82CE0101960F94E08061E080EC53
:10EC70009FE00F9480C160E08FEB9FE00F9480C114
:10EC800060E08EEB9FE00F9480C160E08DEB9FE031
:10EC90000F9480C160E08CEB9FE00F9480C180E016
:10ECA0000E9442F80F94147C0E94CEED1092050D44
:10ECB0001092040D83E0E7E0FDE0DF011D928A95EC
:10ECC000E9F781E00F941B64C855DF4F998388836F
:10ECD000C85AD04087ED9CE10E94A8D30F944A64A3
:10ECE00040E050E061E080E090E00F94F66C40E09E
:10ECF00050E061E081E090E00F94F66CE0905E10EF
:10ED0000F0905F10009160101091611020915A10E6
:10ED100030915B1040915C1050915D1060915610E5
:10ED20007091571080915810909159100F94B677A8
:10ED30000E94A5E91092270220E030E040EA50E46A
:10ED40006091561070915710809158109091591001
:10ED50000F94FAC11B012C01609356107093571049
:10ED6000809358109093591020E030E040EA50E42E
:10ED700060915A1070915B1080915C1090915D10C1
:10ED80000F94FAC19B01AC0160935A1070935B1011
:10ED900080935C1090935D10E0905E10F0905F1097
:10EDA000009160101091611086E09DE09F938F9319
:10EDB000812C912CB0EAAB2EB1E4BB2E82E6C82E9A
:10EDC00080E1D82EC201B1010F942D270F94CB8E74
:10EDD0000F9454640F900F90882311F40C941D8AA3
:10EDE0008DE99CE10E949AD4772089F08DE69CE120
:10EDF0000E94A8D363E080E00E9442F361E070E0EB
:10EE000080E090E00E94C4F187E69CE110C087E4B6
:10EE10009CE10E94A8D362E080E00E9442F361E09E
:10EE200070E080E090E00E94C4F181E49CE10E94E7
:10EE300069F20F94EB6C71102EC084E090E0909317
:10EE400029028093280240E060E086E29CE10E9473
:10EE5000F6D3882321F08EEF9BE10E949AD488E6B6
:10EE60009BE10E949AD482E090E0909329028093E3
:10EE7000280287E49CE10E94A8D362E080E00E941F
:10EE800042F361E070E080E090E00E94C4F181E430
:10EE90009CE10E9469F2609027021092270220E014
:10EEA00030E040E85FE360915E1070915F10809108
:10EEB0006010909161100F94F9C17B018C016093F7
:10EEC0005E1070935F10809360109093611020919A
:10EED0005A1030915B1040915C1050915D10609120
:10EEE0005610709157108091581090915910E6E08B
:10EEF0004E2EEDE05E2E5F924F92812C912CF0EA27
:10EF0000AF2EF1E4BF2EA2E6CA2EA0E1DA2E0F94B6
:10EF10002D270F94CB8E80E090E0A0EAB0E48093A0
:10EF20005E1090935F10A0936010B093611081E029
:10EF30008093270284E00E9484C0E0905E10F090ED
:10EF40005F10009160101091611020915A10309163
:10EF50005B1040915C1050915D1060915610709163
:10EF6000571080915810909159105F924F920F94C2
:10EF70002D270F94CB8E0E94EDBF6092270282E076
:10EF80000F94B88E0F900F900F900F9020E030E00C
:10EF900040EA50E40F9493BC81110C94198A7720B5
:10EFA000E9F0C855DF4F88819981C85AD0400F9445
:10EFB000FA630E94BDEF0E94D0EB0E9470F3882399
:10EFC00011F40C94C9890F94556B803F11F00C9487
:10EFD000158A81E00F94F6670C94158A8AEF0F94D6
:10EFE000F66760E070E088EF9FE00F949AC10F949D
:10EFF000EB6C84ECEDE8F5E1DF011D928A95E9F711
:10F00000EEE7FFE184918F01882339F00F946F556B
:10F010000F5F1F4FF8018491F7CF61E070E080E04F
:10F0200090E00F94596B0F946D56BE016F5A7F4F4D
:10F0300087E49CE10E9496D362968FAD62978430FC
:10F0400020F083E062968FAF629780E090E0A0EAC4
:10F05000B0E480935E1090935F10A0936010B09323
:10F0600061102EE53FE1C657DF4F39832883CA5828
:10F07000D0408CE895E1CE57DF4F99838883C25802
:10F08000D040A0969FAF8EAFA097A8963FAF2EAF6F
:10F09000A89781E090E0A0E0B0E0AE968CAF9DAF85
:10F0A000AEAFBFAFAE970F94EB6C62966FAD629749
:10F0B00080E00E9442F3AE966CAD7DAD8EAD9FAD0B
:10F0C000AE970E94C4F181E49CE10E9469F265E57B
:10F0D00075E585E591E40E9462EBA896EEADFFAD83
:10F0E000A89785919591A591B4918093561090938E
:10F0F0005710A0935810B0935910A896EEADFFADDD
:10F10000A897349685919591A591B49180935A10C2
:10F1100090935B10A0935C10B0935D1060E070E082
:10F1200088E492E40E9462EB00914E1010914F101F
:10F13000209150103091511040914A1050914B1035
:10F1400060914C1070914D10809146109091471035
:10F15000A0914810B09149103F932F931F930F93A4
:10F160007F936F935F934F93BF93AF939F938F93CF
:10F170008AEE9EE19F938F930F949EBB0F94CB8E4C
:10F18000409146105091471060914810709149107D
:10F1900080914A1090914B10A0914C10B0914D105D
:10F1A000C0904E10D0904F10E0905010F090511041
:10F1B00021E00FB6F894DEBF0FBECDBF41315742FC
:10F1C0000CF420E08131974214F00C941F8A822FB6
:10F1D00090E0880F991FFC01EE51F14EA590B4907C
:10F1E000FC01E652F14E85909490DF92CF929F926F
:10F1F0008F92BF92AF921F922F9381EC9EE19F93CB
:10F200008F930F949EBB81EE9CE19F938F930F94FD
:10F210009EBB0F94184F809170008B7F809370007D
:10F22000EF9880916F008D7F80936F000FB6F894F8
:10F23000A8958091600088618093600010926000C2
:10F240000FBE1092030D1092020D8DE691E0909387
:10F25000010D8093000D8DEE91E09093FF0C809353
:10F26000FE0C00E028EC30E0A601B401C5010F94CB
:10F27000850700914E1010914F1020915010309141
:10F28000511040914A1050914B1060914C10709168
:10F290004D108091461090914710A0914810B09168
:10F2A00049103F932F931F930F937F936F935F9317
:10F2B0004F93BF93AF939F938F9381E89DE19F936B
:10F2C0008F930F949EBB8091461090914710A09110
:10F2D0004810B0914910782E692E80914A10909173
:10F2E0004B10A0914C10B0914D10582E492EC0904B
:10F2F0004E10D0904F10E0905010F09051100FB67B
:10F30000F894DEBF0FBECDBF48EF242E4CE1342E63
:10F3100095E0C91697EFD9060CF46EC01A821982CF
:10F320001F921F92A3E0AF93B4E8BF931F92E4E64D
:10F33000EF93DF92CF924F925F926F927F923F92C4
:10F340002F920F949EBB0FB6F894DEBF0FBECDBFB9
:10F3500089819A81803D924030F089819A81803AFA
:10F36000954050F512C0CE0101967C0100E010E0FE
:10F3700024E833E0A601652D742D872D962D0F947A
:10F38000E07D81110C94248AE8CFDE0111967D0185
:10F3900000E010E02CE73CEFA60144565109652D32
:10F3A000742D872D962D0F94E07D882329F0898177
:10F3B0009A8180539D4F1CC089819A8180379840E3
:10F3C00008F04AC0FE0131967F0104EB10E024E80A
:10F3D00033E0A601485C5109652D742D872D962DCB
:10F3E0000F94E07D8823C1F189819A8180569A4FDC
:10F3F0009A8389830C94248A00914E1010914F10A7
:10F40000209150103091511040914A1050914B1062
:10F4100060914C1070914D10809146109091471062
:10F42000A0914810B09149103F932F931F930F93D1
:10F430007F936F935F934F93BF93AF939F938F93FC
:10F4400080E39DE19F938F930F949EBB0FB6F8943A
:10F45000DEBF0FBECDBFD8C389819A8180349B4067
:10F46000A0F49E012F5F3F4F790104EB10E02CE7E1
:10F470003CEFA6014C525140652D742D872D962DE1
:10F480000F94E07D81110C940B8B80E0E981FA816F
:10F49000882311F40C94278A80914610909147108C
:10F4A000A0914810B091491040914A1050914B10D2
:10F4B00060914C1070914D1000914E1010914F10B2
:10F4C0002091501030915110FF93EF931F930F93A1
:10F4D0005F934F939F938F938DE59DE19F938F93C0
:10F4E0000F949EBB40914E1050914F106091501060
:10F4F0007091511000E028EC30E0B401C5010F9488
:10F50000850785E08F9380E78F9381E99EE19F9344
:10F510008F930F949EBB84E08F9388E38F938FE744
:10F520009EE19F938F930F949EBB80914610909184
:10F530004710A0914810B09149106A968CAF9DAFCA
:10F54000AEAFBFAF6A976896CEACDFAC68978091DC
:10F550004A1090914B10A0914C10B0914D10E29632
:10F560008CAF9DAFAEAFBFAFE29780914E10909140
:10F570004F10A0915010B09151106E968CAF9DAF6E
:10F58000AEAFBFAF6E971C0198E4291A310889E02D
:10F590008F9380E68F933F922F92E096AFADE097E6
:10F5A000AF93AF96BFADAF97BF936896EFAD689737
:10F5B000EF936796FFAD6797FF938AEA9DE19F936C
:10F5C0008F930F949EBB40914E1050914F106091BD
:10F5D0005010709151107A0120E931E0E0966EAD43
:10F5E0007FADE09768968EAD9FAD68970F948507C5
:10F5F000E0962EAD3FADE0973450EC963FAF2EAF86
:10F60000EC970FB6F894DEBF0FBECDBF812C912CC6
:10F61000D601B450E896BFAFAEAFE897F601FC5FF5
:10F62000C258DF4FF983E883CE57D040382D317070
:10F63000A3963FAFA39780FC02C00C942D8AEF964F
:10F640008FADEF97C158DF4F9881CF57D04000E082
:10F6500020E931E0A701EC966EAD7FADEC970F94F9
:10F660008507C0904A10D0904B10E0904C10F0905D
:10F670004D108091461090914710A0914810B09184
:10F68000491001E028EC30E0A101B6010F94850794
:10F69000C0904A10D0904B10E0904C10F0904D105C
:10F6A0008091461090914710A0914810B091491058
:10F6B0000FEF28EC30E040E659E0B6010F948507E3
:10F6C00080914E1090914F10A0915010B091511018
:10F6D0007C01A3966FADA39780910B01662311F473
:10F6E0000C94358A816080930B010000840125E031
:10F6F000000F111F2A95E1F7A3968FADA3978823DA
:10F7000011F40C94388A90EC492E55245A94652CA7
:10F71000752CC12CD12C90E4E3969FAFE397A12CDC
:10F72000B12C93B1A70142195309292F207194FFDD
:10F7300002C00C943F8A88EE9FEF840F951F97FDBF
:10F7400002C00C94438A80E090E0A80EB91E80911C
:10F750000B0121110C944D8A846080930B010000F1
:10F7600021110C94508A2E143F0434F484E00F9439
:10F77000A25AA1E0EA1AF10881E00F94A25A8BE59F
:10F7800099E00197F1F7E396FFADE397F150E39627
:10F79000FFAFE397F111C5CFB6E0B694A794BA9541
:10F7A000E1F7A3962FADA397222311F40C945F8A5F
:10F7B0008FE190E08C199D09800F911FFC01E257A9
:10F7C000F84FA0828091461090914710A091481068
:10F7D000B0914910840D951DA61DB71D809346104C
:10F7E00090934710A0934810B0934910C7010F2C75
:10F7F000000CAA0BBB0B80934E1090934F10A0935C
:10F800005010B09351103FEFC31AD30A60E2C616EE
:10F81000D10409F080CF0257184FF0E2BF2EA5EABD
:10F82000CA2EADE1DA2ED8018D918D011F928F93F2
:10F83000DF92CF920F949EBBBA940F900F900F90CF
:10F840000F90B110F0CF83EA9DE19F938F930F94B7
:10F850009EBBBFEF8B1A9B0AEC96EEADFFADEC970B
:10F86000E05CFF4FEC96FFAFEEAFEC970F900F9080
:10F87000F0E28F16910409F0D9CEEEE8AE2EEBE05F
:10F88000BE2E8EEA9BE0F501119211928E179F0712
:10F89000D9F780E090E0DC0175E0AA0FBB1F7A95F4
:10F8A000E1F7A257B84F40E2ED91F0E054E0F59552
:10F8B000E7955A95E1F7EE0FFF1FE257F44F2081CD
:10F8C00031812F5F3F4F31832083415069F701968B
:10F8D0008032910501F72EE8C22E2BE0D22E00E0F7
:10F8E00010E032EEE32E3DE1F32ED6018C9111961D
:10F8F0009C91B2E0CB0ED11C9F938F931F930F93DB
:10F90000FF92EF920F949EBB0F5F1F4F0F900F90CF
:10F910000F900F900F900F900031110531F78091EB
:10F92000900B9091910BE0E9FBE031E021E04191F7
:10F9300051918417950710F4322FCA012F5F20319F
:10F94000B1F7032F1F923F939F938F9389E09EE11E
:10F950009F938F930F949EBBECEAFBE00F900F9068
:10F960000F900F900F900F908EE0329122912A30DD
:10F97000310510F40C94628A8295807F20918E0B61
:10F9800030918F0B2037334010F00C94698A000FB0
:10F99000000F000F182F101B1F921F931F928F93A1
:10F9A0001F920F9382EF9DE19F938F930F949EBBC5
:10F9B0009EE8492E97E0592E0FB6F894DEBF0FBE91
:10F9C000CDBFF201202F30E0012F10E0808190E0C8
:10F9D0002817390710F00C946C8A821B930B982F10
:10F9E00080E0B8010F94A4C66F3F710519F010F0C4
:10F9F0006FEF70E06193AE16BF0641F700E010E0D4
:10FA0000BDEEAB2EBDE1BB2E8BEEC82E8DE1D82E08
:10FA1000C801A5E0880F991FAA95E1F7DC01A2575C
:10FA2000B84F7D01912CF70181917F011F928F9337
:10FA3000BF92AF920F949EBB93940F900F900F9034
:10FA40000F90F0E29F12EFCFDF92CF920F949EBB08
:10FA50000F5F1F4F0F900F9000321105C9F687E618
:10FA60009EE126EE3BE0AEECBBE0FC0145915491FB
:10FA70004D935D9302962A173B07B9F7612C712CC1
:10FA8000E12CF12C10E000E0A12C40E050E0EB96DE
:10FA90004FAFEB972EEC3BE0E8963FAF2EAFE897E9
:10FAA000A0E0B0E080E090E0B12C4A01860C971C09
:10FAB00020E030E014012A0E3B1E6EEF6B0DE39642
:10FAC0006FAFE397B1100C94708A6EEF620F6830DD
:10FAD00010F40C94778A2F5F3F4F2C30310591F74B
:10FAE000B3949096E896EEADFFADE8973296E8961F
:10FAF000FFAFEEAFE897FCE0BF12DACFE816F906E9
:10FB00002CF47C010A2DEB961FADEB974F5F5F4FF6
:10FB10004431510509F0BBCFA39420E2620E711C61
:10FB200034E1A312B2CFFF92EF921F920F931F9274
:10FB30001F938DE19EE19F938F930F949EBB0FB611
:10FB4000F894DEBF0FBECDBF93E4E916F10414F4C0
:10FB50000C94AD8A1F920F931F921F938EE49EE127
:10FB60009F938F930F949EBB1A5FE12EF12CA0E11F
:10FB7000EA1AF108E6E0EE0CFF1CEA95E1F7689658
:10FB8000EEADFFAD6897EE0EFF1E0A5FC02ED12CC2
:10FB9000F0E1CF1AD108F6E0CC0CDD1CFA95E1F7C4
:10FBA000E0962EAD3FADE097C20ED31E6C963FADF2
:10FBB0006C973F936B966FAD6B976F93DF92CF927D
:10FBC000FF92EF928DE39EE19F938F930F949EBBE4
:10FBD00000E028EC30E06C964EAD5FAD6C97B6015E
:10FBE000C7010F9485070FB6F894DEBF0FBECDBFD7
:10FBF00081E0D2011D922D01BEEF4B16BCE05B06E9
:10FC0000C1F781110C94B08A10E08AEA9EE19F93BB
:10FC10008F930F949EBB0F946B358091700084601E
:10FC200080937000EF9A80916F00826080936F00E4
:10FC300098E288E10FB6F894A895809360000FBE13
:10FC4000909360001092030D1092020D1092010D1E
:10FC50001092000D1092FF0C1092FE0C0F900F905E
:10FC6000112311F40C94508920E030E0A901A096F2
:10FC7000EEADFFADA09761817281838194810F9475
:10FC800000B6209156103091571040915810509165
:10FC900059100F94FAC1A096AEADBFADA0971196C2
:10FCA0006D937D938D939C931497C0905A10D09030
:10FCB0005B10E0905C10F0905D1020E030E0A90156
:10FCC00015966D917D918D919C9118970F9400B62A
:10FCD000A70196010F94FAC1A096EEADFFADA097D3
:10FCE000658376838783908720E030E040E850EC9E
:10FCF000C701B6010F9493BC87FF0CC080E090E071
:10FD0000A0E8B0EC80935A1090935B10A0935C1025
:10FD1000B0935D1020E030E040E450E460915E106C
:10FD200070915F1080916010909161100F94FAC1F2
:10FD300060935E1070935F108093601090936110D9
:10FD4000AE968CAD9DADAEADBFADAE970196A11D8B
:10FD5000B11DAE968CAF9DAFAEAFBFAFAE97A896BC
:10FD6000AEADBFADA8971896A896BFAFAEAFA89797
:10FD7000A096EEADFFADA0973896A096FFAFEEAF80
:10FD8000A097AE968CAD9DADAEADBFADAE970597CD
:10FD9000A105B10509F087C980E090E00F947C4A85
:10FDA00020E030E040E950EC60919115709192159F
:10FDB00080919315909194150F9493BC87FF43C045
:10FDC000EDE5FFE184918F01882339F00F946F55A1
:10FDD0000F5F1F4FF8018491F7CF8AE00F946F55A2
:10FDE000EBE2FFE184918F01882339F00F946F5586
:10FDF0000F5F1F4FF8018491F7CF609191157091BB
:10FE00009215809193159091941542E00F94F455BA
:10FE1000E7E2FFE184918F01882339F00F946F5559
:10FE20000F5F1F4FF8018491F7CF42E060E070E070
:10FE300080E990EC0F94F4550F946D56F2E0AF9674
:10FE4000FFAFAF9703C0AF961FAEAF971092BD152F
:10FE50001092BE151092BF151092C0151092C115C8
:10FE60001092C2151092C3151092C41524E6EB9699
:10FE70002FAFEB97A2961CAE1DAE1EAE1FAEA29783
:10FE80006A961CAE1DAE1EAE1FAE6A97CE010196DD
:10FE900064969FAF8EAF6497DE01AF5BBF4F6696EF
:10FEA000BFAFAEAF66976A966CAD7DAD8EAD9FADC0
:10FEB0006A970F94E5C2AA966CAF7DAF8EAF9FAFE5
:10FEC000AA976A966CAD7DAD8EAD9FAD6A970F9483
:10FED00073C5C457DF4F688379838A839B83CC586B
:10FEE000D040A2966CAD7DAD8EAD9FADA2970F9424
:10FEF000E5C2C057DF4F688379838A839B83C059EB
:10FF0000D040A2966CAD7DAD8EAD9FADA2970F9403
:10FF100073C5CC56DF4F688379838A839B83C4592A
:10FF2000D0406496EEADFFAD649720E411922A951F
:10FF3000E9F76696AEADBFAD6697E0E11D92EA9532
:10FF4000E9F780E090E00F947C4A8091BD15909194
:10FF5000BE15A091BF15B091C015C655DF4F88835F
:10FF60009983AA83BB83CA5AD0408091C1159091CE
:10FF7000C215A091C315B091C415C255DF4F888337
:10FF80009983AA83BB83CE5AD040DE01AF5BBF4FBB
:10FF9000C856DF4FB983A883C859D040FE013196B7
:10FFA000AC96FFAFEEAFAC9700E0CC56DF4F888148
:10FFB0009981AA81BB81C459D040B058E6968CAFD4
:10FFC0009DAFAEAFBFAFE697C057DF4F8881998135
:10FFD000AA81BB81C059D040B058EA968CAF9DAF82
:10FFE000AEAFBFAFEA97C457DF4F88819981AA812E
:10FFF000BB81CC58D040B058C258DF4F888399831A
:020000021000EC
:10000000AA83BB83CE57D040AC962EAC3FACAC9706
:1000100010E06CE8462E65E1562E74E0772EC12C78
:10002000D12C7601013011F40C94338B113011F482
:100030000C943F8B002311F1023081F4D201119610
:100040002D913D914D915C911497C258DF4F68817D
:1000500079818A819B81CE57D0400BC0F2012581E6
:10006000368147815085EA966CAD7DAD8EAD9FADF2
:10007000EA970F9400B64B015C0106C0812C912CCD
:1000800050E8A52E5FE3B52E112301F1123081F463
:10009000D20111962D913D914D915C911497C258CA
:1000A000DF4F688179818A819B81CE57D0400BC018
:1000B000F2012581368147815085EA966CAD7DAD90
:1000C0008EAD9FADEA970F9400B604C060E070E07B
:1000D00080E89FE39B01AC01C501B4010F9400B619
:1000E0009B01AC01C701B6010F94FAC16B017C0101
:1000F0000023E1F11123D1F1023011F00C94138BA4
:10010000D20111962D913D914D915C911497AA9633
:100110006CAD7DAD8EAD9FADAA970F9400B64B012F
:100120005C01113011F40C942D8B123011F00C94F1
:10013000208BD20111962D913D914D915C91149798
:10014000AA966CAD7DAD8EAD9FADAA970F9400B60B
:100150009B01AC01C501B4010F9400B69B01AC0139
:10016000C701B6010F94FAC16B017C017A94F8E0E3
:100170004F0E511C711056CFD101CD92DD92ED92F0
:10018000FD921D011F5F143009F043CF3CE8232E80
:1001900035E1332EEEE5FFE16C96FFAFEEAF6C97E5
:1001A000CA57DF4F1882C658D040C456DF4F188256
:1001B000CC59D040C056DF4F1882C05AD04010E012
:1001C000002321F1013049F1023081F4D10111966F
:1001D0002D913D914D915C911497C258DF4F6881EC
:1001E00079818A819B81CE57D0400BC0F101258156
:1001F000368147815085EA966CAD7DAD8EAD9FAD61
:10020000EA970F9400B64B015C010AC0812C912C37
:1002100020E8A22E2FE3B22E03C0812C912C540192
:10022000D10111964D905D906D907C901497A30133
:100230009201AA966CAD7DAD8EAD9FADAA970F943D
:1002400000B66B017C01D10115968D919D910D90A9
:10025000BC91A02DA6968CAF9DAFAEAFBFAFA697B9
:100260006C96EEADFFAD6C9785919591A591B4918B
:10027000CC55DF4F88839983AA83BB83C45AD0406F
:10028000A6962CAD3DAD4EAD5FADA697CC56DF4FDB
:10029000688179818A819B81C459D0400F9400B6CE
:1002A0009B01AC01C701B6010F94F9C1C655DF4FE0
:1002B000288139814A815B81CA5AD0400F94FAC1A2
:1002C000CC55DF4F288139814A815B81C45AD040A7
:1002D0000F94F9C1A50194010F9400B6CA57DF4FDE
:1002E0002881C658D040C456DF4F3881CC59D04001
:1002F000C056DF4F4881C05AD040512F0F94FAC1E9
:10030000CA57DF4F688379838A839B83C658D0405E
:100310000023A9F00130B9F00230D9F0A6962CAD37
:100320003DAD4EAD5FADA697E6966CAD7DAD8EADA5
:100330009FADE6970F9400B66B017C010AC0C12CFB
:10034000D12C760106C0C12CD12C90E8E92E9FE378
:10035000F92E6C96EEADFFAD6C9734968590959026
:10036000A590B490A3019201C457DF4F68817981B1
:100370008A819B81CC58D0400F9400B62B013C0160
:10038000A6962CAD3DAD4EAD5FADA697C057DF4FE5
:10039000688179818A819B81C059D0400F9400B6D1
:1003A0009B01AC01C301B2010F94FAC1C255DF4FEA
:1003B000288139814A815B81CE5AD0400F94FAC19D
:1003C000A50194010F94F9C1A70196010F9400B6FD
:1003D000CA57DF4F288139814A815B81C658D04096
:1003E0000F94FAC1CA57DF4F6883C658D040C4562D
:1003F000DF4F7883CC59D040C056DF4F8883C05A36
:10040000D040192F6C96AEADBFAD6C9718966C9618
:10041000BFAFAEAF6C97B8E02B0E311CECEA2E16D6
:10042000E5E13E0609F0CCCEDC01CB01B058C85660
:10043000DF4FE881F981C859D04081939193A1930E
:10044000B193C856DF4FF983E883C859D0400F5F96
:10045000AC962EAD3FADAC97205F3F4FAC963FAF13
:100460002EAFAC97043009F0CFCD25968CAD9DAD65
:10047000AEADBFAD2597AA968CAF9DAFAEAFBFAF67
:10048000AA978D819E81AF81B885AE968CAF9DAFC6
:10049000AEAFBFAFAE9789859A85AB85BC85A69672
:1004A0008CAF9DAFAEAFBFAFA6978D859E85AF8554
:1004B000B889E6968CAF9DAFAEAFBFAFE6978981A6
:1004C0009A81AB81BC81EA968CAF9DAFAEAFBFAFD6
:1004D000EA9729968CAD9DADAEADBFAD2997C258B8
:1004E000DF4F88839983AA83BB83CE57D040898905
:1004F0009A89AB89BC89C457DF4F88839983AA83C3
:10050000BB83CC58D040898D9A8DAB8DBC8DC057A4
:10051000DF4F88839983AA83BB83C059D0408D8DD8
:100520009E8DAF8DB8A1CC56DF4F88839983AA8367
:10053000BB83C459D0408D899E89AF89B88DC85678
:10054000DF4F88839983AA83BB83C859D0402D96F7
:100550008CAD9DADAEADBFAD2D97CA57DF4F888333
:100560009983AA83BB83C658D04089A19AA1ABA125
:10057000BCA1C456DF4F88839983AA83BB83CC591F
:10058000D0408DA19EA1AFA1B8A5C056DF4F8883F2
:100590009983AA83BB83C05AD0408DA59EA5AFA5E1
:1005A000B8A9CC55DF4F88839983AA83BB83C45AEB
:1005B000D04089A59AA5ABA5BCA5CE54DF4F8883B2
:1005C0009983AA83BB83C25BD04061968CAD9DADFD
:1005D000AEADBFAD6197CA54DF4F88839983AA83BC
:1005E000BB83C65BD04089A99AA9ABA9BCA9C65454
:1005F000DF4F88839983AA83BB83CA5BD0408DA9D0
:100600009EA9AFA9B8ADC254DF4F88839983AA834E
:10061000BB83CE5BD04089AD9AADABADBCADCE5304
:10062000DF4F88839983AA83BB83C25CD040219625
:100630008CAD9DADAEADBFAD2197CA53DF4F888362
:100640009983AA83BB83C65CD04014E6C12CD12C0D
:1006500076014601570126013701A3019201AE96AA
:100660006CAD7DAD8EAD9FADAE970F9400B69B0186
:10067000AC01AA966CAD7DAD8EAD9FADAA970F94DF
:10068000F9C12B013C01A5019401A6966CAD7DAD8D
:100690008EAD9FADA6970F9400B69B01AC01C30130
:1006A000B2010F94F9C12B013C01A7019601E69616
:1006B0006CAD7DAD8EAD9FADE6970F9400B69B01FE
:1006C000AC01C301B2010F94F9C1EA962CAD3DAD66
:1006D0004EAD5FADEA970F94E8C26E966CAF7DAFFA
:1006E0008EAF9FAF6E97C457DF4F288139814A8103
:1006F0005B81CC58D0400F9400B69B01AC01C2582E
:10070000DF4F688179818A819B81CE57D0400F94D9
:10071000F9C12B013C01A5019401C057DF4F68814D
:1007200079818A819B81C059D0400F9400B69B018A
:10073000AC01C301B2010F94F9C14B015C01A701E7
:100740009601CC56DF4F688179818A819B81C4599B
:10075000D0400F9400B69B01AC01C501B4010F94C9
:10076000F9C1C856DF4F288139814A815B81C85958
:10077000D0400F94E8C22B013C01C456DF4F2881C2
:1007800039814A815B81CC59D0406E966CAD7DAD8C
:100790008EAD9FAD6E970F9400B69B01AC01CA570A
:1007A000DF4F688179818A819B81C658D0400F9440
:1007B000F9C14B015C01C056DF4F288139814A8164
:1007C0005B81C05AD040C301B2010F9400B69B01B7
:1007D000AC01C501B4010F94F9C14B015C01A70143
:1007E0009601CC55DF4F688179818A819B81C45AFB
:1007F000D0400F9400B69B01AC01C501B4010F9429
:10080000F9C1CE54DF4F288139814A815B81C25BB7
:10081000D0400F94E8C24B015C01C654DF4F2881E1
:1008200039814A815B81CA5BD0406E966CAD7DADEB
:100830008EAD9FAD6E970F9400B69B01AC01CA546C
:10084000DF4F688179818A819B81C65BD0400F949C
:10085000F9C16B017C01C254DF4F288139814A8183
:100860005B81CE5BD040C301B2010F9400B69B0107
:10087000AC01C701B6010F94F9C16B017C01CE53E5
:10088000DF4F288139814A815B81C25CD040C5013C
:10089000B4010F9400B69B01AC01C701B6010F94DF
:1008A000F9C1CA53DF4F288139814A815B81C65C17
:1008B000D0400F94E8C26B017C01115009F0CDCEFD
:1008C0006E962CAD3DAD4EAD5FAD6E97C655DF4F0C
:1008D000688179818A819B81CA5AD0400F94FAC17C
:1008E0006093BD157093BE158093BF159093C0158E
:1008F000A3019201C255DF4F688179818A819B8172
:10090000CE5AD0400F94FAC16093C1157093C215AE
:100910008093C3159093C415A50194016A966CAD9C
:100920007DAD8EAD9FAD6A970F94FAC16A966CAF9C
:100930007DAF8EAF9FAF6A97A7019601A2966CAD6F
:100940007DAD8EAD9FADA2970F94FAC1A2966CAF0C
:100950007DAF8EAF9FAFA297EB969FADEB97915077
:10096000EB969FAFEB9791119ECA6A966CAD7DADE9
:100970008EAD9FAD6A970F94E5C26093AD157093ED
:10098000AE158093AF159093B0156A966CAD7DADA2
:100990008EAD9FAD6A970F9473C56093B115709338
:1009A000B2158093B3159093B415A2966CAD7DAD3E
:1009B0008EAD9FADA2970F9473C5DC01CB01B058EB
:1009C0008093B5159093B615A093B715B093B8154D
:1009D000A2966CAD7DAD8EAD9FADA2970F94E5C292
:1009E0006093B9157093BA158093BB159093BC159D
:1009F0006A962CAD3DAD4EAD5FAD6A97A2966CADDB
:100A00007DAD8EAD9FADA2970F94F9C16B017C01B6
:100A1000E894F7F8B701A60180E69FE00F9492C131
:100A20002FE132E449E05BE3C701B6010F9445C40E
:100A300018166CF425E33AEF4EE85BE3C701B60104
:100A40000F9445C4181634F001E010E005C000E032
:100A500010E002C002E010E025E33AEF4EE85BE36D
:100A60006A966CAD7DAD8EAD9FAD6A979F770F9402
:100A700045C418167CF025E33AEF4EE85BE3A296F6
:100A80006CAD7DAD8EAD9FADA2979F770F9445C4A1
:100A9000181614F402E010E08091AD159091AE1597
:100AA000A091AF15B091B015AE968CAF9DAFAEAF23
:100AB000BFAFAE978091B5159091B615A091B715BF
:100AC000B091B815A6968CAF9DAFAEAFBFAFA6974D
:100AD0008091BD159091BE15A091BF15B091C01524
:100AE000EE968CAF9DAFAEAFBFAFEE978091B115D4
:100AF0009091B215A091B315B091B415E6968CAF54
:100B00009DAFAEAFBFAFE6978091B9159091BA1582
:100B1000A091BB15B091BC15EA968CAF9DAFAEAF5E
:100B2000BFAFEA978091C1159091C215A091C315EE
:100B3000B091C415C258DF4F88839983AA83BB83C1
:100B4000CE57D040AEE5BFE16C96BFAFAEAF6C976D
:100B50008CE8282E85E1382EF10181809280A380D7
:100B6000B48085819681A781B085AA968CAF9DAF10
:100B7000AEAFBFAFAA976C96EEADFFAD6C97C590C8
:100B8000D590E590F490A5019401AE966CAD7DAD45
:100B90008EAD9FADAE970F9400B62B013C01AA9687
:100BA0002CAD3DAD4EAD5FADAA97A6966CAD7DADBB
:100BB0008EAD9FADA6970F9400B69B01AC01C3010B
:100BC000B2010F94FAC1EE962CAD3DAD4EAD5FADC6
:100BD000EE970F94FAC19B01AC01C701B6010F94C7
:100BE000F9C16B017C016C96EEADFFAD6C9734964C
:100BF0004590559065907490E6962CAD3DAD4EAD08
:100C00005FADE697C501B4010F9400B64B015C01DE
:100C1000EA962CAD3DAD4EAD5FADEA97AA966CADB0
:100C20007DAD8EAD9FADAA970F9400B69B01AC0130
:100C3000C501B4010F94FAC1C258DF4F2881398130
:100C40004A815B81CE57D0400F94FAC19B01AC0121
:100C5000C301B2010F94F9C14B015C01A7019601D8
:100C6000C701B6010F9400B66B017C01A501940188
:100C7000C501B4010F9400B69B01AC01C701B601D8
:100C80000F94FAC10F947EC52DEC3CEC4CE45FE36D
:100C90000F9445C4181614F40EEF1FEFB8E02B0E96
:100CA000311C6C96EEADFFAD6C9738966C96FFAF2D
:100CB000EEAF6C972CEA35E12215330509F04CCFE5
:100CC0000115110509F07AC1A2962CAD3DAD4EADCE
:100CD0005FADA2976A966CAD7DAD8EAD9FAD6A9704
:100CE0000F94FAC120E030E040E05FE30F9400B6DB
:100CF0006B017C010F94E5C22B013C016093AD15A3
:100D00007093AE158093AF159093B015C701B601DF
:100D10000F9473C5A2966CAF7DAF8EAF9FAFA297B5
:100D20006093B1157093B2158093B3159093B41579
:100D3000DC01CB01B058AA968CAF9DAFAEAFBFAF70
:100D4000AA978093B5159093B615A093B715B09355
:100D5000B8154092B9155092BA156092BB157092B1
:100D6000BC151092BD151092BE151092BF151092B1
:100D7000C0151092C1151092C2151092C315109291
:100D8000C4156E961CAE1DAE1EAE1FAE6E976A9653
:100D90001CAE1DAE1EAE1FAE6A97CE57DF4FA881A8
:100DA000B981C258D04011968D909D90AD90BC9065
:100DB000149715968D919D910D90BC91A02DAE9696
:100DC0008CAF9DAFAEAFBFAFAE97C657DF4FE881D8
:100DD000F981CA58D040C590D590E590F490A5010E
:100DE0009401C301B2010F9400B6A6966CAF7DAF1B
:100DF0008EAF9FAFA697AE962CAD3DAD4EAD5FAD1D
:100E0000AE97AA966CAD7DAD8EAD9FADAA970F94AF
:100E100000B69B01AC01A6966CAD7DAD8EAD9FADCD
:100E2000A6970F94FAC19B01AC01C701B6010F94BC
:100E3000F9C12091BD153091BE154091BF1550915B
:100E4000C0150F94FAC16B017C016093BD157093BE
:100E5000BE158093BF159093C01520E030E040E8A8
:100E60005FE36A966CAD7DAD8EAD9FAD6A970F94D2
:100E7000FAC16A966CAF7DAF8EAF9FAF6A97C657C7
:100E8000DF4FE881F981CA58D04034968591959119
:100E9000A591B491A6968CAF9DAFAEAFBFAFA6970C
:100EA000A5019401A2966CAD7DAD8EAD9FADA297CC
:100EB0000F9400B64B015C01AE962CAD3DAD4EAD2E
:100EC0005FADAE97C301B2010F9400B69B01AC01B8
:100ED000C501B4010F94FAC19B01AC01A6966CAD9B
:100EE0007DAD8EAD9FADA6970F94F9C12091C11530
:100EF0003091C2154091C3155091C4150F94FAC199
:100F00004B015C016093C1157093C2158093C315AA
:100F10009093C41520E030E040E85FE36E966CAD3E
:100F20007DAD8EAD9FAD6E970F94FAC16E966CAF8E
:100F30007DAF8EAF9FAF6E97CE57DF4FA881B9813F
:100F4000C258D0401896CE57DF4FB983A883C258F5
:100F5000D040C657DF4FE881F981CA58D040389653
:100F6000C657DF4FF983E883CA58D0402A163B069C
:100F700009F013CF6A962CAD3DAD4EAD5FAD6A97CB
:100F8000C701B6010F94E8C26093BD157093BE15FA
:100F90008093BF159093C0156E962CAD3DAD4EADB0
:100FA0005FAD6E97C501B4010F94E8C26093C1159F
:100FB0007093C2158093C3159093C4154090AD15DE
:100FC0005090AE156090AF157090B015C090B915E7
:100FD000D090BA15E090BB15F090BC158091B1157A
:100FE0009091B215A091B315B091B415A2968CAFA3
:100FF0009DAFAEAFBFAFA2978091B5159091B615DA
:10100000A091B715B091B8156A968CAF9DAFAEAFF1
:10101000BFAF6A97A7019601C301B2010F9400B652
:101020004B015C016A962CAD3DAD4EAD5FAD6A974C
:10103000A2966CAD7DAD8EAD9FADA2970F9400B61C
:101040009B01AC01C501B4010F94F9C14B015C01D6
:101050009B01AC01C701B6010F94E8C26B017C0192
:101060006A966CAD7DAD8EAD9FAD6A979058A50127
:1010700094010F94E8C26A966CAF7DAF8EAF9FAFBC
:101080006A97A2966CAD7DAD8EAD9FADA29790583C
:10109000A50194010F94E8C2CE57DF4F688379838E
:1010A0008A839B83C258D040A5019401C301B20139
:1010B0000F94E8C24B015C014090BD155090BE15E5
:1010C0006090BF157090C0158091C1159091C215A8
:1010D000A091C315B091C415A2968CAF9DAFAEAFD1
:1010E000BFAFA297C092AD15D092AE15E092AF15EA
:1010F000F092B015CE57DF4F88819981AA81BB81CC
:10110000C258D0408093B1159093B215A093B315F7
:10111000B093B4156A968CAD9DADAEADBFAD6A9778
:101120008093B5159093B615A093B715B093B815E5
:101130008092B9159092BA15A092BB15B092BC15C9
:10114000C701B6019058A30192010F9400B66B013C
:101150007C01A2962CAD3DAD4EAD5FADA2976A96D7
:101160006CAD7DAD8EAD9FAD6A970F9400B69B01BF
:10117000AC01C701B6010F94F9C16093BD1570931E
:10118000BE158093BF159093C015CE57DF4F688171
:1011900079818A819B81C258D0409058A3019201E5
:1011A0000F9400B66B017C01A2962CAD3DAD4EAD07
:1011B0005FADA297C501B4010F9400B69B01AC01CD
:1011C000C701B6010F94F9C16093C1157093C215A0
:1011D0008093C3159093C41580E090E00F947C4AEF
:1011E00017FD53C04DEB55E165EB75E18DEA95E1D7
:1011F0000E944BEC4091BD155091BE156091BF15FA
:101200007091C01585EE9FE00F9492C14091C11579
:101210005091C2156091C3157091C41589EE9FE07D
:101220000F9492C14091AD155091AE156091AF15DC
:101230007091B0158DED9FE00F9492C14091B11562
:101240005091B2156091B3157091B41581EE9FE085
:101250000F9492C14091B5155091B6156091B71594
:101260007091B81585ED9FE00F9492C14091B9152A
:101270005091BA156091BB157091BC1589ED9FE036
:101280000F9492C10E94D0EB09C00E3F9FEF190747
:1012900029F4AF96AFADAF97A23049F038010BC03B
:1012A000AF961FAEAF9766246A94762C04C0BEEF4B
:1012B0006B2E77247A94C855DF4F88819981C85A5C
:1012C000D0400F94FA6380E090E0A0EAB0E480930D
:1012D0005E1090935F10A0936010B0936110209106
:1012E0005A1030915B1040915C1050915D106091EC
:1012F0005610709157108091581090915910E6E057
:10130000FDE0FF93EF93812C912CE0EAAE2EE1E417
:10131000BE2EF2E6CF2EF0E1DF2EE12CF12C00EA1A
:1013200010E40F942D270F94CB8E0F900F9077FC25
:1013300022C020E030E046E153E460915E107091FD
:101340005F1080916010909161100F94FAC16093CA
:101350005E1070935F10809360109093611065E54C
:1013600075E585E591E40E9462EB86EA9AE10E94C8
:101370009AD40E9470F381E00E9442F882E00E94B9
:1013800066F0BFEF6B167B0631F489E69AE10E94A6
:101390009AD410E04BC0EEEF6E16EFEF7E0681F4AC
:1013A000AF96FFADAF97FF2329F0F23031F082E224
:1013B00099E1EDCF87EA99E1EACF87E699E1E7CFB6
:1013C000AF962FADAF97211107C033E063167104BC
:1013D00098F087EA99E117C0AF966FADAF9762308A
:1013E00019F484E29AE102C08AED99E10E949AD44C
:1013F0001614170454F309C0F301EE0FFF1FE05356
:10140000FD4F808191810E949AD46720609409F2F7
:1014100086EE0F94F6678FE59FE00F946EC18130E2
:1014200021F08BEC9AE10E949AD411E00E94EDBF6A
:101430002BC18AE89FE10E949AD410E025C183E085
:10144000821B282F0C94E77881E00C94467AF0E90F
:10145000CF1AF1E0DF0A0C948879E7968FADE79711
:10146000E8969FADE8970C94277B8E7F0C94737B56
:1014700080E4482E512C612C712C0C94897B87E1DF
:1014800090E00C949D7B8F3F910509F014F40C942F
:10149000A57B8FEF90E00C94A57B8B7F0C94AD7BAC
:1014A000B0E6EB16B9E0FB0614F00C94BC7B84E0CC
:1014B0000F94A25AEFEFEE1AFE0A0C94BC7BC60101
:1014C0000C94DC7B8150883011F00C94B57C0C942A
:1014D000BC7C00E00C94CA7C80E090E00C94EF7C33
:1014E000EBE0BE1611F40C94657D222311F02B3035
:1014F00039F4E396FFADE397F83010F00C946B7D70
:10150000B101620F731F6257784FFB01F081A39600
:10151000FFAFA397E896EEADFFADE897C080D1800E
:1015200061E070E0022E02C0660F771F0A94E2F7B6
:101530006C217D21672B31F0A396FFADA397F1318C
:1015400048F005C0A3966FADA397613118F40196DA
:101550000C946B7D01970C946B7D80E00C94F97D6D
:1015600084EF91E00F94CB08882311F40C94047E4F
:1015700014E0812C912C5401C12CD12C760188EEE1
:1015800093E00F94CB08882311F40C94047E80918F
:10159000461090914710A0914810B0914910092E23
:1015A000000CAA0BBB0BC80ED91EEA1EFB1E8091B5
:1015B0004A1090914B10A0914C10B0914D10092EF3
:1015C000000CAA0BBB0B880E991EAA1EBB1E115045
:1015D000B1F640904E1050904F10609050107090A7
:1015E0005110C501B40122E09695879577956795CE
:1015F0002A95D1F732E0F694E794D794C7943A95B8
:10160000D1F700E028EC30E0A201C6010F94850775
:1016100011E00C94057E29813A812059374F3A8395
:1016200029830C94467AF2012581368147815085C1
:10163000E6966CAD7DAD8EAD9FADE6970C948D803A
:10164000F2012581368147815085E6966CAD7DADEE
:101650008EAD9FADE6970C94A68060E070E080E8C8
:101660009FE30C94A880112311F40C94B680812C74
:10167000912C40E8A42E4FE3B42E0C9491800111DC
:101680000C947C800C94B68081E00E9442F880E04B
:101690000F94B56C812FC753DF4F0FB6F894DEBFA0
:1016A0000FBECDBFDF91CF911F910F91FF90EF90B3
:1016B000DF90CF90BF90AF909F908F907F906F9072
:1016C0005F904F903F902F90089560E080917A1541
:1016D0000F94D10661E080917A150F94D10660E0F5
:1016E00080917A150F94D1068BE891E00197F1F77C
:1016F0000895CF939C0140916E1550916F15809184
:101700007C1390917D134817590739F4E0917F13AA
:10171000F09180131E161F06A4F1C62FFC01E20FE4
:10172000F31FBF0163597F4F8417950728F481E0A9
:101730004617570738F525C06E3E714000F13496C4
:10174000EE3EF14018F449365105C8F423593F4F95
:1017500042175307B0F04DEE51E0481B590B60E0C3
:1017600070E08F579C4E0F941DC7CC2309F0F8945E
:1017700010927D1310927C13CC2309F0789481E0B1
:1017800001C080E0CF91089581E00F94EC800C942B
:1017900022F3CF92DF92EF92FF920F931F93CF939A
:1017A000DF939CEDE92E96E0F92EC0E0D0E0082F03
:1017B00010E0670161E0F70181917F010F94FF065E
:1017C000B8010C2E02C0759567950A94E2F7617016
:1017D000F60180810F94D1062196C430D10549F7D6
:1017E000DF91CF911F910F91FF90EF90DF90CF90FD
:1017F0006CCFCF92DF92EF92FF920F931F93CF9314
:10180000DF93182F80917B150F94D1068091791565
:101810008F3F19F060E00F94D10680917E15C12FA3
:10182000D0E084FF27C03CEDE32E36E0F32E00E04D
:1018300010E0670161E0F70181917F010F94FF06DD
:10184000BE01002E02C0759567950A94E2F761709B
:10185000F60180810F94D1060F5F1F4F08301105EC
:1018600041F7DF91CF911F910F91FF90EF90DF90A3
:10187000CF902BCFCE0124E0959587952A95E1F75F
:1018800088DF812FDF91CF911F910F91FF90EF9013
:10189000DF90CF907ECF60E0ACCF982F8A3071F48C
:1018A00080917C15843018F08FEF80937C156091C7
:1018B0007C156F5F80E00E9442F320C1E0917015BB
:1018C000E11104C08B3109F017C11BC0E230C8F030
:1018D000F0E0E059FA4E80838091711520ED290FD8
:1018E0002A3060F421E030E00090701502C0220F31
:1018F000331F0A94E2F78160822B01C08E7F8093B0
:1019000071154091701581E0840F8093701550E03F
:101910004830510508F0EDC0FA018827EC57FF4F19
:101920008F4F0D94E7C69B3109F0E3C0E7C01092DA
:1019300071159B3509F0DDC0E1C0923309F4DEC0BA
:101940009F3309F4DBC08091711570C080917215CE
:10195000823331F08F3359F4923309F0CAC0CEC0CC
:101960009A3429F40E9438F810927C15C2C08091F4
:10197000711582FFBEC09B3309F058C0BFC0809173
:1019800072158F3349F480917315823309F0B1C019
:10199000953309F0AEC0B2C08091711582FFA9C025
:1019A000209173152B3311F480FDA8C083FFA1C0D3
:1019B0009B3309F09EC0A2C0609172156F33F9F499
:1019C00080917315823309F094C08091741585332A
:1019D00009F08FC0983651F09C3609F08AC080918A
:1019E00078158D7F80937815886007C08091781571
:1019F000982F9260909378158A604DDF7AC080911D
:101A0000711582FF76C0209173152B3341F484FF4A
:101A100006C0983459F46053809174153CC083FF1C
:101A200068C0909174159B3309F063C080FF61C05A
:101A300065C02091711522FF5CC0809173158B33B6
:101A4000A1F4322F3073303381F4983471F4609103
:101A50007215605380917415880F8056982F990FD6
:101A6000990F890F9091751540C023FF42C03091A6
:101A700074153B33F1F525FF3CC0983471F4609147
:101A80007215660F6056962F990F990F690F805344
:101A9000680F8091751580532AC020FF2AC02EC080
:101AA00080917115282F2C702C3019F52091741508
:101AB0002B33F9F480768036E1F49834D1F46091D8
:101AC0007215660F6056862F880F880F680F8091F9
:101AD00073158053680F80917515880F8056982F65
:101AE000990F990F890F909176159053890F0E9445
:101AF00042F31092701502C061E07BDE81E0089530
:101B0000CCDE80E090E008951092CD1980912D0FE9
:101B10008B7F80932D0F089520914902222359F144
:101B2000FC01808D83FF03C07195619571098091DF
:101B3000A70E9091A80E680F791F7093A80E60935E
:101B4000A70E8091A90E9091AA0E6817790734F418
:101B5000919581959109861797076CF08091030103
:101B600084FF04C0809105018F7E03C08091050130
:101B70008061809305010895809149028823A9F02E
:101B800080910802882389F08091360D882369F0BE
:101B900084E192E20F94C6BB10922F0D1092360D85
:101BA00081E080932A021092270D08951092490235
:101BB00060E087E69FE00F9480C110924A0208958A
:101BC0001F920F920FB60F9211240BB60F921F9314
:101BD0002F933F934F935F936F937F938F939F9335
:101BE000AF93BF93CF93DF93EF93FF938091371021
:101BF000811107C18091900D811103C19091030162
:101C000080910F07892784FFFCC080910301809396
